:020000040100F9
:10000000D85C0020E5000001ED000001EF000001D8
:1000100000000000000000000000000000000000E0
:10002000000000000000000000000000F1000001DE
:100030000000000000000000F3000001F5000001D6
:10004000F7000001F7000001F7000001F7000001D0
:10005000F7000001F7000001F7000001F7000001C0
:10006000F7000001F7000001F7000001F7000001B0
:10007000F7000001F7000001F7000001F7000001A0
:10008000F7000001F7000001F7000001F700000190
:10009000F7000001F7000001F7000001F700000180
:1000A000F7000001F7000001F7000001F700000170
:1000B000F7000001F7000001F7000001F700000160
:1000C0000348854600F02EF900480047012500014D
:1000D000D85C002040BA7047C0BA70470138FDD1E3
:1000E000704700000448804704480047FEE7FEE7E9
:1000F000FEE7FEE7FEE7FEE7A9140001C1000001EC
:1001000030B50B46014600202022012409E00D46AF
:10011000D5409D4205D31D469540491B2546954037
:1001200040191546521E002DF1DC30BD03460B432D
:100130009B0703D009E008C9121F08C0042AFAD29D
:1001400003E00B780370401C491C521EF9D2704723
:10015000D2B201E00270401C491EFBD2704700225F
:10016000F6E710B513460A4604461946FFF7F0FFB6
:10017000204610BD421C0178401C0029FBD1801A8A
:10018000704710B5002200E0521C835C8C5CA342D7
:1001900001D1002BF8D1D8B2E1B2401A10BDC9B2DA
:1001A00003E003788B4203D0401C521EF9D200209A
:1001B000704730B504460020034600E05B1C9342C4
:1001C00003D2E05CCD5C401BF8D030BD03460A781A
:1001D0000270401C491C002AF9D11846704730B5FE
:1001E00005460020034600E05B1C934205D2EC5C10
:1001F000C85C201A01D1002CF6D130BDF7B582B011
:100200000F460026029C01F06FFA009000680190F2
:100210002578641C002D05D000F02CF80068405DA6
:10022000C007F5D12B2D02D02D2D1CD0641E0098B7
:100230000021016039462046049A00F01FF801466B
:10024000002F04D03868A04201D10298386000988D
:10025000006802280BD00098019A0260700506D54C
:10026000484205B0F0BD012080020643DFE70846A2
:10027000F7E70000004870474C350001F7B582B041
:10028000029C00272078641C15460197302802D074
:10029000002D15D015E020780127641C782804D0A3
:1002A000582802D0002D09D00BE0002D01D0102DD0
:1002B00007D1002710252078641C02E0082500E003
:1002C0000A250026009610E00099012769430818C6
:1002D000020C294680B2714300908E183804864281
:1002E00001D3012001902078641C294600F02CF8ED
:1002F0000028E9DA0398002805D0002F01D0641EF9
:1003000000E0029C04600198002806D001F0ECF99E
:1003100002210160C81E05B0F0BD009930040843F9
:10032000F9E70000064C0125064E05E0E36807CC1E
:100330002B430C3C98471034B442F7D3FFF7C4FE6C
:10034000C0380001E03800013A2800D230382023BC
:1003500002469A43412A01D310463738884201D3D6
:100360000020C04370470000F0B58DB006460F4630
:100370002C22444902A8FFF7D9FE02A801F0CEFEC4
:10038000002804D140A002F083F80DB0F0BD022E89
:100390000FDB01A9786802F0D9FC002805D101988B
:1003A00001280DD0019802280AD045A002F070F86B
:1003B000EBE70398012801D1022000E00120019021
:1003C00001990398884204D14CA0019901F092FF51
:1003D000DBE70198012801D104A800E008A8044641
:1003E0000198012801D14C4800E04C480090216858
:1003F0000098814207D16068002804D00721890352
:100400006068884206D96368226845A0019901F0B6
:1004100071FFBAE750A002F03BF86168206801F074
:100420008FFE0546A168A94209D02B46A26858480C
:10043000019901F05FFF57A002F02AF8A5E7636871
:10044000E26861A0019901F055FF0198039002A8AC
:1004500001F06EFD002803D06BA002F019F894E7BC
:100460006EA002F015F8C82001F076FC00BFBFF3C3
:100470004F8F71487149C860BFF34F8F00BF00BFF5
:10048000FEE700000040000161707073773A20625F
:100490006F6F7473657474696E67207265636F72D1
:1004A0006420696E76616C69642C20726566757370
:1004B0006520746F207377697463680D0A0000000B
:1004C00075736167653A206170707377205B317C6A
:1004D000325D20286E6F20617267203D207377693E
:1004E00074636820746F20746865206F7468657227
:1004F0002062616E6B290D0A00000000617070734C
:10050000773A20616C7265616479206F6E2041508A
:1005100050256C750D0A00000080000100400201AA
:1005200061707073773A2062616E6B256C75207212
:1005300065636F726420696E76616C6964202861FE
:100540006464723D30782530386C582073697A6560
:100550003D256C75290D0A0061707073773A20761D
:100560006572696679696E67207461726765742067
:10057000696D616765206372632028666577207303
:1005800065636F6E6473292E2E2E0D0A0000000025
:100590002C3800012020202020202072756E20425F
:1005A0004C45204F544120746F2077726974652048
:1005B000612076616C696420696D61676520666998
:1005C0007273740D0A00000061707073773A2062D4
:1005D000616E6B256C7520696D616765206F6B209E
:1005E000287665722030782530386C582C20256CA0
:1005F000752042292C20737769746368696E672EB1
:100600002E2E0D0A0000000061707073773A20668C
:100610006C617368206661696C0D0A0061707073AB
:10062000773A20646F6E652C207265736574746907
:100630006E672E2E2E0D0A000400FA0500ED00E074
:1006400030B58BB004460D462C2204496846FFF7AE
:100650006DFD684601F0ACFC0BB030BD0040000100
:1006600070B58CB006460C46032E0ADA53A001F092
:100670000FFF5AA001F00CFF5E4801F009FF0CB01B
:1006800070BD6946A06802F061FB002803D05AA043
:1006900001F0FEFEF3E72C225C4901A8FFF746FDBE
:1006A00001A801F03BFD002806D12C2101A8FFF78D
:1006B00056FD57A001F0ECFE63A16068FFF761FDF5
:1006C00000280CD10098012806D00098022803D0F9
:1006D0005FA001F0DDFED2E70098029058E060686C
:1006E0000078622850D160684078312803D0606873
:1006F0004078322848D160684078312801D103A879
:1007000000E007A805466168881C59A1FFF739FD7C
:1007100000280ED158490098884207D057490098C0
:10072000884203D056A001F0B3FEA8E700982860E5
:100730002EE06168881C61A1FFF723FD00280BD122
:10074000072189030098884203D95EA001F0A0FE2A
:1007500095E7009868601BE06168881C62A1FFF75C
:1007600010FD002802D10098A86011E06168881C83
:100770005EA1FFF706FD002802D10098E86007E0BF
:100780005BA001F085FE7AE759A001F081FE76E7D3
:1007900061685DA0009A01F0ADFD01A801F0C8FB01
:1007A000002803D061A001F073FE68E764A001F0A7
:1007B0006FFE01A801F0FCFB00BF60E77573616785
:1007C000653A206273736574203C6669656C643EAB
:1007D000203C76616C3E0D0A000000002020666916
:1007E000656C643A20616374697665203C317C32C3
:1007F0003E0D0A007438000162737365743A20621A
:1008000061642076616C75650D0A0000004000018E
:1008100062737365743A206578697374696E6720D2
:100820007265636F726420696E76616C69642C20F6
:1008300072656275696C642066726F6D2073637295
:10084000617463680D0A0000616374697665000075
:1008500062737365743A20616374697665206D759F
:1008600073742062652031206F7220320D0A0000FF
:100870006164647200000000008000010040020119
:1008800062737365743A2061646472206D75737469
:100890002062652043414949435F415050315F42E6
:1008A000415345206F722043414949435F415050B5
:1008B000325F424153450D0A0000000073697A65BA
:1008C0000000000062737365743A2073697A6520D2
:1008D00065786365656473207468652062616E6B1A
:1008E0002073697A650D0A00637263007665720091
:1008F00062737365743A20756E6B6E6F776E2066E7
:1009000069656C640D0A000062737365743A202592
:1009100073203D2030782530386C582C2077726950
:1009200074696E672E2E2E0D0A00000062737365C7
:10093000743A20666C617368206661696C0D0A0008
:1009400062737365743A206F6B20287665726966EE
:10095000696564290D0A0000F8B5164C164920682F
:10096000884208D12821204601F0EAFBA16A88428A
:1009700001D1012000E00020064665680FA112A009
:1009800001F0B8FC002E03D117A001F081FD022573
:10099000294620A001F0AEFC01F0EAF97D21C90052
:1009A0000090FFF7ADFB074639461FA001F0A2FCFF
:1009B000F8BD00000040000111C011CA56312E30B0
:1009C000302E303700000000626F6F746C6F61640E
:1009D00065723A2025732C20646F776E6C6F6164AA
:1009E000206D6F64650D0A00626F6F7473657474B7
:1009F000696E673A20494E56414C4944202D204F9C
:100A00005441207461726765747320415050310DF8
:100A10000A0000006375722062616E6B3A204150DB
:100A200050256C750D0A0000757074696D653A206B
:100A3000256C7520730D0A0070B506460D46022E12
:100A40001EDB002415E00C2262431B4B995868689A
:100A5000FFF797FB00280BD10C206043164BC01802
:100A600042680C206043195814A001F043FC70BD8B
:100A7000641C0A2CE7D314A0696801F03BFCF6E77C
:100A80001AA001F005FD1FA001F002FD00240BE0FB
:100A90000C206043084BC01842680C206043195872
:100AA00006A001F027FC641C0A2CF1D318A001F069
:100AB000EFFC00BFDBE70000203100012020252DE6
:100AC00038732025730D0A00756E6B6E6F776E207C
:100AD000636F6D6D616E643A20257320287472799E
:100AE000202768656C7027290D0A00006D6F64650A
:100AF0003A20424F4F5420646F776E6C6F61640DE3
:100B00000A000000636F6D6D616E64733A0D0A0038
:100B10006B6579733A20544142203D20636F6D70BC
:100B20006C6574652C2055502F444F574E203D2046
:100B3000686973746F72790D0A00000070B504461D
:100B40000D46034801F0A4FC01200249087070BD65
:100B5000503500010C40002070B588B005460C46A9
:100B6000002007900690022D04DA3EA001F090FCD0
:100B700008B070BD06AA07A9606802F0FFF8002857
:100B800004D145A0616801F0B5FBF1E74D49079834
:100B9000884204D10121042000F08CFB03E00121F4
:100BA000082000F087FB032D4ADB4649079888425E
:100BB00005D16846008B30210840002809D1424900
:100BC0000798884208D16846008BC0210840002859
:100BD00002D03EA001F05CFC684600F07DFA684659
:100BE000008B0090012001906946079800F0F0F911
:100BF000A068007831280DD1A0684078002809D17C
:100C00006846018B079800F081FA3FA0616801F007
:100C100071FB25E0A068007830280DD1A0684078ED
:100C2000002809D16846018B079800F06DFA39A0B9
:100C3000616801F05FFB13E039A001F029FC0FE0CF
:100C40006846018B079800F055FA002801D0012072
:100C500000E00020064632463DA0616801F04AFBF4
:100C600000BF85E775736167653A2070696E7365CB
:100C700074203C70784E3E205B307C315D2020201B
:100C800028652E672E2070696E736574207062303F
:100C90002031290D0A0000006261642070696E3AFB
:100CA0002025732028757365207061302E2E7061A9
:100CB00036202F207062302E2E70623133290D0ABB
:100CC0000000000000080140000C01407761726ED6
:100CD000696E673A205357442F636F6E736F6C656C
:100CE0002070696E202D207265636F6E666967756E
:100CF0007265206D617920627265616B2074686530
:100D0000206C696E6B0D0A002573203D20310D0AA1
:100D1000000000002573203D20300D0A0000000077
:100D200075736167653A2070696E736574203C70F5
:100D3000784E3E205B307C315D20202028303D6C99
:100D40006F772C20313D68696768290D0A00000023
:100D50002573203D2025750D0A00000008A001F034
:100D600097FBC82000F0F8FF00BFBFF34F8F084883
:100D70000849C860BFF34F8F00BF00BFFEE7000007
:100D8000726573657474696E672E2E2E0D0A0000ED
:100D90000400FA0500ED00E070B504460D4605A01C
:100DA00001F076FB0BA001F073FB17A001F070FBC4
:100DB00070BD00007573617274313A2054583D5013
:100DC00042362052583D5042372028414634290DA2
:100DD0000A000000626175643A20343630383030E1
:100DE0002C2038206461746120626974732C206E39
:100DF0006F207061726974792C20312073746F7068
:100E0000206269740D0A0000666C6F7720636F6E54
:100E100074726F6C3A206E6F6E653B2074783A2066
:100E2000706F6C6C65643B2072783A20444D4120B1
:100E300072696E672028334B422C20706F6C6C6592
:100E400064290D0A0000000070B504460D4605A196
:100E500007A001F04FFA1148016811A001F04AFA09
:100E600070BD000056312E30302E303700000000AB
:100E7000626F6F746C6F61646572207665727369FE
:100E80006F6E3A2025732028646F776E6C6F6164F3
:100E9000206D6F6465290D0A0000000000400020ED
:100EA00053797374656D436F7265436C6F636B2028
:100EB0003D20256C7520487A0D0A00000168254AFE
:100EC000114001600021016041608160C1602249E0
:100ED000884208D12049083949680F2211431E4A27
:100EE000083A516035E01C491431884208D11A494A
:100EF00008394968F0221143174A083A516028E03E
:100F000015492831884209D11349083949680F2207
:100F100012021143104A083A51601AE00E493C315E
:100F2000884209D10C49083949680F22120311433C
:100F3000094A083A51600CE007495031884208D10B
:100F40000549083949680F2212041143024A083A38
:100F500051607047FEFF000008000240002904D0E5
:100F6000026801231A43026003E00268014B1A4041
:100F700002607047FEFF00000146486880B270477B
:100F800010B5002202680D4B1A400C6A8B6823438F
:100F90000C6923434C6923438C692343CC69234365
:100FA0004C6A23438C6A23431A430260CB68436034
:100FB0000B6883604B68C36010BD00000F80FFFFAB
:100FC00010B5002B01D0106101E00024146110BDA8
:100FD00070B503460A4600210024002076E0012671
:100FE0008E40156835402C46002C6ED05568022D79
:100FF00002D05568122D20D108250D40002D0ED0AD
:10100000586A4D07EE0E0F25B5400646AE433046F2
:101010004E07F60E5569B540284358620DE0186A30
:101020004D07EE0E0F25B5400646AE4330464E073F
:10103000F60E5569B540284318625568012D08D051
:101040005568112D05D05568022D02D05568122D16
:101050000BD1586801258D400646AE4330461579C0
:10106000ED06ED0F8D402843586018684E000325AB
:10107000B5400646AE4330461579AD07AD0F4E007C
:10108000B54028431860D8684E000325B540064691
:10109000AE4330464E009568B5402843D860986806
:1010A00001258D400646AE433046D5688D40284325
:1010B0009860D86A4E000125B5400646AE433046DA
:1010C0004E001569B5402843D862491C1568CD40CB
:1010D000002D84D170BD0000054901600F214161E0
:1010E0000021416081600121C160002101617047E0
:1010F000FF3F00000246002013690B40002B01D087
:10110000012000E0002070478162704781617047D4
:10111000F7B5D4B004460E460020539005205290F7
:101120000025002700BFEFF310800090FF2145311C
:1011300001A8FFF714F801F087FE05462448854210
:1011400018D101200003844202D1002053902AE0EC
:1011500001204003844202D14011539023E0032038
:101160000003844203D10120400253901BE05298B7
:1011700057B0F0BD1748854213D1012000038442C7
:1011800001D153900FE001204003844201D15390DC
:1011900009E003200003844201D1539003E05298F8
:1011A000E6E75298E4E705AF0137FF2241320A49EA
:1011B00001A8FEF7BBFF012000F0A9FA3146569ABC
:1011C0005398B8475290009800F0A1FA5298CFE790
:1011D000C440130085601300462F000170B504461B
:1011E000002500BF00BFEFF310800546012000F08E
:1011F00091FA00BF01200006241A2046054909681B
:101200008847064600BF284600F084FA00BF3046F3
:1012100070BD00005040002010B508480849086023
:10122000943008490860FF382D3807490860C92202
:10123000920006490938FEF779FF10BD4D52002093
:10124000504000205440002058400020A4310001AC
:10125000F8B504460D461646002700BF00BFEFF361
:1012600010800746012000F055FA00BF012000065B
:10127000241A324629462046054B1B6898470090A1
:1012800000BF384600F046FA00BF0098F8BD0000E5
:1012900054400020002905D0054A52690243044BFE
:1012A0005A6104E0024A52698243014B5A61704715
:1012B00000100240002905D0054A92690243044B00
:1012C0009A6104E0024A92698243014B9A61704735
:1012D0000010024010B500210022214B5B6804245D
:1012E00023401946002902D0042906D102E01D4BF3
:1012F000036005E01C4B036002E01A4B036000BF73
:1013000000BF174B5B683024234019460909174B6F
:101310005A5C0368D3404360114B5B680724240286
:1013200023401946090A124B5A5C4368D340836034
:101330000B4B5B68E40023401946C90A0C4B5A5C0E
:101340004368D340C360064BDB6A10242340002B64
:1013500002D0084B036102E07D23DB03036110BD73
:10136000001002400090D0030048E801A0310001C5
:101370009831000100093D00F1B58AB000200990C4
:101380007D20C00008900125AD02002700200790B5
:101390007F20069040240026002005900390200125
:1013A0000290002001903E490A98884206D83D48A4
:1013B0000068610288433B49086006E039480068DC
:1013C0000121C9030843374908607D21C9000A98F3
:1013D000FEF796FE7D21C9000090FEF791FE4501C3
:1013E00000BF304800687F21090288430190200235
:1013F000019908432B4908600520FEF76FFE10E0B5
:101400000120FEF76BFE2748406B022108400028B0
:1014100000D007E00598411C05910899884200D941
:1014200000E0EDE700BF1F48C06B86B2AE4201D9B5
:10143000771B00E0AF1B0298874203D2E0B2039013
:10144000B8B20290AE4201D3069400E00794069928
:1014500007984018C005000E04900498A04200D1DF
:1014600003E0049C09988742BBD800BF0D48006880
:101470007F210902884301900398000201990843E3
:10148000084908600846406840084000486000BFBE
:1014900004484068042108400028F9D10BB0F0BD91
:1014A0000090D0030010024010B53E48C0690121F1
:1014B000090708433B49C861812000063A4908638F
:1014C0003A4848613A4808623A480068032189036B
:1014D0008843384908603421374800F073F83648AB
:1014E0000069401C002803D033480069002817D148
:1014F0002C4840680121090408432A4948600846ED
:101500004068072109028843264948600846406828
:1015100009150843234948602848FFF72DFF3FE09D
:10152000214880694409640123480078C006C00E40
:1015300004431D4884611B4800680121C903884396
:1015400018490860084600687F210902884304465C
:1015500019480069000220431249086008464068A3
:101560000121090408430F494860084640680721E3
:10157000090288430B49486008464068091508433A
:10158000084948600846006A0D4908400549086254
:101590000846006A0849C968090208430149086207
:1015A00010BD000000100240007000400F08000055
:1015B0001800020000100140604000200090D0039D
:1015C000FF00F8FF70B504460D462A46214601206B
:1015D0000003FFF79DFD70BD002905D0828901231E
:1015E0005B031A43828103E08289024B1A408281A5
:1015F00070470000FFDF0000002A03D0838A0B43FE
:10160000838202E0838A8B438382704702460020F4
:1016100001235B02994200D100BF13880B40002BCD
:1016200001D0012000E0002070470000F0B589B033
:1016300005460E4600240020089000BF00BF00278A
:10164000B089002800D000BF2F462C8A20480440D3
:10165000F08804432C82AC891E480440B08831894C
:101660000843718908430443AC81AC8A1A4804409A
:10167000B0890443AC8201A8FFF72CFE17488742CB
:1016800002D10498089001E0039808903268910014
:101690001923089A5A431046FEF732FD0790642139
:1016A0000798FEF72DFD04012109642041430798A6
:1016B000411A069106990901084632306421FEF765
:1016C0001FFD0007000F04432C8109B0F0BD00008E
:1016D000FFCF0000F3E90000FFFC000000380140EC
:1016E000CA05D20D82807047004870475C400020D8
:1016F00002E008C8121F08C1002AFAD170477047DB
:10170000002001E001C1121F002AFBD1704780F3C5
:101710001088704780F31088704700000020074948
:1017200008700749086007490860074908600749C9
:10173000086007490870074908707047104000208A
:1017400024400020284000202C400020344000206D
:101750004440002045400020002002490870024912
:10176000088070474C40002048400020F7B584B006
:101770000746494906980860002686E0BC5D474850
:101780000078002804D0012810D0022874D13AE053
:10179000CA2C0AD142480470012042490880052021
:1017A0004149088001203D4908706BE03D480188AF
:1017B0000088401C3B4A1080394844541046008839
:1017C00005281FD13649C978354A127912021143CA
:1017D0000846FF21E131884205D900212F4A1170C6
:1017E000304A11800DE0C11D2F4A11801146098831
:1017F0002C4A1288914201D1002100E00221274A9F
:10180000117000BF3EE0274801880088401C254A2F
:101810001080234844541046008823490988884290
:1018200028D11F48C0781E49097909020843054696
:10183000281D81B21A48401C00F024FF0390681D47
:101840001749095CA81D164A105C00020143029169
:1018500002990398884207D11046817840782B4638
:10186000521D019000F034F800200C4908700D4919
:10187000088000BF06E0FFE700200849087009491A
:10188000088000BF00BF701C86B20598864200DA4F
:1018900074E707B0F0BD0000404000204C4000203D
:1018A000C44F0020484000204A40002031B5064A7D
:1018B00001216846FFF75AFF0448047800200349D5
:1018C0000870204638BD0000652C0001464000200D
:1018D000F8B504460D4616461F46102C06D0112CAE
:1018E0000AD0122C0ED0132C24D111E03A463146E6
:1018F000284600F00DFF1EE03A463146284600F02B
:10190000BFFF18E03A463146284601F08DF812E054
:10191000FFF704FF0948002213210368284601F05D
:1019200063F9074800680749884202D10120064947
:10193000087000E000BF00BFF8BD00002440002098
:1019400040400020652C00014640002010B51148A1
:10195000007800281CD000F00BFA0F490968441ADF
:101960000E480078002803D0FF202D30844203D297
:101970007D20000184420AD300BFBFF34F8F084887
:101980000849C860BFF34F8F00BF00BFFEE700BF2C
:1019900010BD00003A4000203C40002039400020AB
:1019A0000400FA0500ED00E0F8B507460D4638469C
:1019B000FEF7E0FB84B20BA000F06AFD002604E015
:1019C0000BA000F065FD701C86B2AE42F8DB05A0EE
:1019D00000F05EFD002C03D02146384600F090FA5E
:1019E0002046F8BD0D63616969632D3E000000006B
:1019F000200000000EB5002400270026651E0020F0
:101A00000290684800F044FD00BFFFF79FFF664862
:101A10000078002810D000F0ABF90299401A634911
:101A2000884209D9002060490870FFF795FE60A040
:101A300000F02EFD0024002701A800F035FA002850
:101A400000D1E2E758480078002811D000F090F962
:101A5000029068460079FFF729FF002807D0002090
:101A6000514908705CA000F013FD00240027CCE76A
:101A7000012E08D1684600795B2801D1022000E0E0
:101A800000200646C1E7022E3BD1002668460079B9
:101A9000412817D1681C5B490978884230DA6D1CEF
:101AA000284600F011FC014600905748FEF78EFBD7
:101AB00039465548FFF778FF07465348FEF75AFB6B
:101AC00084B21DE068460079422819D1002D17DB49
:101AD0006D1E002D08DB284600F0F6FB0146009045
:101AE0004948FEF773FB02E0002047490870394679
:101AF0004548FFF759FF07464348FEF73BFB84B2D2
:101B000083E7684600790D280ED006DC08281FD030
:101B1000092827D00A282CD107E01B2802D07F28CB
:101B200027D116E001263BE000BF38A000F0B0FC52
:101B3000002035490855084600F08AFB324800F07D
:101B400021FB00240027651E21A000F0A1FC27E056
:101B500000BF002C05D0601E84B22DA000F098FCC0
:101B600027461DE02146284800F054F80446274641
:101B700016E068460079202811D3684600797F284E
:101B80000DD24F2C0BD2684602792046611C8CB2D4
:101B90001D490A54012101A800F0B2F9274600BFEF
:101BA00000BF32E7C03600010C400020B80B000037
:101BB0000D0A5B6F74615D2062696E617279206DE0
:101BC0006F6465204F4646202869646C65290D0ABC
:101BD00063616969632D3E000D0A5B6F74615D206E
:101BE00062696E617279206D6F6465204F46462090
:101BF0002861626F7274290D0A63616969632D3E01
:101C0000000000000D400020744F00200D0A00006D
:101C100008200800F0B597B007460C4600250020C4
:101C20000290224620213846FEF7B9FA002802D059
:101C3000204617B0F0BD0020385500262AE00C20C1
:101C40007043414908580190224639460198FEF7F1
:101C5000C6FA00281DD10298002808D103A80199CE
:101C6000FEF7B4FA03A8FEF785FA85B20EE001E0AC
:101C7000681E85B2A54206DD2A4603A80199FEF733
:101C8000AEFA0028F4D1002003A948550298401C60
:101C90000290761C0A2ED2D30298002801D1204649
:101CA000C7E70298012819D109E003A90819012101
:101CB00000F026F903A8005D3855601C84B24F2C53
:101CC00001D2AC42F1DB4F2C06D220203855601CEB
:101CD00084B21EA000F0DCFB2046AAE7A5420FDD7F
:101CE00009E003A90819012100F00AF903A8005D21
:101CF0003855601C84B24F2C23D2AC42F1DB20E07B
:101D000013A000F0C5FB002612E00C2070430E4922
:101D100008580190224639460198FEF760FA0028DB
:101D200005D1019800F0B4FB0AA000F0B1FB761CCD
:101D30000A2EEAD306A000F0ABFB21463846FFF797
:101D400033FE204675E7000020310001200000002E
:101D50000D0A00002020000000B5024600F008F83F
:101D6000034600BF00F004F8C01A9042FAD300BD49
:101D700007480069012109040840002804D00548EB
:101D80000068401C03490860024800687047000072
:101D900000E000E00840002000B595B001210820D7
:101DA000FFF788FA01218803FFF784FA0FA8FFF7ED
:101DB00093F940200F9002201090042014900FA956
:101DC0003148FFF705F980200F90042014900FA9E7
:101DD0002D48FFF7FDF8E120C0020B900021684676
:101DE00001864186818601870C21C1860BA927487F
:101DF000FFF71CFC01210846FFF74CFA002124489C
:101E0000FFF7ACF82248FFF759F80123204A204990
:101E10001C390320FFF7D4F81C48001D00901D4812
:101E20000190002002900320800203900020049083
:101E30008020059000200690079020200890000246
:101E4000099000200A9069461148FFF799F8002090
:101E50001149088001210E48FFF780F80122402136
:101E60000A48FFF7C9FB01210848FFF7B5FB0B48FB
:101E70000B4948610020886105200861002009495C
:101E8000086015B000BD0000000C014000380140A2
:101E90001C0002409440002004400020FFF9000094
:101EA00000E000E00840002070B5044600F01CF897
:101EB00005460B480088A84201D1002070BD0948A2
:101EC00007490988405C2070032189020448008882
:101ED000401CFEF715F9024801800120EEE70000E2
:101EE000044000209440002010B50448FFF744F857
:101EF00003218902081A80B210BD00001C000240B4
:101F000070B505460E4600240CE0295D0748FFF732
:101F1000E7FB00BF80210548FFF778FB0028F9D0D8
:101F2000601C84B2B442F0DB70BD00000038014098
:101F300010B5044600F02EF810482060204600F04E
:101F400021F8A0620E48FFF749F9002801D00120CE
:101F500010BD2C2221460A48FFF77AF9002801D04B
:101F60000120F5E72C2206492046FEF722F9002839
:101F700001D00120ECE70020EAE7000011C011CAFF
:101F80000040000110B504462821204600F0D8F892
:101F900010BD000010B505480078002804D1FFF7F7
:101FA0003BF901200149087010BD00004D400020A0
:101FB00070B50446204600F0B1F8002801D015A005
:101FC00000E016A005462A461A491BA000F092F927
:101FD00020A0216800F08EF925A0616800F08AF940
:101FE00029A02369E268A16800F084F932A0616940
:101FF00000F080F936A0236AE269A16900F07AF95D
:102000002DA0616A00F076F93DA0A16A00F072F996
:1020100070BD000076616C6964000000494E564155
:102020004C49442028626164206D616769632F63B5
:102030007263290000400001626F6F7473657474ED
:10204000696E6720402030782530386C583A20255A
:10205000730D0A0020206D61676963202020202015
:1020600020203D2030782530386C580D0A000000C3
:1020700020206163746976655F62616E6B203D202C
:10208000256C750D0A000000202062616E6B313AEC
:1020900020616464723D30782530386C5820736953
:1020A0007A653D256C75206372633D307825303844
:1020B0006C580D0A00000000202020202020202045
:1020C000207665723D30782530386C580D0A000056
:1020D000202062616E6B323A20616464723D307818
:1020E0002530386C582073697A653D256C752063FE
:1020F00072633D30782530386C580D0A00000000BE
:1021000020206372633332202020202020203D20B5
:1021100030782530386C580D0A00000010B50446A0
:1021200006492068884207D12046FFF72BFFA16AA5
:10213000884201D1012010BD0020FCE711C011CA66
:1021400030B502460B460021C94312E01078521CFC
:10215000414000240BE04808CD07ED0F002D01D0D1
:10216000074D00E0002568400146601CC4B2082C01
:10217000F1DB18465B1E0028E8D1C84330BD0000E3
:102180002083B8EDF0B589B0074600263C4621E033
:1021900000E0641C20782028FBD020780928F8D0A3
:1021A0002078002800D11AE03046761C800001A972
:1021B0000C5000E0641C2078002805D020782028EE
:1021C00002D020780928F5D12078002802D00020FC
:1021D0002070641C2078002801D0082ED8DB00BFB6
:1021E000002E02D1002009B0F0BD002513E00C2222
:1021F0006A430D4B99580198FDF7C3FF002809D198
:102200000C2068430849401801A98268304690476D
:102210000020E8E76D1C0A2DE9D304A0019900F025
:1022200069F80120DFE7000020310001756E6B6E58
:102230006F776E20636F6D6D616E643A2025732039
:1022400028747279202768656C7027290D0A0000B0
:1022500070B504462078002800D170BD174800787A
:1022600000280FD016480078401E45076D0F5021FA
:102270006943144A88182146FDF783FF002800D1DE
:10228000EBE700BF0E490978502251430D4A8818E8
:102290002146FDF79BFF0A480078401C4007400F8D
:1022A0000749087005480078082804DA03480078D0
:1022B000401C0249087000BFCFE700000D4000201D
:1022C0000E400020944C00200146084B1B785B1EFA
:1022D0005B1A18460830C3175B0F1B18DB10DB00B6
:1022E000C21A50205043024BC01870470E400020C5
:1022F000944C00200FB4F0B589B0644C0FA808903E
:10230000B0E00E98007807900E98401C0E90079849
:10231000252803D007982070641CA3E000200690B5
:10232000202605900E9800782D2804D101200690D3
:102330000E98401C0E900E980078302803D130265D
:102340000E98401C0E900BE00E9800780E99491CD8
:102350000E91014630390A2205985043081805901D
:102360000E980078302803DB0E9800783928EBDDD2
:102370000E9800786C2802D10E98401C0E900E9892
:102380000578002D02D00E98401C0E90642D21D0AF
:1023900006DC252D58D0582D45D0632D58D112E09C
:1023A000732D04D0752D2CD0782D51D13AE02020FA
:1023B0000090089802C808902046069B059A00F0F5
:1023C00065FD04464CE008980178001D08902170D6
:1023D000641C45E0089880C80890FB0F002F01DAC4
:1023E000784200E038460A2202A9019000F075FD0B
:1023F000009602A92046069B059A00F047FD044678
:102400002EE0089901C900230A22089102A900F0D0
:1024100064FD009602A92046069B059A00F036FD51
:1024200004461DE000BF089901C90023102208914D
:1024300002A900F052FD009602A92046069B059ACB
:1024400000F024FD04460BE025202070641C07E00A
:1024500025202070641C002D01D02570641C00BF55
:1024600000BF00BF0E980078002804D00748543001
:10247000844200D245E7002008902070034800F015
:1024800007F809B0F0BC08BC04B01847144F00208E
:1024900070B504462046FDF76DFE85B229462046FC
:1024A000FFF72EFD70BD000001460A684B68094821
:1024B00082420DD3084882420AD808460830834237
:1024C00006D3072080030818834201D201207047F9
:1024D0000020FCE70140002000C00020044601204D
:1024E000C007204305490863206880F3088800BFBF
:1024F00062B66068804700BFFEE7000000700040E1
:102500001CB5304C30480190002700262F49206828
:1025100088421CD128212046FFF712FEA16A88427A
:1025200015D16168022902D12146183101E0214606
:10253000083108460127244A0168914206D3412206
:1025400092040168914201D20168019100BFFFF736
:1025500023FC1FA000F06CFC002E1BD1FFF708FC31
:1025600005460FE06846FFF79FFC002809D0684643
:1025700000780D2803D0684600780A2801D101268A
:1025800007E000BFFFF7F4FB401B7D2109018842F3
:10259000E8D300BF002E0AD1002F08D10A48FFF768
:1025A00083FF002803D1012619A000F041FC002E72
:1025B00004D024A000F03CFCFFF71CFA0198FFF7C0
:1025C0008DFF0000004000010080000111C011CA11
:1025D0000D0A5B626F6F745D2043414949432D4290
:1025E0004F4F542056312E30302E3037202D20457D
:1025F0006E7465722077697468696E2032733A2050
:10260000646F776E6C6F6164206D6F64650D0A0096
:102610005B626F6F745D206E6F2076616C69642001
:1026200061707020696D6167652C20666F726365EB
:102630006420646F776E6C6F6164206D6F64650DEC
:102640000A0000005B626F6F745D20444F574E4C70
:102650004F4144204D4F444520286F74612F636CD7
:1026600069206F76657220554152542C2027686589
:102670006C702720666F7220636F6D6D616E64737E
:10268000290D0A0030B502460F4817E01578521C94
:102690002C02604000230EE00124E4030440002CDF
:1026A00004D04400094D6C40A4B201E04404240C61
:1026B00020465C1CE3B2082BEED300BF0B464C1E39
:1026C000A1B2002BE2D130BDFFFF000021100000BD
:1026D00010B5044611E00C4909680C4A12688818C4
:1026E000FEF77CFD002801D0052010BD07480068DA
:1026F0000121090340180549086004480068A04208
:10270000E9D30020F1E70000144000202C40002015
:10271000F7B586B00C4615460C2D09D0102D07D004
:10272000002301221021069800F05EFA09B0F0BDE6
:10273000204600F04DFA0646201D00F049FA0590AB
:102740002046083000F044FA0490102D04D12046B1
:102750000C3000F03DFA00E000200390364800788D
:10276000002807D03548022210210368069800F09F
:102770003BFADBE7324F33493868884208D12821D9
:102780003846FFF7DDFCB96A884201D1012000E03C
:10279000002001900198002804D07868012801D118
:1027A000294800E029480290042E03D30720800323
:1027B000864206D9002303221021069800F014FA5D
:1027C000B4E723480078002804D1FEF725FD012056
:1027D0001F4908700120184908701E4902980860B6
:1027E0001D4806601D49059808601D490498086049
:1027F0000020124908601B4908601B4908601B49FA
:1028000008600398C007C00F002806D01848006869
:102810001849884201D1012000E0002016490870C3
:1028200000201649087000231A461021069800F06F
:10283000DBF900BF7AE700001040002024400020B0
:102840000040000111C011CA0040020100800001D7
:102850003840002014400020184000201C40002078
:1028600020400020284000202C4000203440002040
:1028700040400020652C00014440002045400020DD
:10288000F7B582B061480078002807D10023022202
:102890001121029800F0A8F905B0F0BD04980428B1
:1028A00007D25B48012211210368029800F09CF9CD
:1028B000F2E7039800F08CF901900398061D049844
:1028C000041F0094524901980968884212D0514867
:1028D0000078002803D050480078002809D14C48DF
:1028E000022211210368029800F07EF901204A4972
:1028F0000870D1E7464800680019484909688842CD
:1029000007D94348032211210368029800F06CF9AB
:10291000C2E73F48006800193D4908600846006862
:10292000FFF7D6FE0546002D21D13D48006800285E
:102930001DD00AE031783A4802680068401C384BE4
:10294000186038488154761C641E35480068042895
:1029500001D2002CEED132480068042807D10421AE
:10296000304800F019F9054600202D490860002D77
:102970000BD1042C09D3A708BF003946304600F01C
:102980000BF90546F619E41B00BF002D08D1002CF9
:1029900006D0224631462348FDF7C8FB2048046094
:1029A000002D09D01A482A4611210368029800F028
:1029B0001BF9FEF7B3FE6FE70020174908701548B2
:1029C0000078002819D0124801680098081A000BF6
:1029D00000030F490968090B0903884205D10C4817
:1029E00000680E490968884206D109480022112171
:1029F0000368029800F0F8F84EE70548002211211C
:102A00000368029800F0F0F800BF45E7104000208E
:102A10002440002044400020454000201840002071
:102A20003440002030400020F7B50E465048007872
:102A3000002806D1002302221221009800F0D4F8C9
:102A4000FEBD0298042807D04A48012212210368DB
:102A5000009800F0C9F8F3E7304600F0B9F80546F1
:102A60004448006844490968884207D04148022226
:102A700012210368009800F0B7F8E1E73F480068CA
:102A8000002820D008E0FF213C4802680068401C74
:102A90003A4B18603A488154384800680428F2D309
:102AA0000421374800F078F8002809D03148052281
:102AB00012210368009800F097F8FEF72FFEBFE799
:102AC00000202E4908602C4801682E480068FFF756
:102AD00037FB0446AC4203D12B480068844209D03E
:102AE0002448042212210368009800F07DF8FEF7C4
:102AF00015FEA5E723480068001D00F069F80746A9
:102B0000204800680830874206D31E4800681A49EA
:102B100009684018B84209D81648062212210368ED
:102B2000009800F061F8FEF7F9FD89E700F0A8F8D9
:102B3000002809D00F48052212210368009800F0F0
:102B400053F8FEF7EBFD7BE70020104908700A48B8
:102B5000002212210368009800F046F8FFF708F9F8
:102B60000B49086001200B49087000BF68E70000AE
:102B70001040002024400020184000203440002055
:102B800030400020144000201C400020394000202C
:102B90003C4000203A40002070B505460C460A49EA
:102BA00009680A4A1268881822462946FEF750FB2F
:102BB000002801D0052070BD0448006800190349B1
:102BC00008600020F7E700001440002028400020A3
:102BD000014608784A78120210438A78120410439A
:102BE000CA78120610437047FFB587B005460E46F7
:102BF0001C46684606750999417584752004010EC6
:102C00006846C1752002010E68460176200E6946AD
:102C100048761348006800281FD0CA216846017111
:102C20001F21417185710621C171002101720622A7
:102C300005A90930FDF77AFA0A2101A80130FFF74A
:102C400021FD07466846C773391201740D2101A89A
:102C5000034A126890470BB0F0BD00BFFBE70000CD
:102C60004040002070B504460D4629462046FFF737
:102C700047F901200149087070BD0000394000206B
:102C800010B58CB02C222A4901A8FDF74FFA29492A
:102C90000198884206D128212548FFF751FA0B995F
:102CA000884203D02C2101A8FDF759FA2148019050
:102CB000214800682149884201D1012000E002201A
:102CC00002901D4800681D49884201D103A800E018
:102CD00007A804461848006820601948006860602A
:102CE00018480068A06018480068E060282101A822
:102CF000FFF726FA0B900E48FEF770FA002802D074
:102D000005200CB010BD2C2201A90948FEF7A0FA3D
:102D1000002801D00520F4E72C22054901A8FDF781
:102D200048FA002801D00520EBE70020E9E7000081
:102D30000040000111C011CA1440002000800001B1
:102D4000184000201C40002020400020F8B5044618
:102D50000D4600200090002269462046FDF74EFAFD
:102D600006460098A04203D000980078002801D0C1
:102D70000120F8BD2E600020FBE7000070B503467F
:102D80000C46154600221878702804D01878502870
:102D900001D0002070BD5878612802D058784128B1
:102DA00002D1214820600AE05878622802D0587881
:102DB000422802D11D48206001E00020EAE7991C6A
:102DC0000878302802DB0878392801DD0020E1E7A7
:102DD00009E00A2050430E78303E82190F2A01DDA7
:102DE0000020D7E7491C0878302802DB087839280A
:102DF000EFDD0878002801D00020CBE70A4E2068DC
:102E0000B04203D1062A01DD0020C3E7074E206847
:102E1000B04203D10D2A01DD0020BBE70120904024
:102E200028800120B6E7000000080140000C0140A6
:102E300010B5044604E02046641C0121FFF760F849
:102E400020780028F7D110BD70B5D2B0002400253D
:102E500000BFEFF310800646FF21453101A8FDF7C2
:102E60007EF901AC01349822074901A8FDF75EF90B
:102E70000120FEF74CFCA04705463046FEF747FC14
:102E8000284652B070BD000086300001F8B50446F7
:102E90000D4616461F462846FDF76CF90090002F98
:102EA00008D102E006982070641C3046761E009916
:102EB0008842F7DC03E0287820706D1C641C2878B9
:102EC0000028F8D102E020202070641C3046761ED5
:102ED00000998842F7DC2046F8BDFFB583B007466D
:102EE0000C46002500BF38460599FDF709F90E4646
:102EF0000A2E02D23046303001E030463730C2B2BE
:102F00002846691CCDB269460A5438460599FDF732
:102F1000F7F80746002FE6D10698002805D02D22A5
:102F20002846691CCDB269460A5406E0681EC0B244
:102F300005466946085C2070641C002DF6D100200F
:102F4000207007B0F0BD40BA7047C0BA7047013872
:102F5000FDD170470000F7B50325AD06286A82B0A1
:102F600016460C46400840002862286A02210843A1
:102F70002862286A8007FCD46620686001272F61D8
:102F8000A86AC005FCD5992068602F61A86AC005B1
:102F9000FCD5FF209130FFF7DAFFFF230133AB624E
:102FA0006846EF60352169602F61A96AC905FCD5C3
:102FB000AB62A969EF60C9B205226A602F61AA6A93
:102FC000D205FCD5AB62AA690902D2B211430180D5
:102FD000C80702D0032005B0F0BDAB626869FF21CD
:102FE0000831884368616869C91E084368610298AE
:102FF0000002483068600820A860EE602F61A86A6F
:10300000C005FCD5FF200130A8620023F61CB008E3
:103010000ED0B2081148006899006054060A0919D8
:103020004E70060C000E8E705B1CC8709A42F1D870
:10303000FF200130A8626869FF2108318843686178
:10304000686938436861286A800880002862286AB5
:1030500038432862002005B0F0BD8000000C03203A
:1030600080064169FF220832914341614269012192
:103070000A434261026A920892000262026A0A43AB
:10308000026270470000002003218906096A49088E
:1030900049000322920611621146096A0222114375
:1030A00003229206116200BF03218906096A0222E7
:1030B00011400229F8D0D101032292069162032126
:1030C000D1609F2151600121116100BF0321890658
:1030D000896AFF22013211409142F7D10322920600
:1030E0009162114688694969FF220832914303229F
:1030F0009206516111464969012211430322920649
:1031000051611146096A8908890011621146096AEC
:103110000122114303229206116270470000000051
:103120009C37000168370001390A00014C37000163
:103130003C370001490E000160370001683600018C
:1031400059090001A43700011037000141060001B0
:10315000E4370001C0350001610600012438000198
:10316000EC370001690300010C3700013036000123
:103170003D0B0001D4370001A03600015D0D0001B8
:10318000DC370001F8350001590B0001543700010C
:10319000AC370001990D000100000000010203049A
:1031A000000001020138FDD170470000F0B4032493
:1031B000A406236A5B085B002362236A02252B4373
:1031C0002362236A9B07FCD4FF230133A362656952
:1031D000DE1DB543656165691E1D354365610002ED
:1031E0006B3060600820A060E26001262661A06A62
:1031F000C005FCD5A3620023D21C90080ED0950810
:103200000F4800689A008854070A52185770070C34
:10321000000E97705B1CD0709D42F1D86069FF2151
:10322000083188436061606930436061206A8008CA
:1032300080002062206A30432062F0BC002070478A
:103240008000000CF8B5064601200025C004864227
:1032500001D90520F8BD0324A406206A40084000D7
:103260002062206A022108432062206A8007FCD481
:10327000FF270137A76200F0BBF8002801D0032523
:1032800015E00620606001212161A06AC005FCD51F
:10329000A7623002203060602161A06AC005FCD5C1
:1032A000A7620C4800F0C8F8002800D10225606928
:1032B000FF21083188436061606901210843606132
:1032C000206A800880002062206A08432062284625
:1032D000F8BD0000E6960100F7B506460120C004DF
:1032E00082B01546864202D9052005B0F0BD032004
:1032F0008006016A490849000162016A02221143FD
:103300000162016A8907FCD4FF2101318162F2B2B6
:103310008C1AA54200D8ACB20398009000F068F86F
:10332000002840D106214806416001210161816ADF
:10333000C905FCD5FF210131032080068162416966
:10334000FF220832914341614169042211434161E6
:10335000310232314160C4600022002C16D900983D
:1033600087183B78F87819467B7800061B021943CA
:10337000BB781B04194301430802F978000A0906C7
:10338000084319490860121DA242E8D30121032015
:1033900080060161816AC905FCD5FF210131816286
:1033A000124800F049F8A54209D0039836190019CF
:1033B0002D1BFF2401340390A542ADD8ABE70320B9
:1033C00080064169FF22083291434161416901222F
:1033D00011434161016A890889000162016A114350
:1033E0000162002005B0F0BD8000000C1A0600004C
:1033F00038B40125032080066A46C5603521416046
:103400000561816AC905FCD5FF24013484628169A4
:10341000C560CBB2052141600561816AC905FCD553
:10342000846280691902C0B2014388B21180C0076A
:1034300000D0012038BC7047F8B4002101250322D8
:1034400092066B46D560352454601561946AE40594
:10345000FCD5FF27013797629469D560E4B2052651
:1034600056601561966AF605FCD597629669240246
:10347000F6B234431C80E30722D0814202D9F8BC63
:1034800000207047032292066B46D56035245460B5
:103490001561491C946AE405FCD597629469D5606E
:1034A000E4B2052656601561966AF605FCD597626A
:1034B00092692402D2B21443A2B21C80D207DCD19A
:1034C000F8BC0120704700000040404040404040B0
:1034D00040404141414141404040404040404040E7
:1034E000404040404040404040050202020202028B
:1034F00002020202020202020220202020202020DA
:1035000020202002020202020202909090909090ED
:1035100010101010101010101010101010101010AB
:10352000101010100202020202028888888888881F
:10353000080808080808080808080808080808080B
:10354000080808080202020240000000C934000115
:103550005B6F74615D2062696E617279206D6F646A
:1035600065204F4E202D2073656E642030784341D6
:10357000204F5441206672616D6573206E6F770D28
:103580000A28626C655F70726F746F636F6C2E6D6A
:10359000642073656374696F6E20362E363B204F4E
:1035A00054415F41424F5254206F7220337320695F
:1035B000646C65206578697473290D0A0000000049
:1035C0006273736574203C6669656C643E203C766A
:1035D000616C3E3A20777269746520626F6F747314
:1035E000657474696E67206669656C642028636120
:1035F000726566756C21290070696E736574203C74
:1036000070784E3E205B307C315D3A207365742FBC
:1036100072656164204750494F206C6576656C2067
:10362000287061302D362F7062302D313329000023
:103630006F74613A205541525420656E74657273FF
:10364000204F54412062696E617279206672616D0B
:1036500065206D6F646520287365652068656C70F2
:10366000206F74612900000073686F7720626F6FAC
:103670007420696E666F202B206375722062616E04
:103680006B20284F544120777269746573207468E9
:1036900065204F544845522062616E6B290000003E
:1036A00072657365743A2073797374656D20726501
:1036B00073657420287265626F6F742900000000C2
:1036C0000D0A434C492072656164792028626F6F4E
:1036D000746C6F6164657220646F776E6C6F616487
:1036E000206D6F6465292E205479706520276865E8
:1036F0006C702720666F7220636F6D6D616E6473EE
:103700002E0D0A63616969632D3E00006F746100CC
:10371000627364756D703A2073686F7720626F6FA3
:103720007473657474696E67207265636F72642068
:103730002B2063726320636865636B0073686F7727
:1037400020626F6F746C6F6164657220766572734E
:10375000696F6E0075617274696E666F00000000BB
:10376000646576696E666F0068656C70205B636D7A
:10377000645D3A206C69737420636F6D6D616E6473
:1037800073202F2073686F77206F6E6520636F6DD5
:103790006D616E6427732068656C700068656C707D
:1037A00000000000627364756D70000075617274D2
:1037B000696E666F3A2073686F7720555341525493
:1037C000312070696E732F626175642F666F726D40
:1037D00061740000726573657400000070696E7337
:1037E000657400006273736574000000617070732B
:1037F00077205B317C325D3A20737769746368208F
:10380000626F6F742062616E6B2028637263207632
:103810006572696669656429202B207265626F6F25
:103820007400000061707073770000006170707345
:10383000773A2062616E6B256C7520696D616765F2
:1038400020637263206D69736D61746368202872F0
:1038500065636F72642030782530386C582C206195
:10386000637475616C2030782530386C58290D0AE6
:103870000000000020202020202020202062316134
:103880006464727C6232616464727C623173697AEE
:10389000657C623273697A657C62316372637C62D3
:1038A000326372637C62317665727C6232766572F5
:1038B000203C6865787C6465633E0D0A000000006A
:1038C000E03800010040002060000000F016000118
:1038D0004039000160400020781C00000017000102
:1038E0000090D00300000000000000000000000075
:1038F00000000000000000000000000000000000C8
:1039000000000000000000000000000000000000B7
:1039100000000000000000000000000000000000A7
:103920000000000000000000000000000000000097
:103930000000000000000000000000000000000087
:1040000011C011CA010000000080000100E800009A
:104010000114E5592200010000000000000000002A
:0C4020000000000000000000FB7F96A6DE
:10800000F0BD0020698100017181000139BA0001D1
:108010000000000000000000000000000000000060
:1080200000000000000000000000000055BE00013C
:1080300000000000000000002781000159BE00017F
:108040007B8100017B8100017B8100017B8100013C
:108050007B8100017B8100017B8100017B8100012C
:108060007B8100017B8100017B8100017B8100011C
:108070007B8100017B8100017B8100017B8100010C
:108080007B8100017B8100017B8100017B810001FC
:108090007B8100017B8100017B8100017B810001EC
:1080A0007B8100017B8100017B8100017B810001DC
:1080B00061C000017B8100017B8100017B810001A7
:1080C0000348854601F080F8004800477109010126
:1080D000F0BD002040BA7047C0BA70470138FDD1EA
:1080E0007047000040BA7047C0BA7047704670478A
:1080F000084B19680868203080F30988022080F353
:108100001488BFF36F8F3FBCAE4608BC04BC62B698
:1081100018470000CC470020EFF3108072B670477C
:1081200080F310887047EFF309800E4B1A682038EF
:108130001060F0C044464D4656465F46F0C008B554
:1081400072B60CF053F862B60CBC116808681030B7
:10815000F0C8A046A946B246BB4680F3098820383D
:10816000F0C81847CC47002004488047044800471F
:10817000FEE7FEE7FEE7FEE7FEE7FEE7B1BE000131
:10818000C180000130B50B460146002020220124A9
:1081900009E00D46D5409D4205D31D469540491B3B
:1081A0002546954040191546521E002DF1DC30BD84
:1081B00070B500242546002801DA01244042002938
:1081C00001DA01254942FFF7DDFFAC4200D0404211
:1081D000002C00D0494270BDF0B51FB40646002007
:1081E00082B005464024019100901BE0019922468F
:1081F0000F46304600F037FE049A059B801A9941DD
:1082000010D310461946224600F01DFE361A8F4143
:108210000197224601200021009F00F014FE38182B
:108220004D4100902046641E0028DFDC019B009831
:108230002946324607B0F0BD01464139192900D818
:10824000203070470549064A08685043054A80189F
:1082500008604008704701490860704724480020C2
:108260006D4EC6413930000003460B439B0703D0D7
:1082700009E008C9121F08C0042AFAD203E00B78EB
:108280000370401C491C521EF9D27047D2B201E063
:108290000270401C491EFBD270470022F6E710B561
:1082A00013460A4604461946FFF7F0FF204610BD64
:1082B000421C0178401C0029FBD1801A704710B580
:1082C000002200E0521C835C8C5CA34201D1002B95
:1082D000F8D1D8B2E1B2401A10BDC9B203E00378B8
:1082E0008B4203D0401C521EF9D20020704730B59B
:1082F00004460020034600E05B1C934203D2E05C8E
:10830000CD5C401BF8D030BD03460A780270401C9B
:10831000491C002AF9D11846704730B5054600209F
:10832000034600E05B1C934205D2EC5CC85C201A5B
:1083300001D1002CF6D130BD0FB400B58DB009903D
:108340000B9010A900200091C0430A9000200C90CF
:1083500006480690064807906A4609A80F9900F05B
:10836000BBFD0DB008BC04B018470000F98E000139
:10837000198F0001FFB5087889B01546FF2805D090
:10838000491C2D2804D00022002407E000240BE023
:108390000122F9E70A235C430419491C0878FF28E5
:1083A000F8D1002A00D06442002004902A780146C7
:1083B0002D2A01D02B2A0FD16D1C2D2A02D000228C
:1083C000049209E00122FBE700260A2233466D1CD5
:1083D00000F0FCFC381871412F78FF2FF4D10C9A73
:1083E000A218069202460A4304D0FF23069A91334C
:1083F000DA4205DA002109980A4606C00DB0F0BD40
:108400000024B74AB54D2646079200F01BFC0290A7
:1084100006980391002801DA474200E00746390533
:108420000020AF4A001C51410191009012E0F80772
:1084300007D022462B463046079900F0D9FA064667
:10844000079122462B461046194600F0D1FA044601
:108450000D467F10002FEAD10698019B0028009A54
:108460000399029806DA00F02BFB3246079B00F0D6
:1084700027FB05E000F0BCFA3246079B00F0B8FA93
:10848000049A002A02D00122D2075140099A03C25D
:10849000B4E7FFB591B0002009900025ED432E20F0
:1084A0009E685C681F460190B9696D1C12988847E8
:1084B0000090396A88470028F6D10098401C0AD0FD
:1084C0000D20C0018443002E12DD00982B2809D016
:1084D0002D280DD103E00020C04315B0F0BD0120D0
:1084E00080020443B9696D1C12988847761E00907B
:1084F00003A9600501D52D2000E02B206A461073EA
:10850000491C0CA80F9102900AE0B9696D1C1298E1
:10851000884700900120400204431398761E0560AE
:10852000002E02DD00983028EFD001990098884293
:1085300046D18020044308E00998401E099001209C
:10854000400204431399681C0860B9696D1C761ECB
:108550001298884700903028EED031E00199884287
:1085600005D1200603D480200443761E1EE0009827
:1085700003F084FF002826D001204002044307A90D
:108580000F980331761E88420BD200980F9930382D
:1085900008700F98401C0F90200607D50998401EC0
:1085A00003E0200602D40998401C0990A00502D5DA
:1085B0001399681C0860B9696D1C1298884700906F
:1085C000002ECBDC59E0002E57DD0098652801D045
:1085D000452852D1A00550D5032000028443B96933
:1085E0006D1C761E129888470090002E0CDD2B28FB
:1085F00004D02D2808D1FF2001300443B9696D1C37
:1086000012988847761E0090E00501D52D2100E0E4
:108610002B21029801700298401C0290019025E0E5
:108620000120400204430EA902980131761E8842BF
:108630000ED20098029930380006000E087003D15F
:108640000299019881420AD90298401C029006E0E2
:10865000E00501D5234801E0224840420990B9696C
:108660006D1C12988847009013980560002E04DD59
:10867000009803F003FF0028D2D1F96912988847C7
:108680000F99FF200870029903AA087000200A9031
:108690000B900CA90AA8099BFFF76CFEA00502D459
:1086A0000120C04319E72420044209D0E00713D178
:1086B00038680B9A0A99031D3B60006806C00BE0FE
:1086C0000B990A9800F066FB0146E00704D1386870
:1086D000021D3A60006801602846FEE60000144072
:1086E0000000F03FF1D8FFFFF7B582B00F4600263B
:1086F000029C03F0AFFD0090006801902578641C97
:10870000002D05D000F0D4FB0068405DC007F5D116
:108710002B2D02D02D2D1CD0641E0098002101604D
:1087200039462046049A00F009FC0146002F04D087
:108730003868A04201D10298386000980068022889
:108740000BD00098019A0260700506D5484205B02A
:10875000F0BD012080020643DFE70846F7E7F8B5E1
:1087600002464A40D40F42004B0052085B089A422E
:1087700002D20246084611464A0023D0C30D4A00E1
:10878000DDB2120EAD1A202D35DA49020126490A52
:10879000F6058A19002C00D0524220214F1B1146A9
:1087A000B9402A411018C20D9A4221D0002C17D08E
:1087B000012D08DCDA05801AD20F8019D207DBB24E
:1087C00000F06AFCF8BDDA05801A012340001B06A0
:1087D000C01880185A428018CA0F1043490007E099
:1087E0004908C2071143DA05801A80194008801829
:1087F00000F04AFCF8BD61000122511A001BF7E7A6
:108800000122D2075140AAE70122D2075040A6E731
:10881000024670B54A40D30FDB0740002DD04A0016
:108820002AD0010E140E000212020919400A520A3F
:108830008418E50104465443000A120A2E045043EA
:10884000A4194219200CC543AA18120C0125AD0326
:10885000521C521912047F39240400D0521C1043B8
:1088600001D44000491EC2B20C06C0092018401CA9
:108870004008802A02D003E0002070BD400840007C
:10888000002900DA0020184370BD0000F0B507464B
:108890000846584087B0C00F049048000E46590063
:1088A00040084908BC1A884105D2384631461E4660
:1088B00017460B4602465800400810434CD0300D76
:1088C000039040055900400D490D0590401A029053
:1088D000402872DA18030121000B090508430190B2
:1088E00004980092002805D0019952420020884146
:1088F00000920190029840210A1A0199009800F014
:10890000A2FA05460C466B4607CB00F0BDFAC0192B
:108910007141039A0E0D0023D71756401A467A402C
:10892000164344D0049A002A2DD0029A012A039AB1
:1089300015DC1205C01A914101263605001C714153
:10894000D20F059ED2070093019202962A46234633
:1089500000F0E8FB07B0F0BD38463146FAE71605EF
:10896000224A0F46B218C01AB74101210905001C5E
:108970004F4100187F41114618187941E20F10430A
:108980006D19644113E0E2076D0815436408C207DE
:108990001443039A01261205C01A91413605001CA2
:1089A0007141CE07400830434908C01851412A465A
:1089B000234600F0AAFBCDE7FFE704980122400020
:1089C000C117121A00238B4104983146C417381A74
:1089D000A141EEE730B40124E407634030BC55E721
:1089E00030B40124E407614030BC4FE70000E0FFF1
:1089F000F0B51FB488B00B99099800244840099934
:108A0000C00F490049080991C0070B99009049001F
:108A100049080B9109990898A64608431CD00B9960
:108A20000A98084318D0099801244000420D4800D4
:108A3000410D099824050003000B204309900B9871
:108A40000003000B20430B9050181C4940180022D3
:108A500001901446104605E0002001460DB0F0BD1F
:108A6000032801DA034600E003239C46C11A0AAE3C
:108A70000AE05F0008ADED5B4F00F75B7D43002728
:108A8000AA187C41491C5B1E6145F2DD410004AB24
:108A90005A522104120C0A43240C401C0828DFDB24
:108AA000019802900099704601910090059B049AEC
:108AB0000799069800F036FBD0E700000DFCFFFF99
:108AC000F0B50C465C4085B0E40FE40703944C001D
:108AD000002664085900944649080246029622433B
:108AE00021D062460A431ED06200570D4A000E0391
:108AF0002303550D012402462C492405781B1B0B2A
:108B0000360B401823432643614600901C46501AFA
:108B1000B44103D30098401C009002E092180098E2
:108B20005B41002803DA0020014605B0F0BD0020BB
:108B3000012109050746864611E064461D46141BBF
:108B4000B54106D36546521BB341744607430C43F7
:108B5000A646CD0740084908284392185B410546C0
:108B60000D43EAD11046184313D0604619465040D1
:108B70007140084306D06046101AB34106D2012264
:108B8000002306E000220123DB0702E00122D2439A
:108B90005310009874460105381C6141029C039DE6
:108BA0000019694100F0B1FABFE70000FD030000C1
:108BB00070B54B005B0803430BD04B005C0D0026E7
:108BC00033466542B341D417AD1AA34102DB0020FE
:108BD000014670BD12053018514170BDC217C10F5A
:108BE000504010B54018CA079623002100F054FAEF
:108BF00010BD10B500229623114600F04DFA10BDAD
:108C00000EB5C217C10F5040CA0740180021054BCE
:108C10000293019200910A460B4600F083FA03B0DA
:108C200000BD0000330400000EB50549029100218B
:108C300000910A460B46019100F074FA03B000BDA2
:108C4000330400000EB5054A02920022009213463A
:108C5000019200F067FA03B000BD00003304000089
:108C6000C20F410040020123400ADB05D207090E72
:108C7000C0187F2901DA00207047962903DC96236B
:108C8000591AC84001E096398840002AF4D0404281
:108C90007047000070B5CD0F4A0009030123090B8E
:108CA0001B0519430B4BED070024520D9A4201DAC4
:108CB000002070BD074B34339A4203DC9A1A00F04F
:108CC000D2F802E00449511888402C43F1D04042C8
:108CD00070BD0000FF030000CDFBFFFF4A00090349
:108CE0000123090B1B0519430A4B10B5520D9A427B
:108CF00002DA0020014610BD064B34339A4203DCF1
:108D00009A1A00F0B0F810BD034BD21800F09BF88F
:108D100010BD0000FF030000CDFBFFFFC20FD20714
:108D2000400040080BD0C10D0723DB01C9184002E9
:108D30000905400A1143C20840071143704700204B
:108D40000146704710B5002904DB0124E4074042C6
:108D50008C412146002B04DB1C460123DB075242D9
:108D6000A3418B4200D1824210BD000010B5002902
:108D700004DB0124E40740428C412146002B04DB44
:108D80001C460123DB075242A341994200D1904285
:108D900010BD0000CB0FDB07490010B549080246A3
:108DA0000A4307D00A0D07240903E401090B121B2B
:108DB000002A01DC002010BDC900440F0C43C10093
:108DC000E018D205801800F05FF910BDF0B51FB4AF
:108DD00086B000200090019002900698069980B21B
:108DE00004900798090C020400141143079000270F
:108DF000089D099806913E463C4603900398A9B207
:108E00000204000C039004982D0C154348430021E4
:108E1000224600F018F8C719714110340E46402C54
:108E2000ECDB3846029A00F00EF8009A019B80189D
:108E30000090594102980191103002904028CCDBFB
:108E400000980BB0F0BD10B5202A04DB0146203A93
:108E50009140002010BD914020239C1A0346E3401E
:108E60001943904010BD10B5202A04DB0846203A73
:108E7000D040002110BD0B46D340D0402024A21A80
:108E800091400843194610BD10B5202A06DBCB17C8
:108E90000846203A1041C1170B4306E00B46134128
:108EA000D0402024A21A91400843194610BD00006A
:108EB000004870476C5B010110B50446FFF7F8FFEE
:108EC0000068005DC007C00F10BD00000268137885
:108ED000511801601846704710B5D16004495161BE
:108EE0000449116200211161114600F08FF910BD93
:108EF000CD8E0001B98E00014268002A08D00168B9
:108F00000B78491C002B03D0521E06C01846704730
:108F10000121C160881E70474268002A0BD0C368D7
:108F20000168002B07D183688B4204D0491E521C74
:108F300006C0002070470020C0437047F7B582B0DC
:108F4000029C00272078641C15460197302802D027
:108F5000002D15D015E020780127641C782804D056
:108F6000582802D0002D09D00BE0002D01D0102D83
:108F700007D1002710252078641C02E0082500E0B6
:108F80000A250026009610E0009901276943081879
:108F9000020C294680B2714300908E183804864234
:108FA00001D3012001902078641C294600F01EF9AD
:108FB0000028E9DA0398002805D0002F01D0641EAC
:108FC00000E0029C04600198002806D003F042F9FA
:108FD00002210160C81E05B0F0BD009930040843AD
:108FE000F9E700000FB400B589B00CA900910B9906
:108FF0000023CB60204B214A069307920422019262
:109000001F4A02921F4A089202466B460020FFF751
:1090100040FA09B008BC04B0184770B586B00646DF
:109020000020C0430190002015460C46009102919B
:1090300004903246694604A8FFF7D4FF024604981C
:109040002118002D05D0002801D0084600E0204658
:109050002860049800280DD0002A02DD009888427C
:1090600008D0081B0190009432466946029404A877
:10907000FFF7B8FF06B070BDF98E0001198F00012F
:10908000FFFFFF7FB98E0001002904DA401C490070
:1090900001D140084000704770B40024050C05D190
:1090A0001024000402D1002921D01124050E01D181
:1090B00000020834050F01D10001241D850F01D1E4
:1090C0008000A41C002801DB4000641C002908D09B
:1090D00020252E1B0D46F540A14000D0012129433B
:1090E000084301061B1B000ADB1D02D5002070BCD3
:1090F0007047DB05181880180029F8DA401C490071
:10910000F5D170BC40084000704710B5002B08DA5C
:109110000024401C614192185B411A4301D1400870
:10912000400010BDF0B51FB482B005460C0003D05E
:10913000084603F077F802E003F074F820300246A6
:10914000009021462846FFF77EFE049B059A0446C0
:109150000F4618431143084314D0184610431BD040
:10916000009840210A1A18460599FFF77CFE05462B
:109170000E46009A05990498FFF765FE084305D04E
:10918000012004E02046394607B0F0BD0020C11799
:1091900005430E432C43374300990E986305401A4C
:1091A0007905E40A00220C43FD0A0A3002D50020AA
:1091B0000146E9E70105101969410C9C0D9D001954
:1091C0006941FFF7A2FFDFE7064C0125064E05E0E7
:1091D000E36807CC2B430C3C98471034B442F7D3D8
:1091E000FEF772FFC8610101E86101013A2800D26F
:1091F0003038202302469A43412A01D3104637389B
:10920000884201D30020C04370470000F3B58DB001
:1092100000200A9001200B90002608460C300C46D6
:1092200009906269012109989047051E2ED0252DCD
:109230002DD0216A8847002818D062690121099839
:109240009047216A88470028F7D1411E6269099832
:10925000904700E0761CA1690D988847216A8847ED
:109260000028F7D1E1690D988847DAE7A1690D98E0
:1092700088470746A84201D1761CD2E7E1690D98DC
:1092800088477F1C02D10A98002877D049E100273F
:1092900062693D463946099890472A280CD162698F
:1092A000012109989047012506E00A214F433F1804
:1092B000303FEBD4102005436269012109989047A3
:1092C000014630390A2903D29B498F42DEDCECE7A4
:1092D000E90600D4994F6C280AD04C2810D0682891
:1092E00024D06A282ED074280CD07A280AD00DE019
:1092F00062690121099890476C2823D004211CE061
:10930000202005436269012109989047A7606560A4
:1093100065284FD026DC582839D01ADC452849D09A
:1093200012DC252834D04128B0D143E06269012104
:1093300009989047682802D008210D43E6E70120EC
:10934000C002DEE70220DCE7462833D047282CD1D4
:1093500030E05B2870D061282CD063286CD0642862
:1093600023D161E06F284FD009DC662822D067281E
:1093700020D0692826D06E2817D12EE0CDE07028A5
:109380004DD073286FD075284ED078280DD154E079
:10939000A1690D9888470546252800D16CE7E16949
:1093A0000D9888476D1C00D16DE7BAE00A224CE0A9
:1093B0000A2252E0012023466A46C0430D99FFF776
:1093C00068F8A3E02846402108436060A8072346C8
:1093D00001D5002239E000223FE0E80700D020E775
:1093E0002068011D21600068290501D5067018E775
:1093F000290701D5068014E7A90703D5F1170660F0
:1094000041600EE706600CE7284640210843606093
:10941000A807234601D5082217E008221DE0484985
:1094200028460840606016E02846402108436060F6
:10943000A8072346BCD5B9E715E0284640210843D4
:109440006060A80707D5234610220120C0430D996C
:10945000C046C0465AE0234610220120C0430D9961
:10946000C046C04652E000210C910B460091632893
:1094700002D05B2807D043E0E80601D40120A060B9
:10948000012000903CE062690121099890475E2824
:1094900005D101200C900146626909989047216925
:1094A000002906D10B4601AA8F00491CD351082977
:1094B000FADB002835D0216900290ED1C117C90E69
:1094C00009184A11930001AA9A1849094901411A39
:1094D00001201368884003431360626901210998E1
:1094E00090475D28E5D10C98002808D0002001ABFA
:1094F00081005A58401CD2435A500828F8DB01AB6F
:1095000001202246C0430D99C046C04600280ADA11
:10951000401C06D10B98002803D00020C0430FB098
:10952000F0BD0A98FBE7E90702D10A99491C0A91A4
:10953000361800200B9074E6CCCCCC0CFFFFFF7FDC
:10954000F1F7FFFF70B58C180578401C6B075B0FB7
:1095500001D10378401C2A1106D10278401C03E097
:1095600006780E70401C491C5B1EF9D12B0705D4F0
:109570000023521E0DD40B70491CFAE70378401CDF
:10958000CB1A921C03E01D780D70491C5B1C521E07
:10959000F9D5A142D8D3002070BD000003B4014822
:1095A000019001BD232A000003B40148019001BDD0
:1095B0006D56000003B40148019001BD65600000D4
:1095C00003B40148019001BDAF7F000003B401481E
:1095D000019001BDB551000003B40148019001BDE7
:1095E000D37E000003B40148019001BD697E0000F4
:1095F00003B40148019001BDC37F000003B40148DA
:10960000019001BDE954000003B40148019001BD7F
:109610009957000003B40148019001BDED570000C7
:1096200003B40148019001BD1D7C000003B4014852
:10963000019001BD0D2A000003B40148019001BD55
:10964000AB52000003B40148019001BDF58F00004A
:1096500003B40148019001BDE1FE000003B40148DC
:10966000019001BD250E010003B40148019001BD28
:10967000B143000003B40148019001BD85290000F9
:1096800003B40148019001BD71840000C9434160E9
:1096900070470268702392B29A430A43026070478F
:1096A00070B5044602F0C4FC002818D08069002878
:1096B00015D0FFF79EFA05462046FFF79AFA29468D
:1096C000FFF7A2F8FFF72AFB064A074BFFF7F8F966
:1096D0000022064BFFF7DAF8FFF75CFB70BD044D84
:1096E000EAE700001F85EB51B81E01400000394039
:1096F00000803B4470B50D460646002402F098FCFD
:10970000002816D0C169002913D0026A002A10D09F
:109710008BB290B289B292B2102D0CD0202D0AD00B
:10972000302D17D0402D15D0502D13D0602D11D0D5
:1097300022E0002070BD891AB01AAF229200504377
:10974000FEF736FD044696340FD47D20C0008442D7
:1097500011DC11E0191AAF22301A12015043FEF742
:1097600027FD4B21C900441801D5002404E0E12065
:109770000001844200DD0446204670BD70B5104CE7
:10978000A0421BD185140121284602F0DFFA0021F6
:10979000284602F0DBFA0121284602F0CBFA0948FC
:1097A00060610020206060601F21A1600649216186
:1097B000A06160622062A0620448E06170BD0000A8
:1097C00000080240080A02000000FC0F2E6D000095
:1097D0000029016802D00122114301E04908490033
:1097E0000160704704220029816902D01143816120
:1097F00070479143816108480649C1620749016386
:1098000007494163074981630749C163084907481C
:10981000086070472200780000080240E700E1007D
:109820009F00BF04190C051670206E286E2B0000D7
:109830004008024002220029016801D0114300E0E3
:10984000914301607047C06880B270470246526819
:1098500000200A4200D0012070470000044A9068AE
:10986000C90640094001C90E0143916070470000DC
:109870000008024070B5054649480C464EC88CB0F9
:1098800003960293019200914EC8079606930592A3
:109890000491426801688068099208910A90414ADF
:1098A00000996846914217D1282104F095FF0A9942
:1098B000884211D1022D1ADB0020646802460B9009
:1098C0000BA92046FEF710FF05460B98A04209D0D1
:1098D0000078002806D101E033A004E0012D0AD071
:1098E000022D08D03EA005F0B5F80CB070BD01986F
:1098F000012809D001250198A84207D1294647A08F
:1099000005F042F80CB070BD0225F4E7012D6C465D
:1099100014D01834012D13D047482268824206D152
:109920006068002803D00721890388420AD92946A4
:1099300042A0636805F028F80CB070BD0834E9E770
:109940004C48EAE74CA005F085F86168206804F00F
:1099500043FFA268824206D003462946544805F0D8
:1099600013F854A0BFE729465FA06368E26805F0DA
:109970000BF86846019504F0D1FA002801D06AA0DE
:10998000B1E76EA005F066F8C8200AF025FBBFF32A
:109990004F8F72497048C860BFF34F8FFEE70000D9
:1099A0000040000111C011CA61707073773A2062E3
:1099B0006F6F7473657474696E67207265636F721C
:1099C0006420696E76616C69642C207265667573BB
:1099D0006520746F207377697463680D0A00000056
:1099E00075736167653A206170707377205B317CB5
:1099F000325D20286E6F20617267203D2073776989
:109A000074636820746F20746865206F7468657271
:109A10002062616E6B290D0A000000006170707396
:109A2000773A20616C7265616479206F6E204150D5
:109A300050256C750D0A00000040020161707073C2
:109A4000773A2062616E6B256C75207265636F7268
:109A50006420696E76616C69642028616464723D7B
:109A600030782530386C582073697A653D256C75DF
:109A7000290D0A000080000161707073773A20762A
:109A80006572696679696E672074617267657420B2
:109A9000696D61676520637263202866657720734E
:109AA00065636F6E6473292E2E2E0D0A0000000070
:109AB000346101012020202020202072756E204278
:109AC0004C45204F544120746F2077726974652093
:109AD000612076616C696420696D616765206669E3
:109AE0007273740D0A00000061707073773A20621F
:109AF000616E6B256C7520696D616765206F6B20E9
:109B0000287665722030782530386C582C20256CEA
:109B1000752042292C20737769746368696E672EFB
:109B20002E2E0D0A0000000061707073773A2066D7
:109B30006C617368206661696C0D0A0061707073F6
:109B4000773A20646F6E652C207265736574746952
:109B50006E672E2E2E0D0A000400FA0500ED00E0BF
:109B600010B50B488CB01EC803940293019200916B
:109B70001EC80794069305920491426801688068A4
:109B80000A9009920891684604F0F6F90CB010BDED
:109B900000400001F0B58DB00E46032807DA54A04E
:109BA00004F058FF5AA004F055FF5F480FE000246E
:109BB000B76822460BA938460B94FEF795FD05467B
:109BC0000B98B84202D00078002804D057A004F0C7
:109BD00041FF0DB0F0BD5A4B87CB03970292019124
:109BE000009087CB07970692059104909A68596870
:109BF00018680A920991534A009908906846914260
:109C000005D1282104F0E8FD0A9988420DD000947E
:109C10000194029403940494059406940794089480
:109C2000099449A00A9404F015FF55A17068FEF745
:109C300046FB002804D070680178622908D02BE028
:109C4000012D03D0022D01D04FA0C0E701953AE0CD
:109C50004178312902D0322902D01DE002AC00E067
:109C600006AC51A1801CFEF72AFB002816D07068B4
:109C70004FA1801CFEF723FB002819D070684EA16D
:109C8000801CFEF71CFB00281AD070684BA1801CBA
:109C9000FEF715FB002815D049A098E74E488542ED
:109CA00004D04E48854201D04DA090E725600AE0DF
:109CB00007208003854201D958A088E7656002E04B
:109CC000A56000E0E5602A465DA0716804F05CFED6
:109CD000684604F023F9002801D062A077E766A067
:109CE00004F0B8FE684604F047F90DB0F0BD00007E
:109CF00075736167653A206273736574203C6669A9
:109D0000656C643E203C76616C3E0D0A00000000EC
:109D100020206669656C643A206163746976652009
:109D20003C317C323E0D0A007C6101016273736537
:109D3000743A206261642076616C75650D0A0000DA
:109D40000040000111C011CA62737365743A206546
:109D500078697374696E67207265636F72642069D5
:109D60006E76616C69642C2072656275696C642022
:109D700066726F6D20736372617463680D0A000010
:109D8000616374697665000062737365743A20617B
:109D90006374697665206D75737420626520312067
:109DA0006F7220320D0A00006164647200000000CE
:109DB00073697A6500000000637263007665720063
:109DC00062737365743A20756E6B6E6F776E206682
:109DD00069656C640D0A000000800001004002010A
:109DE00062737365743A2061646472206D75737474
:109DF0002062652043414949435F415050315F42F1
:109E0000415345206F722043414949435F415050BF
:109E1000325F424153450D0A0000000062737365D2
:109E2000743A2073697A6520657863656564732088
:109E30007468652062616E6B2073697A650D0A0033
:109E400062737365743A202573203D203078253085
:109E5000386C582C2077726974696E672E2E2E0D1F
:109E60000A00000062737365743A20666C6173685F
:109E7000206661696C0D0A0062737365743A206F25
:109E80006B20287665726966696564290D0A000091
:109E900000B583B0002103200B4601220191009000
:109EA000920203A103480AF0FFFC03B000BD0000CA
:109EB000434C4900BDA2000110B5022805DB4868EB
:109EC0000DA1FEF7FCF9002805D00D480078002808
:109ED00004D00CA103E008F03FF810BD0BA110A0C6
:109EE00004F052FD124C13A0218904F04DFD1CA07A
:109EF000E16804F049FD10BD6A736F6E0000000058
:109F0000B047002076616C6964000000646566619A
:109F1000756C7420286E6F742073617665642900F7
:109F2000706172616D733A2025730D0A00000000A4
:109F3000CC6A002020206C6564203D2025752020FF
:109F4000286C65643120626C696E6B2068616C6698
:109F500020706572696F642C206D73290D0A0000F2
:109F6000202070776D203D20256C7520202870778B
:109F70006D20647574792C202525290D0A000000B8
:109F8000F3B595B015980D46032807DA6F4804F02D
:109F900061FD6FA004F05EFD79A023E07FA16868F9
:109FA000FEF78DF9002810D00020AE680246009020
:109FB00069463046FEF798FB04460098B04202D04E
:109FC000007800287BD077A00CE000240226B000A7
:109FD00014902858FEF76CF90746E019801C5028A9
:109FE00004D975A004F036FD17B0F0BD002C03D0E5
:109FF000202069460855641C14983A46295868463A
:10A000000019FEF731F91598E419761C8642DEDB5B
:10A01000002069460855451E6E462C4606F070FB2A
:10A02000304604F02FFB060023D004F010FB00287C
:10A030001FD069A1304604F0D3FA074604F0FEFAB7
:10A04000002800D07D6965A1304604F0C9FA0746B2
:10A0500004F0F4FA002800D07C69002D13DA002CFB
:10A0600022DA5FA004F0F6FC304604F08FFA17B055
:10A07000F0BD65A004F0EEFC002EF8D0304604F0F0
:10A0800085FA17B0F0BD294666483239814209D3B6
:10A09000654A322165A004F077FC304604F076FA78
:10A0A00017B0F0BD002C0BDB642C09DD642164A02B
:10A0B00004F06AFC304604F069FA17B0F0BD14E011
:10A0C000304604F063FA002D01DB62480581002C64
:10A0D00001DB6048C46007F093FF002801D05EA058
:10A0E00080E707F039FF17B0F0BD3BA16868FEF7C5
:10A0F000E6F8002807D039A16868FEF7E0F80028E4
:10A100000DD05CA06EE7204646493238884203D322
:10A11000454A322145A015E04E48048109E0642CEF
:10A1200005D9642146A004F02FFC17B0F0BD4948C2
:10A13000C46007F065FF002801D055A052E7224611
:10A1400059A0696804F020FC17B0F0BDF06001016F
:10A1500020206C6564203D206C65643120626C6950
:10A160006E6B2068616C6620706572696F64203563
:10A17000302E2E3130303030206D730D0A0000004B
:10A18000202070776D203D2070776D206475747984
:10A1900020302E2E31303020250D0A006A736F6E6C
:10A1A000000000006170707365743A206261642081
:10A1B00076616C75650D0A00617070736574206A54
:10A1C000736F6E3A206C696E6520746F6F206C6FD0
:10A1D0006E670D0A000000006C65640070776D000A
:10A1E000617070736574206A736F6E3A206E6F20B1
:10A1F0006B6E6F776E206B657920286C65642C2000
:10A2000070776D290D0A0000617070736574206AA3
:10A21000736F6E3A207061727365206661696C0DB0
:10A220000A000000DF260000102700006C65642093
:10A2300072616E67652025752E2E25750D0A00004A
:10A2400070776D2072616E676520302E2E25750D3A
:10A250000A000000CC6A0020617070736574206A87
:10A26000736F6E3A20666C617368206661696C0D6D
:10A270000A000000756E6B6E6F776E207061726100
:10A280006D20286C65642C2070776D290D0A000004
:10A290006170707365743A20666C617368206661E2
:10A2A000696C0D0A000000002573203D20256C75A7
:10A2B0002C2073617665640D0A000000002498B0BC
:10A2C000F9A527461594661E28461294FDF7F0FF5F
:10A2D00081B2284604F098F803F004FDFE480025FA
:10A2E000807800283BD003F0FDFC6421684603F031
:10A2F00075FF002816D06846007803F0BDFA0028E4
:10A300000ED0F5490020887004F05CF8F3A52846CB
:10A31000FDF7CEFF81B2284604F076F804F062F82B
:10A32000002518E0643503F0F7F9F648854212D3AA
:10A33000E9490020887003F0EFF903F0E1F904F037
:10A3400041F8F1A00190FDF7B3FF81B2019804F04C
:10A350005BF804F047F8E04880780028C3D100217A
:10A36000C943684603F03AFF0028B5D01598002885
:10A3700005D000211591694609788142ACD0129828
:10A3800001281FD0022826D0684600781B287DD0DF
:10A3900009287CD00D287BD00A287AD0082879D0CB
:10A3A0007F2877D0014620395F2995D23F2C72D281
:10A3B000E0490855641CA4B20121684604F024F861
:10A3C000274689E7684600785B2802D00020129073
:10A3D00082E70220FBE700201290684600784128BF
:10A3E00016D04228EDD1002EEBDB761E57D4BA48AA
:10A3F0004078801BC01DC117490F0918C908C90042
:10A40000401A8101CC4809184038FDF77DFF49E02A
:10A41000B148711C02789142D3DA4078761C801BD7
:10A42000C01DC117490F0918C908C900401A810188
:10A43000C14809184038FDF767FFBE480290FDF794
:10A4400037FF85B2BDA42046FDF732FF81B220461A
:10A4500003F0DAFF0024002F0BD9BBA00190FDF719
:10A4600027FF81B2019803F0CFFF641CA4B2BC4265
:10A47000F3D3B2A42046FDF71BFF81B2204603F0C0
:10A48000C3FF002D34D02946029805E036E038E0BD
:10A49000E2E0E3E081E18EE103F0B6FF28E0A549C8
:10A4A00000200870A3480290FDF702FF85B2A3A424
:10A4B0002046FDF7FDFE81B2204603F0A5FF0024F3
:10A4C000002F0BD9A0A00190FDF7F2FE81B20198F8
:10A4D00003F09AFF641CA4B2BC42F3D397A42046B5
:10A4E000FDF7E6FE81B2204603F08EFF002DCAD1B3
:10A4F0002F469048FDF7DCFE84B2EDE60120129075
:10A50000EAE603F05FFF8B4800252F46019004F038
:10A5100092F91390224620210198FDF7DEFE0028D3
:10A5200060D1019908551399149000295AD91498AB
:10A5300004F084F9224616900199FDF7EEFE0028FA
:10A5400019D1002F0AD102A81699FDF7DDFE02A845
:10A55000FDF7AEFE85B20DE06D1EADB2A54206D987
:10A560002A4602A81699FDF7D8FE0028F4D100214A
:10A5700002A841557F1C14981399401C14908842DE
:10A58000D5D3002F64D0012F1AD0A5422BD902AF0A
:10A590003F2C5DD2AC425BD23819012103F034FF6D
:10A5A0000198395D0155641CA4B2F1E73819012105
:10A5B00003F02AFF0198395D0155641CA4B200E044
:10A5C00002AF3F2C44D2AC42F0D301992020085571
:10A5D000641C5DA5A4B22846FDF76AFE81B2284638
:10A5E00003F012FF34E059A52846FDF761FE81B261
:10A5F000284603F009FF1398002500281CD9284697
:10A6000004F01CF9074622460199FDF786FE002852
:10A610000ED13846FDF74CFE81B2384603F0F4FE09
:10A620004BA73846FDF744FE81B2384603F0ECFEF6
:10A6300013986D1C8542E2D344A52846FDF738FEE9
:10A6400081B2284603F0E0FE2146019804F0B2F9F9
:10A65000274603F0C7FE3FE60A2000E00D201590D4
:10A6600003F0B0FE39A52846FDF722FE81B2284648
:10A6700003F0CAFE2F49002008550D46287800280F
:10A6800077D0154C207800280AD06078C01D40078C
:10A69000C10D294808182946FDF711FE002868D089
:10A6A00060788101244856E00D0A434C49207265C8
:10A6B0006164792E2054797065202768656C702755
:10A6C00020666F7220636F6D6D616E64732E0D0A6C
:10A6D00063616969632D3E00504700200D0A5B6F7E
:10A6E00074615D2061626F727465642C20626163C5
:10A6F0006B20746F20434C490D0A63616969632DB7
:10A700003E000000102700000D0A5B6F74615D20A1
:10A7100069646C652074696D656F75742C20626165
:10A72000636B20746F20434C490D0A636169696350
:10A730002D3E0000E85C0020285D00200D6361696B
:10A7400069632D3E00000000200000000D0A00009B
:10A75000202000000DE008182946FDF7D5FD60789F
:10A76000401C4007400F60702078082801D2401C30
:10A770002070002004F068F9134804F0ABF813A42B
:10A780002046FDF795FD81B2204603F03DFE03F023
:10A7900029FE00242746661E9EE5002CFCD0641E80
:10A7A0000CA5A4B22846FDF783FD81B2284603F02C
:10A7B0002BFE274690E508A52846FDF779FD81B2D6
:10A7C000284603F021FE87E5E85C002063616969A3
:10A7D000632D3E00082008000700000010B50C465D
:10A7E000022812DB0EA16068FDF769FD002809D080
:10A7F0000CA16068FDF763FD002804D00AA004F0F6
:10A8000029F910BD012002F0F9FB02F0F1FB00284C
:10A8100001D003A100E003A10AA004F0B5F810BD27
:10A820006F6E00006F66660075736167653A20623F
:10A830006C656C6F67205B6F6E7C6F66665D0D0A82
:10A8400000000000626C65206C6F673A2025730D74
:10A850000A000000F8B502F063FE074602F05CFE55
:10A860000546254A25A128A004F08EF802F086FEB0
:10A8700001462CA004F088F82F48874203D12FA06E
:10A8800004F0E8F815E001F0D3FB044602F0A8FE5E
:10A8900006460A213846FDF78BFC0A460146002C85
:10A8A00001D0A06900E00020009033462BA004F006
:10A8B0006BF802F0B1FE014632A004F065F83548AD
:10A8C000854203D134A004F0C5F803E029463AA03C
:10A8D00004F05AF80AF0B4F87D21C900FDF752FCE3
:10A8E000014639A004F050F809F0B2FC01463AA044
:10A8F00004F04AF8F8BD00002200010056312E3065
:10A90000302E3334000000006669726D7761726525
:10A910003A202573202830782530386C58290D0AC4
:10A92000000000006375722062616E6B3A20415036
:10A930005025750D0A000000FF7F000063686970F4
:10A940002074656D703A2041444320726561642033
:10A9500074696D656F75740D0A0000006368697035
:10A960002074656D703A2025642E256420432028CC
:10A970006164633D2575207472696D3D256C752990
:10A980000D0A00007664643A202575206D560D0A84
:10A9900000000000FFFF000066616E2072706D3ADB
:10A9A000206E2F6120286E6F20746163686F6D6563
:10A9B000746572290D0A000066616E2072706D3A2E
:10A9C0002025750D0A000000757074696D653A20C8
:10A9D000256C7520730D0A006672656520686561D7
:10A9E000703A20257520420D0A000000F3B585B0AD
:10A9F00000200090029005980A250E46022804DAED
:10AA000075A004F027F807B0F0BD0224022823DD6A
:10AA1000A700F05980A1FDF752FC002812D0F05990
:10AA20007EA1FDF74CFC00280FD0F0597CA1FDF76A
:10AA300046FC002809D0A00031587AA003F0A4FFFA
:10AA400007B0F0BD0120009000E010250598641CBF
:10AA50008442DDDB102D0CD074687A480026049403
:10AA600001902178374630462D2933D02B2934D018
:10AA700034E073680022187816461946302805D14C
:10AA80005878782801D0582800D18B1C18780446B3
:10AA9000303C092C01D820460AE00446613C052CD4
:10AAA00001D8573804E00446413C052C05D8373816
:10AAB0001201024301265B1CE8E7002E02D00006CB
:10AAC000000E01D060A045E010460292FEF791F81A
:10AAD000064648E00127641C00E0641C21783039F8
:10AAE000092912D820783038FEF778F803905B49AE
:10AAF0003046FDF78DFE0399FDF731FE617806467D
:10AB000001203039641C0929ECD921782E291AD169
:10AB10006178641C3039092915D820783038FEF75F
:10AB20005DF80199FDF774FE3146FDF718FE064603
:10AB300044490198FDF76CFE01906078641C303840
:10AB40000928EAD901E0002802D02078002805D0A1
:10AB500043A0049903F018FF07B0F0BD002F02D006
:10AB60000120C00746402A463046009903F0D4FF32
:10AB7000102D0AD039493046FDF74AFEFF21C9059C
:10AB8000CE420ED3BF2109060DE00098012806D061
:10AB9000432237A0029903F0F7FE07B0F0BD46222A
:10ABA000F7E73F210906FDF7DAFDFEF759F80446FD
:10ABB0000A21FDF7FDFA0A214143621A00D55242EB
:10ABC0000099012906D0432301462FA003F0DCFEA3
:10ABD00007B0F0BD4623F7E775736167653A2064F7
:10ABE000697370203C76616C75653E205B665D2004
:10ABF0005B6865785D20202028652E672E206469BB
:10AC000073702033362E352C20646973702066668D
:10AC100020686578290D0A006600000068657800E4
:10AC200031360000626164206D6F64653A202573DF
:10AC300020287573652066202F20686578290D0A05
:10AC400000000000CDCCCC3D6261642068657820B6
:10AC500076616C75653A2025730D0A00000020416D
:10AC60006261642076616C75653A2025730D0A0077
:10AC7000646973706C6179203D203078256C5820B0
:10AC800025630D0A00000000646973706C6179200F
:10AC90003D2025642E25642025630D0A0000000058
:10ACA00010B50C46022812DB0EA16068FDF707FB09
:10ACB000002809D00CA16068FDF701FB002804D032
:10ACC0000AA003F0C7FE10BD012003F009FF03F046
:10ACD00001FF002801D003A100E003A10AA003F0B6
:10ACE00053FE10BD6F6E00006F666600757361677E
:10ACF000653A20646973706175746F205B6F6E7C58
:10AD00006F66665D0D0A00006175746F206469737B
:10AD1000706C61793A2025730D0A0000F0B589B096
:10AD20000C460646022801DA74A01AE07DA160688C
:10AD3000FDF7C5FA002500280CD07BA16068FDF75F
:10AD4000BEFA002806D060680178702959D05029D1
:10AD500057D061E0032E28DBA0684078002824D17A
:10AD600003E003F077FE09B0F0BD03F0B3FE002866
:10AD700002D06EA003F06EFE01263746A06807AA37
:10AD8000057806A9304603F0B3FE00280DD06846CA
:10AD900000F034FE6846808B0090312D07D0302DB6
:10ADA00010D07A2D19D05A2D17D06FA0D9E701975E
:10ADB0006946069800F0C6FD6846818B069800F04B
:10ADC00034FE11E001976946069800F0BBFD684625
:10ADD000818B069800F027FE06E00020019002908B
:10ADE0006946069800F0AEFD761CF6B2072EC5D96E
:10ADF000A16808787A2801D05A2800D162A164A0FD
:10AE000026E04178692901D049291FD181786E292E
:10AE100001D04E291AD1C01C01780A46313A072ABE
:10AE200014D24078002811D13039C8B2694608736D
:10AE300002AA04A903F05CFE002807D069465B4B18
:10AE400004980A89984207D1412306E058A0616816
:10AE500003F09AFD09B0F0BD42230020D7070FD1BF
:10AE6000401C5208C0B2D707FAD00A2808D3502293
:10AE70000A7031224B708A702630C8700D7105E05F
:10AE800050220A704B7030308870CD70032E24DB56
:10AE900003F020FE002802D024A003F0DBFDA06810
:10AEA0004178002906D101786846007B03F0D2FC86
:10AEB000012801D048A054E7A06803787A2B05D078
:10AEC0005A2B03D06A46117B4CA012E06A46117BD4
:10AED0004FA003F059FD09B0F0BD0989049800F0B6
:10AEE0009BFD002801D0012300E000236A46117B6E
:10AEF0004DA003F049FD09B0F0BD00007573616716
:10AF0000653A2064697370736574203C70696E31B2
:10AF10002D377C616C6C3E205B307C317C7A5D0D22
:10AF20000A000000616C6C00414C4C007761726E4D
:10AF3000696E673A206175746F20646973706C6123
:10AF400079206973204F4E202D207573652027646A
:10AF50006973706175746F206F6666272066697209
:10AF600073740D0A0000000075736167653A206410
:10AF700069737073657420616C6C205B307C317C0C
:10AF80007A5D0D0A00000000686967682D5A0000AC
:10AF9000616C6C203720646973706C617920706912
:10AFA0006E73203D2025730D0A000000000801404B
:10AFB0006261642070696E3A20257320287573657C
:10AFC0002070696E312E2E70696E37206F7220618D
:10AFD0006C6C290D0A00000075736167653A206486
:10AFE000697370736574203C70696E312D373E2033
:10AFF0005B307C317C7A5D0D0A00000070696E2543
:10B00000752028257329203D2025630D0A000000A6
:10B0100070696E25752028257329203D2068696791
:10B02000682D5A0D0A00000070696E2575202825CC
:10B030007329203D2025750D0A00000002F02EFD29
:10B0400000280DD007A003F005FDC82008F0C4FFBC
:10B05000BFF34F8F11491048C860BFF34F8FFEE711
:10B060000FA0F0E7666163746F72793A20666C61D5
:10B070007368207772697465206661696C65642CF9
:10B0800020726573657474696E6720616E7977618B
:10B09000792E2E2E0D0A00000400FA0500ED00E0C6
:10B0A000666163746F72792064656661756C747330
:10B0B00020726573746F7265642C20726573657499
:10B0C00074696E672E2E2E0D0A00000003A003F097
:10B0D000C1FCC82008F080FFFEE7000068616E67D1
:10B0E000696E67206E6F77202D20776174636864C6
:10B0F0006F672073686F756C642072657365742068
:10B10000696E207E3473202E2E2E0D0A0000000062
:10B1100070B51A4D0E46022819DB00240C2060433E
:10B1200029587068FDF7CBF8002807D0641C152C4F
:10B13000F4D313A0716803F027FC70BD0C204443C6
:10B1400060194268295917A003F01EFC70BD18A0B1
:10B1500003F080FC19A003F07DFC002420460C21A4
:10B16000484341194A6829580EA003F00DFC641C9D
:10B17000152CF3D314A003F06DFC70BD9C59010194
:10B18000756E6B6E6F776E20636F6D6D616E643A76
:10B190002025732028747279202768656C70272910
:10B1A0000D0A00002020252D38732025730D0A007C
:10B1B0006D6F64653A204150500D0A00636F6D6DEC
:10B1C000616E64733A0D0A006B6579733A205441DD
:10B1D00042203D20636F6D706C6574652C20555066
:10B1E0002F444F574E203D20686973746F72790D5C
:10B1F0000A00000070B50C46032823DB6068017864
:10B20000312902D0322906D01CE04078002819D11B
:10B21000184E012504E04078002813D1164E402531
:10B2200016A1A068FDF74BF800280FD014A1A06864
:10B23000FDF745F800280ED012A1A068FDF73FF8F1
:10B2400000280DD011A003F005FC70BD2946304642
:10B2500000F074FC08E02946304600F06BFC03E087
:10B260002946304600F062FC11A0A268616803F034
:10B270008BFB70BD000C0140000801406F6E0000A8
:10B280006F666600746F67676C6500007573616751
:10B29000653A206C6564203C317C323E203C6F6E08
:10B2A0007C6F66667C746F67676C653E0D0A000094
:10B2B0006C656420257320257320646F6E650D0A0C
:10B2C0000000000010B5034803F0C4FB02F000F8D2
:10B2D00010BD0000C05B0101F0B5064687B00D4609
:10B2E000002069460883022E01DA50A07FE06968D9
:10B2F00000200A788C4606AB702A01D0502A36D13D
:10B300004A78612A06D0412A04D0622A04D0422A0F
:10B3100002D02CE0524C00E0524C8A78891C303A22
:10B320000A2A24D2092A0BD80A270A787843303807
:10B3300010180F281BDC4A78491C303A092AF3D927
:10B340000978002913D146498C4201D106280EDC28
:10B35000444A944201D10D2809DC01273A46824033
:10B360003F481A80844208D10121042007E0614649
:10B370003DA003F009FB07B0F0BD0121082000F05B
:10B38000FDFC032E42DB3648844204D16846008B24
:10B390008006800F07D13348844207D16846008B6E
:10B3A0000006800F02D03BA003F054FB684600F07B
:10B3B00025FB6846008B009069460197204600F007
:10B3C000C1FAA8680178312902D030290BD00DE0EC
:10B3D000407800280AD16846018B204600F025FB02
:10B3E0003BA069680EE04078002804D03BA003F041
:10B3F00031FB07B0F0BD6846018B204600F013FB1F
:10B4000042A0696803F0C0FA07B0F0BD6846018B3E
:10B41000204600F001FB002801D0012200E00022BC
:10B420003DA0696803F0B0FA07B0F0BD75736167BD
:10B43000653A2070696E736574203C70784E3E20CA
:10B440005B307C315D20202028652E672E207069BE
:10B450006E736574207062302031290D0A0000007F
:10B4600000080140000C01406261642070696E3A7E
:10B470002025732028757365207061302E2E706131
:10B4800036202F207062302E2E70623133290D0A43
:10B49000000000007761726E696E673A205357446E
:10B4A0002F636F6E736F6C652070696E202D207234
:10B4B00065636F6E666967757265206D617920627C
:10B4C0007265616B20746865206C696E6B0D0A0093
:10B4D0002573203D20310D0A00000000757361675F
:10B4E000653A2070696E736574203C70784E3E201A
:10B4F0005B307C315D20202028303D6C6F772C2024
:10B50000313D68696768290D0A0000002573203DF8
:10B5100020300D0A000000002573203D2025750D08
:10B520000A00000006A003F095FAC82008F054FDB8
:10B53000BFF34F8F07490648C860BFF34F8FFEE740
:10B54000726573657474696E672E2E2E0D0A000085
:10B550000400FA0500ED00E010B509F071FA7D2154
:10B560000446C900FCF70EFE0246214610A003F077
:10B570000BFA08F053FC014614A003F005FA08F09A
:10B580006DFE044608F064FE024609212346C90206
:10B5900011A003F0F9F91DA003F05CFA274900207F
:10B5A0000870084608F038FD244803F053FA10BD2F
:10B5B000757074696D653A20256C75207469636BCC
:10B5C000732028256C752073290D0A007461736B34
:10B5D000733A2025750D0A00686561703A20746F12
:10B5E00074616C20257520422C20667265652025CB
:10B5F0007520422C206D696E20657665722066721A
:10B60000656520257520420D0A0000006E616D659C
:10B610002020202020202020202020202073746142
:10B62000746520207072696F2020737461636B28C9
:10B63000772920206E756D0D0A000000085B002040
:10B6400010B506A003F006FAE121C9020BA003F031
:10B650009BF9164803F0FEF910BD00007573617286
:10B6600074313A2054583D5042362052583D504291
:10B67000372028414634290D0A00000062617564B4
:10B680003A20256C752C2038206461746120626931
:10B6900074732C206E6F207061726974792C203164
:10B6A0002073746F70206269740D0A00705B010171
:10B6B00010B5E124E402204602F04AFE214602A031
:10B6C00003F062F910BD0000757361727420726539
:10B6D0007365743A20256C7520384E312C207278B1
:10B6E00020717565756520666C75736865640D0AF3
:10B6F0000000000010B506A108A003F045F90DA058
:10B7000003F0A8F91948016819A003F03DF910BD2C
:10B7100056312E30302E3334000000006669726DD1
:10B72000776172652076657273696F6E3A20257352
:10B730000D0A00006D636D2D6464632D626C653AC3
:10B7400020424C4528726474737329202B20467262
:10B75000656552544F53202B205541525428444D77
:10B760004129202B20434C490D0A000000400020B5
:10B7700053797374656D436F7265436C6F636B20AF
:10B780003D20256C7520487A0D0A0000044A0029E6
:10B79000516801D0014300E08143516070470000CF
:10B7A000401002404860704701681A4A1140016029
:10B7B0000021016041608160C160174A17499042D1
:10B7C00004D148680F22104348607047144A9042E1
:10B7D00004D14868F022104348607047114A9042F3
:10B7E00005D148680F2212021043486070470E4A84
:10B7F000904205D148680F221203104348607047F9
:10B800000A4A9042FBD148680F2212041043486054
:10B8100070470000FEFF00000800024000000240E8
:10B820001C00024030000240440002405800024028
:10B830000029016802D00122114301E0014A1140B0
:10B8400001607047FEFF0000406880B2704702460A
:10B8500009680020114200D00120704730B403680D
:10B860000D4A0C6A13408A684D6922430C692C43C7
:10B8700022438C692243CC6922434C6A22438C6A5E
:10B8800022431A430260CA6842600A6882604968BB
:10B89000C16030BC704700000F80FFFF002B01D05B
:10B8A0001061704700201061704700000149486135
:10B8B0007047000000040140054B002219685B69D5
:10B8C0000140034202D0002900D0012210467047F7
:10B8D0000004014010B4837919490268002B28D074
:10B8E0000B6893430B604A6803689A434A60027985
:10B8F000521813680468234313608A6803689A43E4
:10B900008A60CA6803689A43CA604279102A06D0DE
:10B9100051180A68006802430A6010BC70478A68C0
:10B9200003681A438A60CA6800680243CA6010BC90
:10B9300070470079401801689143016010BC70475E
:10B94000000401400B680022002B56D0F0B4012403
:10B950000B68944023424AD04B68022B01D0122B33
:10B9600016D113070AD5456A5307DB0E0F269E40F2
:10B97000B5434E699E402E43466209E0056A53076F
:10B98000DB0E0F269E40B5434E699E402E43066255
:10B990004B68012B05D0112B03D0022B01D0122BA9
:10B9A00006D14568DB06DB0FA54393402B4343607C
:10B9B0000568530003279F400E79BD43B607B60FB5
:10B9C0009E402E430660C5688E68BD439E402E4350
:10B9D000C66085680126A543CC6894402C438460EA
:10B9E000C46A9E400D69B4439D402543C5620B68FF
:10B9F000521CD340ABD1F0BC704770470549016081
:10BA0000002242600F218260416101210261C16018
:10BA100070470000FF3F00000246126900200A4202
:10BA200000D0012070478162704781617047426990
:10BA30004A4042617047000082B0EFF30884FCF78F
:10BA400055FB400701D5EFF309840AA000F0B0FBD5
:10BA5000E06800900CA0A3686268216800F0A8FB71
:10BA6000E069009014A0A3696269216900F0A0FB5D
:10BA7000FEE700000A2A2A2A20486172644661759E
:10BA80006C74202A2A2A0A00523020203D253038A2
:10BA90006C5820523120203D2530386C58205232CD
:10BAA00020203D2530386C5820523320203D253051
:10BAB000386C580A00000000523132203D253038E1
:10BAC0006C58204C5220203D2530386C5820504373
:10BAD00020203D2530386C5820785053523D253079
:10BAE000386C580A00000000014988607047000067
:10BAF000003000400249014808607047CCCC00008B
:10BB0000003000400249014808607047AAAA0000BE
:10BB1000003000400149486070470000003000409C
:10BB200001490860704700000030004010B5FFF781
:10BB30007EFF10BD10B5FFF776FF10BD10B5FFF703
:10BB400074FF10BD10B400214156FF23CAB2920702
:10BB5000D40E4278A3409207120EA24000290BDABD
:10BB60000907090F08398C081049A4006118CC692D
:10BB70009C431443CC6107E08C080D49A400611874
:10BB80000C689C4314430C60827801210078002AE1
:10BB900004D0C006C00E8140064803E0C006C00EB7
:10BBA00081400548016010BC7047000000ED00E0D6
:10BBB00000E400E000E100E080E100E0F7B5FFB064
:10BBC00004460025A5B00520EFF31087FF21009063
:10BBD000453102A8FCF761FBEFF31086FF214531E8
:10BBE00053A8FCF75AFB53A8013001909822224930
:10BBF00053A8FCF739FB012080F310880198804797
:10BC000086F3108801221D491203032653003603D0
:10BC100088420AD194421AD09C4201D1151116E0F3
:10BC2000B44210D101256D0211E0154988420AD1B4
:10BC3000944201D115460AE09C4201D11D4606E01E
:10BC40003546AC4203D000987FB028B0F0BD06ACBA
:10BC5000FF22013441320B4902A8FCF705FB012009
:10BC600080F310882846A69AA599A04787F31088E4
:10BC70007FB028B0F0BD00006C4E0101C44013003D
:10BC8000856013002C4D010110B5EFF310840121E4
:10BC900081F31088FF210906401803490968884785
:10BCA00084F3108810BD00000440002010B508483F
:10BCB000064901600749416007498160C922920035
:10BCC00006490748FCF7D0FA10BD000009490020DA
:10BCD000044000209D49002071480020104F0101C0
:10BCE0006848002010B5EFF31084012383F3108817
:10BCF000FF231B06C018034B5B68984784F310882A
:10BD000010BD0000044000200448416A0122114394
:10BD10004162416A91434162704700000010024055
:10BD2000034AD16A102399430143D162704700004E
:10BD300000100240044A0029516901D0014300E08B
:10BD4000814351617047000000100240044A0029FD
:10BD5000916A01D0014300E0814391627047000085
:10BD600000100240044A0029D16901D0014300E0DB
:10BD70008143D1617047000000100240044A00294D
:10BD8000916901D0014300E0814391617047000057
:10BD9000001002400122054912060128086802D05D
:10BDA0009043086070471043FBE70000001002401A
:10BDB00030B4164A516804231940154B01D00429A8
:10BDC00001D0036001E0134901605168124B8906FC
:10BDD000890F5B5C0168D940416053680F4C5B057B
:10BDE0005B0FE35C0D46DD40856053689B045B0F91
:10BDF000E35CD940C160D16AC90601D5084901E0B8
:10BE00007D21C903016130BC704700000010024071
:10BE10000090D0030048E801044F0101084F0101E0
:10BE200000093D0000224109094B01290BD00229DC
:10BE30000BD0596AC006C00E012383400B4200D0CC
:10BE40000122104670471968F4E7196AF2E700000A
:10BE5000001002407047000010B5FCF75DF9044681
:10BE600008F0F4FD002803D00120034900074860D2
:10BE70002046FCF755F910BD00ED00E010B50A4C66
:10BE80002069411C01D000280AD101200649342232
:10BE90000003FFF793FE2069411C03D0002801D066
:10BEA000024810BD002010BD344800205D4800202D
:10BEB000F0B5564C85B0E06921040843E06181206B
:10BEC000534D00062863534868615348286253481D
:10BED0000322016892039143016051493422801486
:10BEE000FFF76CFE4E4B4F4E18694F4F411C29D047
:10BEF000002827D0A9691A7849094901D206D20E2B
:10BF00000A43AA612168EA139143216021687F22D4
:10BF10001202914300020843206060683043606071
:10BF20006068B84360606068211508436060206AFB
:10BF30003E4908402062206AD9680902084320620D
:10BF400005B0F0BD61682046314361606168B94366
:10BF5000616061680127BF0239436160002104917B
:10BF60007D21C9000391002100917F2140240025FB
:10BF700002950191026861028A4302600E11234911
:10BF800008687F2212029043220202430A600520C1
:10BF9000FCF7A4F80120FCF7A1F81C48406B8007CF
:10BFA00004D4284603996D1C8842F3D91748C06B06
:10BFB00080B2B04201D9811B00E0311AB94202D2ED
:10BFC000E2B28FB20292B04201D3019400E0009439
:10BFD000019A00988018C005000EA04203D00446C4
:10BFE00004988142CBD8094801687F22120291430C
:10BFF000029A12020A4302604168490849004160FE
:10C0000041684907FCD405B0F0BD000000100240B3
:10C01000007000400F0800001800020000100140EE
:10C02000344800200000010000070000FF00F8FF76
:10C0300010B50A4C2069411C01D000280AD101200A
:10C04000064934220003FFF7B9FD2069411C03D0E3
:10C05000002801D0014810BD002010BD3448002048
:10C0600010B502F051F910BD10B40B06CC065B0FF1
:10C07000E40E0121A140012B07D0022B07D0143080
:10C08000002A026805D00A4304E00C30F8E71030BB
:10C09000F6E78A43026010BC7047000000298189DE
:10C0A00003D001225203114301E0024A1140818171
:10C0B00070470000FFDF0000002A828A01D00A4397
:10C0C00000E08A43828270470246128800200A42BA
:10C0D00000D00120704770B40A06530FCE06012528
:10C0E000F60E2A460024B240012B0FD0022B10D0AE
:10C0F000838A1340090A00888D402840002B02D013
:10C10000002800D00124204670BC7047838913406A
:10C11000F0E7038AEDE7000070B50446008A86B0B8
:10C120000D461B490840E98801432182A08919492D
:10C130002A890840A98811436A8902431143A181D1
:10C14000A08A15490840A9890143A1826846FFF7E2
:10C150002FFE1248844201D1039800E0029829681A
:10C16000192289005043FCF70DF806466421FCF7BC
:10C1700009F80501280964214843301A00013230CA
:10C18000FCF700F80007000F2843208106B070BDBF
:10C19000FFCF0000F3E90000FFFC00000038014081
:10C1A0008088C005C00D7047C905C90D81807047E2
:10C1B0000FB410B503A9044B044A029800F066F9C5
:10C1C00010BC08BC04B01847A1F10001C401002054
:10C1D0000FB410B504A9074B02AA039800F056F952
:10C1E000044602A9002000F0F8FC204610BC08BC60
:10C1F00004B01847DBCB00017CB515460246002091
:10C200001C4600290BD0491E00920191044B6A463E
:10C210002146284600F03AF9009A002111707CBDB1
:10C22000C5CB00012021020C01D010211046020ACA
:10C2300001D010460839020901D01046091F8208B2
:10C2400001D01046891E420801D0881E7047081A86
:10C2500070470000004870473048002030B5002883
:10C2600005D0164C021F20680023014605E0084651
:10C2700030BD904203D8034640680028F9D1002B16
:10C2800000D05968002B0AD01C68D51AA54204D1E9
:10C290001268A4181A461C6002E05A6000E022608E
:10C2A000002807D01468851AA54203D105686419CF
:10C2B000146040685060184630BD000028480020D7
:10C2C000F1B50E4C0F480C4E001B0D4FC508ED008C
:10C2D00000221146009804F02BFA002803D13068A0
:10C2E000002801D00020F8BD3C600020256060607F
:10C2F00001203060ECE700002C480020F4B300205F
:10C3000028480020F0B50020F0B51FB486B0099889
:10C31000089A030D0021024314D05148514A1818BD
:10C32000504305141198012810981AD0281A401C5F
:10C3300000264D4F4D49009601910490002812DAD5
:10C34000444211E01198012449A3012801D1109819
:10C35000C1430698119A84600360C26041600BB0CB
:10C36000F0BD4042E4E70446210500203F4A001C9E
:10C3700051410391029012E0E00707D032463B465C
:10C3800001990098FCF734FB0191009032463B463E
:10C3900010461946FCF72CFB06460F466410002C8D
:10C3A000EAD10498039B0028029A0999089806DAB2
:10C3B000FCF71EFB019B009AFCF71AFB05E0FCF75B
:10C3C0007FFB019B009AFCF77BFB04460E46002294
:10C3D000284BFCF7CBFC03D80020C043014607E004
:10C3E0000022254B20463146FCF750FAFCF776FC3C
:10C3F000102409E0002C0ADB0A220023FBF7ECFEE4
:10C40000079B30321A55641E02460A43F2D11122AC
:10C41000641C079B121B1C19119B012B03D00123C9
:10C4200008430ED10AE0084304D0112010900020E8
:10C43000119077E71098151A6D1E0BE01098824244
:10C4400002DD00236D1C03E0824201DA00236D1E31
:10C45000002BEED0069811998260C16030C07EE753
:10C4600001FCFFFF104D0000000014400000F03FF1
:10C47000300000000000F0430000E03F30380A28A0
:10C4800001D201207047002070470000FFB597B02F
:10C490000646002518E2252877D100242746FD49C5
:10C4A000049400E00443761C32780120203A904046
:10C4B0000842F7D130782A280ED00222307801467F
:10C4C0003039092916D804990A23594330394018BC
:10C4D0001443761C0490F1E7189802C80491189050
:10C4E000002904DA0120400304434842049002205A
:10C4F0000443761C30782E2814D10420044370782D
:10C50000761C2A2809D11898761C80C8189009E052
:10C510000A214F43303FC719761C30780146303925
:10C520000929F5D930786C2810D006DC4C281AD0AF
:10C5300068280ED06A2817D104E0742813D07A280E
:10C5400012D110E00120400504430CE0012109054F
:10C5500001E0032109050C437178814203D10120D8
:10C5600000052418761C761C3078119066280BD0B4
:10C5700013DC58287DD009DC00287BD04528F6D074
:10C580004628F4D047281AD1A5E118E0632835D011
:10C59000642870D0652812D19DE170286CD008DC29
:10C5A0006728F1D069287BD06E280DD06F2806D17E
:10C5B000BAE073282ED0752871D0782859D01A9AED
:10C5C000199990476D1C7EE16002400F022809D046
:10C5D00003280DD00428189801680DD00D60001DA7
:10C5E000189070E11898EA1701680D604A60F6E744
:10C5F000189801680D80F2E70D70F0E718986A4608
:10C6000001781172001D18900020507202A800904D
:10C61000012005E0189802C8189000200091C0433E
:10C6200061070DD5002101E00199491C0191B94232
:10C6300012DA8142F8DB009A515C0029F4D10BE058
:10C64000002101E00199491C01918142FADB019A24
:10C650000099895C0029F5D1019904981A9B471A21
:10C6600021463846199A00F097FA01994019451861
:10C670000BE04FE02CE113E04EE0009800990078C9
:10C68000491C00911A9A199990470198401E0190EF
:10C69000401CF2D1214638461A9B199A10E137E026
:10C6A0000A200021009001916002410F022907D069
:10C6B000189A01CA1892C2179446032908D00AE0B2
:10C6C0001898C01DC108C90005C91891944607E013
:10C6D00000B2C2179446042902D140B2C1178C4659
:10C6E00000226146944506DA0A4600214042914103
:10C6F0008C462D2102E0210504D52B216A461173B9
:10C70000012103E0E10701D02021F7E7029155E084
:10C710000A200AE0102008E01020009000210420E8
:10C7200004430191082703E00820002101910090B3
:10C730006002410F022907D0189A01CA18920022FC
:10C740009446032908D008E01898C01DC108C90004
:10C7500005C91891944603E080B2042900D1C0B203
:10C7600000210291210729D51199702906D0009A3C
:10C770001021019B4A401A4305D00EE040216A4631
:10C780001173012108E06146014306D030216A4659
:10C7900011731199517302210291009A0821019B92
:10C7A0004A401A430AD16146014301D1610705D5C8
:10C7B00030216A46117301217F1E02911199582977
:10C7C00004D035A10E910DA90D910DE037A1F9E727
:10C7D0006146019B009AFBF7FFFC0E9B8C469B5C1D
:10C7E0000D9A521E0D92137061460143F0D10D98BF
:10C7F00005A9081A20300190600703D50120000424
:10C80000844300E001270198874201DD381A00E0E7
:10C810000020019900904118029809180498401AC4
:10C820000490E00306D421461A9B199A049800F05C
:10C83000B3F94519002706E003A81A9AC05D1999B3
:10C8400090476D1C7F1C02988742F5DBE0030CD5F6
:10C8500021461A9B199A049800F09EF9451904E0A4
:10C860001A9A3020199990476D1C0099481E009023
:10C870000029F5DC08E00D980D990078491C0D9110
:10C880001A9A199990476D1C0199481E0190002928
:10C89000F1DC63E1092801003031323334353637B9
:10C8A00038396162636465660000000030313233FC
:10C8B000343536373839414243444546000000009C
:10C8C00000F05AF94519761C3078002800D0E2E5CE
:10C8D00028461BB0F0BD600700D406271898C01D7D
:10C8E000C108C90048680A680831C30FDB071891FE
:10C8F000190001D09CA108E0210501D59BA104E00D
:10C90000E10701D09AA100E09AA1430011985B08C9
:10C91000109165280CD006DC452809D046281DD08A
:10C92000472841D141E0662818D067283CD13CE037
:10C930000021112F01DB112000E0781C01910090F3
:10C9400008A911A8FFF7E0FC139905910021119A9D
:10C9500015927F1C12980197009150E00120C007AA
:10C9600003900120019008A9009711A8FFF7CCFCC3
:10C97000139A149905920022119B00921298159314
:10C98000059A0192002901D0104602E0791C401856
:10C990000190381A01D5019804E04042401E0090F1
:10C9A000781C0190C01B029043E0012F00DA0127A0
:10C9B0000021112F01DD112000E038460191009087
:10C9C00008A911A8FFF7A0FC13990591119A00215D
:10C9D000129815920091019721070CD40599B9423C
:10C9E00001DB019900E00191012904DD159A491E3E
:10C9F000515C302906D0B84201DA011D05DA012167
:10CA0000029115E00199491EEDE7002805DC009927
:10CA1000411800910199091A03E0019A411C9142C1
:10CA200000DD01910099401A401C02900120C007CE
:10CA30000390200706D402990198814202DB00206E
:10CA4000C043029000206946C87707AF01210398D0
:10CA50000337C907884224D0022011902B2012905E
:10CA6000039800280CDA404203902D20129007E032
:10CA70000A210398FBF786FB30317F1E0390397043
:10CA80001199481E11900029F2DC03980028EFD17B
:10CA9000791E129808703078202108404530BF1E5A
:10CAA000387006A8C01BC01D03901098007800289D
:10CAB00000D00120019941180298C0170918039865
:10CAC00009180498401A401E0490E00306D4214639
:10CAD0001A9B199A049800F05FF84519109800788D
:10CAE000002803D01A9A199990476D1CE00324D5A9
:10CAF00021461A9B199A049800F04EF845191CE03B
:10CB00000098002807DB00990598884203DD1598F6
:10CB1000405C199901E0199930201A9A90470098C1
:10CB20006D1C401C00900298401E0290002804D109
:10CB30001A9A2E20199990476D1C0199481E019050
:10CB40000029DDDC05E038781A9A7F1C1999904796
:10CB50006D1C0399481E03900029F4DC21461A9BA2
:10CB6000199A0498ACE600002D0000002B0000008C
:10CB70002000000000000000F8B5044600251E4615
:10CB80001746880404D405E039462020B0476D1CC0
:10CB9000641EF9D52846F8BDFFB50446002581B0CE
:10CBA0001E46C80301D5302700E02027880404D59D
:10CBB00005E038460399B0476D1C641EF9D5284638
:10CBC00005B0F0BD4A68002A06D00A68531C0B6005
:10CBD00010704868401E486070470A68531C0B601C
:10CBE00010707047002903D0002801D0884201D17D
:10CBF000002070478268002A08D05268002A03D0BB
:10CC000011604A608068416001207047816049601E
:10CC100000200860F8E7FFB581B007000A981446C5
:10CC20000D4605D0002D03D0002C01D0A74202D123
:10CC3000002005B0F0BD01267602002802D0E06891
:10CC4000304307E02846049901F0B2FD051EF0D0FC
:10CC5000E068B0430646A089800505D4206A002814
:10CC600002D0049949688847E66021463846256223
:10CC7000FFF7B8FF05B0F0BD00B599B06021684678
:10CC8000FBF70BFB042008AAD07012A000680190EB
:10CC90000B2010AAD070024610A109A8FBF7E4FAF5
:10CCA000002010AA107101215171D07191719073FF
:10CCB0001175D082A02010839176B4209083192022
:10CCC000C001D08308480090684603F0EFFF19B018
:10CCD00000BD000003160A18000000000AFFFFFF55
:10CCE0004E6174696F6E7300EDCC000170470000F7
:10CCF00010B507490020087000F07AF9002802D02A
:10CD000004A0FFF755FAF72004F044F910BD000025
:10CD1000374700205B424C455D20636F6E6E656354
:10CD20007465640D0A00000010B503F0E3FF00F025
:10CD30006DF905490020087000F05AF9002802D06A
:10CD400002A0FFF735FA10BD374700205B424C4583
:10CD50005D20646973636F6E6E65637465642C2017
:10CD60006164766572746973696E67207265737445
:10CD700061727465640D0A0010B58CB000240094D3
:10CD800001940294039404940594069407940894DF
:10CD900009940A94FFF772F8002804D0014601A80C
:10CDA000FCF7FCFB07E012A001886A4691804188ED
:10CDB000D180808810816946CC704C810A208870AF
:10CDC00012220A7303A80CA10130FBF74DFA0C20C4
:10CDD0006946088418204884FF208C84F530C88474
:10CDE0000A480885684604F023F80CB010BD00001E
:10CDF000010203040506000043414949432D4D4308
:10CE00004D2D323032363039303200008813000078
:10CE100000B583B00D4900910D49002001910290A9
:10CE200069460872684604F007F9FFF7A5FF00F0AD
:10CE300027FAFFF721FF074803F0A4FE064803F096
:10CE4000A1FE03F057FF03B000BD00005DCE00015E
:10CE5000E1DC0001B9D30001C9DA000170B5007846
:10CE6000012811D000250F4C02280ED003280BD129
:10CE700003F040FF00F0CAF8257000F0B9F8002870
:10CE800002D00948FFF794F970BD257000F0B0F8A2
:10CE9000002802D00548FFF78BF9F72004F07AF854
:10CEA00070BD0000374700204CCD000114CD0001BB
:10CEB000F8B50646244F0020388178810124481EA9
:10CEC0000D463E2814D80A4631462048FBF7CCF9D7
:10CED0001E49002048551E4801F0B6FD1B4801F0D0
:10CEE000F9FC0446002001F0AFFD388900280CD180
:10CEF000002C12D017A00090FBF7DAF984B222467A
:10CF000019480099FBF7B0F93C81B878002819D08E
:10CF100016A0FFF74DF900240CE019A0EBE7315DF6
:10CF2000084620385F2800D32E2117A0FFF740F9CC
:10CF3000641CA4B2AC4201D23F2CF0D3398913A0B7
:10CF4000FFF736F9F8BD00005A470020286100209D
:10CF50001DEA0001756E6B6E6F776E20636F6D6DED
:10CF6000616E640D0A000000A36400205B424C4522
:10CF70005D20636C6920657865633A2022000000BB
:10CF80006F6B0D0A000000002563000022202D3E7B
:10CF900020257542207273700D0A000030B40C49D0
:10CFA000098E182902D3891E8AB200E01422094C86
:10CFB000094D63892189ED18C91A89B2914200D9B6
:10CFC00011465A1862810180284630BC7047000023
:10CFD000D84D00205A470020A364002003480021B8
:10CFE00001708180C1804170704700005A47002065
:10CFF00001488078704700005A470020002800D080
:10D0000001200149887070475A47002010B5054932
:10D01000002008708880488100F054FF00F070FB09
:10D0200010BD00005A470020F3B583B004980024D7
:10D0300000287AD95B4802905B4A03981178005D1A
:10D04000002904D001290BD002291AD122E0CA28D4
:10D050006CD156490870012090800521D18017E0DD
:10D06000524B91885854491C88B2908005285DD154
:10D070000298417803780802FF211843E131884281
:10D0800003D900201070908084E0C01DD080022061
:10D0900010707FE0444A454B91885854491C88B22F
:10D0A0009080D188884275D102980022417800781A
:10D0B0000D0205433E488446281D86B23D48002E99
:10D0C00014D93D4F6146895C0902484000210304A0
:10D0D00002D54000784000E04000491CC9B280B24F
:10D0E0000829F4D3521C92B2B242EBD32F4E7119DD
:10D0F0008A794B7911021943884247D17778B07801
:10D1000001902948761D8078002806D03346009586
:10D1100039462AA0019A05F0FFFE112F2AD006DC1D
:10D12000012F09D0102F31D124E039E032E0122F45
:10D1300020D0202F2AD124E001273F2D11D82A46C4
:10D1400031461F48FBF790F81D49002048551D48FF
:10D1500001F07AFC1A4801F0BDFB0746002001F0FF
:10D1600073FC6846077001236A460320019900F0AA
:10D170002BF80BE02B4632463846019900F090FB25
:10D1800004E02A463146019800F004FA06480021DE
:10D1900001708180641C0498A4B2844200D24BE7E1
:10D1A00005B0F0BDAB6100205A470020A861002007
:10D1B000A9610020FFFF000021100000525800006C
:10D1C00068610020E12E0101FFB5D81D80B283B057
:10D1D0001D460190FB2803D90020C04307B0F0BDD5
:10D1E000214CCA202070039860700498A070280A0F
:10D1F000E5702071002D04D02A46601D0599FBF7CB
:10D2000033F8281D83B2194F19480024002B13D975
:10D21000184E395D090248400021020402D5400041
:10D22000704000E04000491CC9B280B20829F4D324
:10D23000641CA4B29C42ECD30B4949194871000A02
:10D2400088710D488078002806D000950BA0059BBA
:10D25000049A039905F060FE0348019900F03AFE34
:10D26000002007B0F0BD0000A8630020A9630020E3
:10D27000FFFF0000211000005A4700205458000012
:10D2800000B587B0002001900090039004906A469A
:10D29000069010730C4902910521917003231370BD
:10D2A0001023D3705070107101235371907150731B
:10D2B000064805907D20917300011082104604F00D
:10D2C00081FB07B000BD000040E2010000B0030197
:10D2D00001490120887070475047002010B502486E
:10D2E00004F018F9002010BD7C4E00202F48007972
:10D2F00000285AD1F8B56D202C23032207214001C4
:10D300000AF41AD4A0210446017029480027C178E4
:10D31000617027710321E180677201266671072120
:10D32000244D2177A9796177687B002803D0E780B5
:10D33000032060710EE0E87900280BD0A87902285C
:10D3400000D166772671E6802046A97920304170A9
:10D350008670077015488079022804D0032815D0FC
:10D3600004281BD116E004F01FFB00280BD0052079
:10D37000E0806771688A6061688AA06120460A302F
:10D3800004F040F90AE0094903208871288B6061A4
:10D39000288B02E0E88B6061E88BA061034806718E
:10D3A000467120460AF404D4F8BD7047D84D0020D9
:10D3B0005C4E0020C84E002010B584B00A23032222
:10D3C000072110480AF4B8D31B21017000214170D5
:10D3D0001424448003228280C1800B4A02810AF413
:10D3E000E7D36846048009480190684603F0ECFDE5
:10D3F000684604810648039002A805F0E3F904B0EA
:10D4000010BD00001B0D0000FF0100004458010189
:10D410006DEE0001FFB585B0054602A800901C46E0
:10D420002846069904F018FB6846007A002866D062
:10D4300006980090280A334A019403900E2826D0BB
:10D44000314800240178002951D92F48E1000818FB
:10D45000828803998A4240D1009A81689646019A4F
:10D46000284694460A791206120E36D00968254BD2
:10D47000D700083FCE1937887668BFB2874201D0FF
:10D480009F4226D1634603227146B04725E01F49DB
:10D49000681809282BD800981D49844608792E461B
:10D4A00000062346000E1ED0C4000F68083C3C193D
:10D4B00027886468BFB2B74201D0974204D10322E3
:10D4C00061462846A0470EE0401E0006000EEBD144
:10D4D00009E0521E1206120ECAD10B48641C0078D5
:10D4E000E4B2A042B1D86846007A002807D00948C3
:10D4F000426C002A02D0284606999047002009B0C5
:10D50000F0BD0000FFFF0000844D0020EEF1FFFFA2
:10D5100094530101D84D002000487047FFFF0000E0
:10D5200070B5124D01212846FCF784F9142006F04D
:10D5300053FD702002F0F4FF702002F0F1FF04466A
:10D5400000212846FCF776F90948448009488442BE
:10D5500001D1401070BD2046FCF7A2F80649FBF748
:10D5600057F9FBF77DFB00B270BD000000080240D8
:10D57000A4470020FFFF00000000204110B500F08C
:10D580008BF90349884201D1022010BD012010BD52
:10D5900000400201F0B5074600208DB015460E464A
:10D5A000002A04D0012D04D13178FF2901D10B4E7E
:10D5B00007250024002D08D90146325D684602F097
:10D5C000E5FF641CA4B2AC42F6D303466A46394672
:10D5D0002120FFF7F9FD0DB0F0BD0000985A0101C0
:10D5E0000148408870470000A447002070B50646F7
:10D5F0000020074D044601462A5D064802F0C6FF9A
:10D60000641CA4B2072CF6D33080024870BD000021
:10D61000985A01019A6A002010B5602002F080FF3C
:10D620000449884201D1002010BD6021FCF762F856
:10D6300080B210BDFFFF000010B503F031FF0448B9
:10D640000169002901D004208847002010BD000096
:10D65000E84E002070B5224C606B224DC00722D0EE
:10D66000A06B21497E2209685143401A2988491E2E
:10D6700029804B21C90040181C49884213D300203F
:10D680002880206A40084000206219490868020486
:10D69000930F184A01D0904300E0104308601648E9
:10D6A000407F03F035FC298801200029216B07D039
:10D6B000014321630522032110480AF4FFD40DE041
:10D6C000FF22120291432163216B05229202114332
:10D6D0002163216B0143216304F0B4F9002070BD84
:10D6E00000100240344700208C000020B1040000EC
:10D6F0000010014000C00000384E0020010F000063
:10D70000044800210170016241628162016301717C
:10D71000417170476847002002480021C1710181B2
:10D720007047000068470020054A91890180002960
:10D7300001D00120907000209081024870470000C5
:10D74000684700208A6A0020F7B5414982B08A63A1
:10D7500003980024002879D93E483F4F00903C4A66
:10D760000298D179005D002904D001290CD002294A
:10D770001BD128E0CA2864D13849087001211181E1
:10D7800005205081D1715CE0344B11895854491CFB
:10D7900088B21081052854D1009841780378080296
:10D7A000FF211843E131884203D90020D071108154
:10D7B00047E0C01D80B25081052802D00220D07100
:10D7C0003FE00020FBE7224A244D11896854491CA0
:10D7D00088B210815189884233D10098204D417818
:10D7E0000278080210430346001D81B24A1E1D48FC
:10D7F00096B2002914D029780902484000216D1CF6
:10D80000020402D54000784000E04000491CC9B243
:10D8100080B20829F4D33146761EB6B20029EAD187
:10D820000E4AD1188D794E7929023143884204D1AC
:10D8300091785078521D00F033F805480021C171ED
:10D840000181641C0398A4B2844288D305B0F0BD62
:10D8500068470020A668002021100000A36800206F
:10D86000A4680020FFFF000010B5024AFFF76CFF1C
:10D8700010BD0000211B010101B5054A01216846C8
:10D88000FFF762FF0349002288798A7108BD000012
:10D89000351F0101684700200048704700800001E3
:10D8A000F0B51D464E4E83B013460C46102815D0D9
:10D8B00011287AD0122879D013280DD1FFF720FF34
:10D8C000002213212046336A04F0E4FA4548B16B84
:10D8D000814201D10120B07103B0F0BD1446009126
:10D8E0000C2D09D0102D07D0002301221021009803
:10D8F00004F0D0FA03B0F0BD104604F0B9FA0746C0
:10D90000201D04F0B5FA02902046083004F0B0FA69
:10D910000190102D0BD00025307800280DD0022268
:10D920001021336A009804F0B5FA03B0F0BD204628
:10D930000C3004F09DFA0546EEE72B482B492C4CA1
:10D94000884202D0A0420CD10C462A49381F884296
:10D950000FD3002303221021009804F09BFA03B098
:10D96000F0BD002302221021009804F093FA03B0C6
:10D97000F0BD7078002803D1FEF798F9012070708F
:10D9800001203070776134610298B0610198002104
:10D9900031627162B1623163F061E80707D011480A
:10D9A000B26B824203D1012002E00BE011E00020C3
:10D9B0003071717100231A461021009804F06AFA40
:10D9C00003B0F0BD2A461946204604F0BBF803B068
:10D9D000F0BD2A461946204604F072F903B0F0BDA6
:10D9E00068470020351F0101008000010080000110
:10D9F00000400201FDBF010010B50E4CE078002888
:10DA000016D007F01DF8616B401AA178002903D0E9
:10DA1000FF212D31884203D27D210901884207D39D
:10DA2000BFF34F8F05490448C860BFF34F8FFEE72F
:10DA300010BD0000684700200400FA0500ED00E07A
:10DA4000F8B5342211491248FAF70EFC104C114F68
:10DA500020680125104EB8420BD16068012808D11A
:10DA60002046302100F0B8FE216B884201D135708C
:10DA7000F8BD34210648FAF710FCFF202760F53086
:10DA8000656020810020E0603070F8BD006000011A
:10DA9000CC6A00207ADA12CAB047002010B53421CF
:10DAA0000748FAF7FAFB0648064901600121416080
:10DAB000FF21F53101810021C16004F0A1FA10BD00
:10DAC000CC6A00207ADA12CA10B584B0142303227B
:10DAD000072112480AF430D01B2101700021417047
:10DAE0004724448003228280C1800D4AC2600D4ACF
:10DAF00002610D2202720AF45BD0684604800A4873
:10DB00000190684603F060FA684604810748039074
:10DB100002A804F057FE04B010BD00001B0D000069
:10DB200064580101545801014C580101613601014A
:10DB300000207047F8B5184D184FE879002801D03B
:10DB40002E7B00E0FE780322331D0721144809F4E0
:10DB5000F3D7A921044601701248C17861700021F1
:10DB60006180E8791049002803D02A7B896C201D48
:10DB700002E0FA78201D091DFAF776FB6088022181
:10DB80008019608007480279062A00D0017141712E
:10DB900020460AF40DD0F8BDC84E0020A84E002043
:10DBA000A60D0000D84D0020884E0020F8B51F2695
:10DBB000232303220721284809F4BED70446AA20BC
:10DBC000264F2070F878264D6070E8786080EA78FB
:10DBD0002449201DFAF748FB6288B01AC1B2201D03
:10DBE0001018214A0326032910D92B79002B0DD0B8
:10DBF0000670192343705389091F1B0AC370937A57
:10DC000083706388C9B21B1D6380001D02291AD965
:10DC10006B79002B17D0137B891E8B4200D21946DB
:10DC2000CDB2691C0170117BA94201D1092100E02C
:10DC3000082141702A460D49801CFAF715FB6088BF
:10DC4000AD1C401960803879062800D03E717E7185
:10DC5000204609F4ADD7F8BDA60D0000D84D002030
:10DC6000C84E0020AC4E00205C4E0020694E0020C3
:10DC700070B53A2303220721164809F45DD7A42181
:10DC8000154D04460170E8786070A97913480022A8
:10DC9000022910D0032913D0042916D062802271E2
:10DCA000807902F06DFD05202871042068712046FE
:10DCB00009F47ED770BD018A642359436180EEE781
:10DCC000C18A642359436180E9E7818B6423594306
:10DCD0006180E4E7A10D0000D84D0020C84E00206F
:10DCE0007047000010B506F09BFE022803D106F035
:10DCF000A7FE0149086010BD3847002010B58620F6
:10DD0000FEF790F8002802D00FA0FEF751FAFDF7B9
:10DD1000FBFF01210807FEF725F801210846FDF762
:10DD200035FD1148FDF7FCFE0520FDF7F3FE7D20D3
:10DD3000C000FDF7D9FEFDF7E5FEFDF7DBFE0B4960
:10DD40000020086010BD0000204C617374207265D3
:10DD50007365743A20495744472077617463686457
:10DD60006F67210A00000000555500003847002069
:10DD7000FFB50F4683B00021009101911646694618
:10DD8000FBF712FC040030D10521C9026846FBF7FD
:10DD900011FC002828D121496846FBF70BFC00281C
:10DDA00022D11F496846FBF705FC00281CD11D49FC
:10DDB0006846FBF7FFFB002816D1292109026846B7
:10DDC000FBF7F8FB00280FD117496846FBF7F2FB79
:10DDD000002809D115496846FBF7ECFB002803D160
:10DDE00000988088C10B03D00624204607B0F0BD00
:10DDF00000050099000D0D186888B04200D2072474
:10DE00002988B819884201D90D24EEE7A8193A46A5
:10DE1000001D0699FAF728FA6F80E6E7012800004E
:10DE20000328000002280000022900000329000046
:10DE3000084C06F0F5FD022802D106F001FE206034
:10DE40001DF4AED200F012F8FFF7D6FD012006F067
:10DE5000C3F8EEE73847002010B5034900200870EA
:10DE600000F004F810BD00005447002012480021C3
:10DE7000007800281FD070B5104D86B02878002893
:10DE800017D1A8886C88A04213D00D4E6A4680B284
:10DE9000A04209D0335C5354401CC005491CC00D3E
:10DEA00089B2A8801429F2D301202870104605F009
:10DEB000DBFB06B070BD7047374700205447002099
:10DEC000285F002002490020488088800870704741
:10DED00054470020F0B484460D480078002814D040
:10DEE0000022002911D90B480B4D878843881C4616
:10DEF0005B1CDB05DB0DBB4207D06646B65C521CE3
:10DF00002E5592B243808A42F0D3F0BC7047000095
:10DF10003747002054470020285F002070B5134D7C
:10DF200004462878002803D1FDF7C0FE01202870A0
:10DF30000F4820602821204600F04EFC0D4DA062C5
:10DF40002846FDF7A1FE00280DD12C2221462846A7
:10DF5000FDF7C8FE002806D12C2229462046FAF7F4
:10DF6000C6F9002800D0012070BD0000B247002093
:10DF700011C011CA0040000110B5044600681949DB
:10DF8000884208D12046282100F026FCA16A884258
:10DF900001D115A200E016A21B491CA000F0F4FC60
:10DFA00021A0216800F0F0FC26A0616800F0ECFCE4
:10DFB0002AA02369E268A16800F0E6FC33A0616949
:10DFC00000F0E2FC37A0236AE269A16900F0DCFC02
:10DFD0002EA0616A00F0D8FC3EA0A16A00F0D4FC3B
:10DFE00010BD000011C011CA76616C6964000000A8
:10DFF000494E56414C49442028626164206D616756
:10E0000069632F637263290000400001626F6F74BF
:10E0100073657474696E6720402030782530386CE1
:10E02000583A2025730D0A0020206D61676963202E
:10E030002020202020203D2030782530386C580DBD
:10E040000A00000020206163746976655F62616E7A
:10E050006B203D20256C750D0A00000020206261B8
:10E060006E6B313A20616464723D30782530386CD3
:10E07000582073697A653D256C75206372633D3065
:10E08000782530386C580D0A000000002020202030
:10E0900020202020207665723D30782530386C585D
:10E0A0000D0A0000202062616E6B323A20616464C8
:10E0B000723D30782530386C582073697A653D257B
:10E0C0006C75206372633D30782530386C580D0ACA
:10E0D00000000000202063726333322020202020C3
:10E0E00020203D2030782530386C580D0A00000083
:10E0F00030B58DB001210820FDF740FE01218803D5
:10E10000FDF73CFE02A8FDF779FC402002900220BA
:10E110002C4D0424039002A907942846FDF712FC15
:10E1200080210794029102A92846FDF70BFCE1200B
:10E13000C0020890002069468884C88408858885C4
:10E140000C204885204D08A92846FDF7E5FF012150
:10E150000846FDF7EFFD1D4C2046FDF725FB01238A
:10E1600022461B490220FDF799FB01228021284607
:10E17000FDF7A2FF00220121402006F0AFF8154C68
:10E18000032260600021012006F0A8F8A0600120B1
:10E1900006F092F8E06000F077F801220E49284678
:10E1A000FDF762FF1C2069460870032048700120BB
:10E1B00088706846FDF7C6FC01212846FDF76EFF12
:10E1C0000DB030BD000C0140003801400800024095
:10E1D000000002403C47002024040000F3B5274F14
:10E1E00081B00C460025786800280AD006F018FC9B
:10E1F000022806D100220199786806F0C9F90128A1
:10E2000016D01F48FDF720FB03218902081A398820
:10E2100080B281420ED01B483988415C0198017060
:10E22000032138888902401CF9F7ACFF39800120AE
:10E2300003B0F0BD002C0AD0601C01D0A54206D26C
:10E24000B868002803D006F0EBFB022802D00020BB
:10E2500003B0F0BD1426601C03D0601B142800D24C
:10E2600006467D213046C9004843F9F78BFF014639
:10E27000B86806F02EFAAD19B5E700003C4700205B
:10E280001C000240084F002030B5194D8BB0002112
:10E290002846FDF7CDFA2846FDF786FA01232A46DF
:10E2A00014490320FDF7FAFA13480090134801902F
:10E2B00003208002039000248020059020200890F5
:10E2C00004940002029409900694079469460A9403
:10E2D0002846FDF7C3FA0A48048001212846FDF7C5
:10E2E000A7FA012240210748FDF7E6FE0BB030BD3A
:10E2F0001C0002400000024004380140084F00208A
:10E300003C4700200038014038B500200D4C0090FB
:10E310000B492046FDF7DFFE002810D02046FDF710
:10E320003FFF09488068002802D0694606F0F6F8E9
:10E330000098002803D0012004490007486038BD38
:10E3400024040000003801403C47002000ED00E0BC
:10E3500030B5194D85B0044640212846FDF7B4FE7E
:10E360000028F9D000212846FDF798FE00206946D4
:10E3700000948880C880088188810C2048812846C4
:10E38000FDF7CAFEFFF780FF0C4C6068002807D03D
:10E3900006F046FB022803D10021606805F0C0FFAB
:10E3A000012207492846FDF75FFE01212846FDF7B7
:10E3B00075FE05B030BD0000003801403C4700202C
:10E3C0002404000010B5064CE068002807D006F0D1
:10E3D00027FB022803D1C11EE06806F07AF910BDC0
:10E3E0003C47002010B5074CE068002809D006F033
:10E3F00017FB022805D100231A461946E06805F0EC
:10E40000C6FF10BD3C47002000283FD000293DD06A
:10E41000F0B51F4E0C4605468BB000213046FDF787
:10E4200007FA1C4F02203946FDF7BCF91A48009044
:10E430001020029000208021059104900321019575
:10E440000394090306900790089009910A90694681
:10E450003046FDF703FA01213046FDF7E9F9394668
:10E460000220FDF7F4F90028F9D000213046FDF72D
:10E47000DFF939460220FDF795F9084C4021204686
:10E48000FDF722FE0028F9D00BB0F0BD7047000068
:10E4900008000240000002400438014000380140FA
:10E4A00010B4002807D00368002B04D042688168AC
:10E4B000914201D206E0002010BC7047491C8160E7
:10E4C000002804D0914202D25C5C202CF6D9914203
:10E4D000F2D1491E816010BC70470000F8B50C46AF
:10E4E00005461046194600F013F806460020009035
:10E4F000064B324621462846FEF78DFB0028304663
:10E5000002D100F043F80020F8BD0000BC47002015
:10E5100070B505460E46124800F0A2F804001CD063
:10E52000E6610820A561E0600E4A0F4B284631469F
:10E53000FAF71CFC02D80D4860610EE000220C4B7B
:10E5400028463146FAF7FEFB02D80120C00703E057
:10E5500028463146FAF79EFB6061204670BD0000F8
:10E56000BC4700200000C0FFFFFFDF41FFFFFF7F2F
:10E570000000E0C110B5044800F072F8002801D096
:10E580004021C16010BD0000BC470020002824D0FD
:10E59000F8B5124E04460027A0892568C0050DD4A1
:10E5A000A068002804D0FFF7F1FFA089C00505D4BA
:10E5B0002069002802D0716888472761A0898005FA
:10E5C00005D4206A002802D07168884727627168E4
:10E5D000204688472C00DFD1F8BD7047BC4700209B
:10E5E00010B5002201F0F4FE10BD000030B4124A54
:10E5F0000E4D0F4B0F4C0028136013D001680029FB
:10E6000000D0116054604068002800D050600020A5
:10E6100090601068984203D15068A04200D1956084
:10E6200030BC70479560546030BC7047BD3A010102
:10E63000C1C200015DC20001BC470020002803D018
:10E64000007B082801D00020704701207047002877
:10E6500003D0007B402801D0002070470120704784
:10E6600010B501682820884700280AD000210160E1
:10E6700041608160C160016141618161C16101628C
:10E68000416210BD70B5002604463546002808D00A
:10E69000F9F70EFE411C2B463246204600F004F8E6
:10E6A00070BD002070BD0000FFB5002489B0064693
:10E6B00000940194344802940394049405940694BD
:10E6C000046015464460002E5AD000293FD002460F
:10E6D00000960191D16890681269049006920591A4
:10E6E0002A48FFF7BDFF0790002830D000986F46FA
:10E6F000002802D00298002801D000200DE00198E7
:10E70000042809D9032222A10098F9F706FE00285F
:10E7100002D10298C01C02903846FFF7C1FE0146A4
:10E72000079803F0D3FD00280ED00C98002814D0D1
:10E730006846FFF7B5FE02990198814204D202991A
:10E740000098405C002808D00798FFF71FFF019948
:10E75000029888420AD204460BE0002D03D00299A9
:10E7600000984018286007980DB0F0BD081E00D032
:10E77000441E002D01D03019286003480660446013
:10E7800000200DB0F0BD0000B4470020BC470020C1
:10E79000EFBBBF0010B5024A002104F0B5F810BD70
:10E7A000BC4700200149496808470000BC470020D9
:10E7B000002810D070B50E460446F9F779FD401CCC
:10E7C000336805469847061E04D02A462146F9F7C5
:10E7D0004BFD304670BD7047002230B4D243491E15
:10E7E0000FD3094C03785A400023401C5508D20728
:10E7F00000D022465B1C6A40DBB2082BF6D3491ED0
:10E80000F0D230BCD04370472083B8ED02468B88ED
:10E810000020022B01D00D207047C988002A05D0A6
:10E820000029F9D00129F7D0812070470029FCD0B8
:10E830000229F9D17047152070470000152804D22D
:10E840000C214843024908587047002070470000D7
:10E850009C59010110B588B00C4607AA06A900F022
:10E8600047F9002811D06846FDF7C8F86846808B44
:10E8700000900120312C0CD0302C15D07A2C1ED0D9
:10E880005A2C1CD0002008B010BD0020C04308B096
:10E8900010BD019069460698FDF754F86846818BD3
:10E8A0000698FDF7C2F811E0019069460698FDF759
:10E8B00049F86846818B0698FDF7B5F806E0002018
:10E8C0000190029069460698FDF73CF8012008B0D7
:10E8D00010BD000070B588B000246A46234616E0DB
:10E8E000401C01782029FBD00929F9D00906090E1E
:10E8F00012D0A1005050641C00E0401C0178002997
:10E900000AD0202901D00929F7D10370401C0178D1
:10E91000002901D0082CE4DB002C14D0104E002577
:10E9200028460C21484331580098F9F7C8FC0028C4
:10E930000CD06D1C152DF3D30AA0009900F024F81B
:10E94000012008B070BD002008B070BD0C20454308
:10E95000A8198268694620469047002008B070BD1B
:10E960009C590101756E6B6E6F776E20636F6D6DD4
:10E97000616E643A202573202874727920276865B7
:10E980006C7027290D0A00000FB410B503AB60218D
:10E990000648029AFDF730FC05490020C877034875
:10E9A00000F058F810BC08BC04B01847885C002080
:10E9B000C85C0020F3B581B00D460198F9F778FCEA
:10E9C000144C86B22046F9F773FC81B22046FFF75B
:10E9D0001BFD0024002D0BD90F4F3846F9F768FCBA
:10E9E00081B23846FFF710FD641CA4B2AC42F3D3E9
:10E9F000084C2046F9F75CFC81B22046FFF704FD85
:10EA0000002E03D031460198FFF7FEFC304603B0DC
:10EA1000F0BD00003CA7000148A7000130B401256B
:10EA2000074B084CAD0203E06254491C1981401C9D
:10EA30000278002A02D01989A942F5D330BC704768
:10EA40005A470020A3640020014908607047000075
:10EA50004C47002010B507490968002901D08847B4
:10EA600010BD0446F9F724FC81B22046FFF7CCFC28
:10EA700010BD00004C470020F0B51FB405460398B8
:10EA8000144646000198760847007F08334628461A
:10EA90003946FAF76BF902D22846394601E020469A
:10EAA00031463322D243FAF783F806460F46224610
:10EAB0002846039B0199F9F78DFF490049083B4619
:10EAC0003246FAF73FF902D8012005B0F0BD002028
:10EAD00005B0F0BD0148807870470000A8470020CD
:10EAE000002800D00120014988707047A847002005
:10EAF000431E072B01D300207047C3000548181898
:10EB00000346803B9B6F40380B60808F1080012054
:10EB100070470000A85A0101024B586019705A70E2
:10EB200070470000A847002001250024794E8AB0D4
:10EB300027466846FCF762FFE0008119898800914A
:10EB40000197029730586946FCF7FCFE641CE4B25A
:10EB5000072CEED3FFF7C6F86F498878002814D049
:10EB6000486801250A7802924A78002106AC019192
:10EB7000FF236354491CC9B20529F9D3102A1CD0BC
:10EB8000D905C8423BD301213AE0002D7ED00024B4
:10EB9000604D26466846FCF731FFE0004119898840
:10EBA00000910196029628586946FCF7CBFE641C3A
:10EBB000E4B2072CEED30025A5E0FAF751F80122C4
:10EBC000002104235F1A0607360F491C08AB000911
:10EBD000C9B2DE550529F4D30020FF21002A06D052
:10EBE0001E5C002E03D1042801D2215402E01E5CD9
:10EBF00000222654401CC0B20528EFD345E0002176
:10EC00000091002902D00121C9074840434901264B
:10EC1000884200DD08464249F9F7FAFD3F2109061E
:10EC2000F9F79DFDFAF71CF800270A21F9F7C0FA59
:10EC30000422D31B7F1C03AAFFB2D154052FF4D3A7
:10EC40000020FF21002E06D0135C002B03D10428E6
:10EC500001D2215402E0135C00262354401CC0B2B0
:10EC60000528EFD301200190009800280DD0002046
:10EC7000215CFF2903D1401CC0B20528F8D300282D
:10EC800003D0102120182038C17700E03BE0012696
:10EC900006A880192038C07F092802D821490F5CB6
:10ECA00009E0102804D2204908182038877D02E0A6
:10ECB00010282CD00027002F13D000240120A040C2
:10ECC00038420AD0A0190721F9F75CFA80190A46E0
:10ECD000401EC1B2104605F033F8641CE4B2072CA4
:10ECE000ECD3761CF6B2052ED2D90298002803D0B8
:10ECF0000521062005F024F80198002803D00621FC
:10ED0000002005F01DF8142005F066F922E74027E1
:10ED1000D1E70000A85A0101A84700209A3F1C46ED
:10ED200000002041E05A0101A05A010102460020E2
:10ED3000802901D98D207047062A06D0072A07D0DE
:10ED4000082AF8D10729F5D170470829F2D1704770
:10ED50000629EFD370477047704770B5C468054601
:10ED60006068002803D00020002802D00CE00120B9
:10ED7000FAE7201DFAF724FC08F4CED560680028D5
:10ED800008D000200028F4D00020E860204608F4D5
:10ED9000C3D570BD0120F5E730B40446A28909202F
:10EDA000521C93B2E48900222546D540ED0707D0D6
:10EDB0005D1C8D4202D130BC104670479B1C9BB23B
:10EDC000521CD2B2092AEFD330BC7047FFB585B0D0
:10EDD0000E9D04462F8801201E4600213A46CA4057
:10EDE000D20704D04B0003225B1C9A401043491CFD
:10EDF000C9B20929F2D3049030461E210840218A65
:10EE0000184A00230191009302920390132304AA4D
:10EE100015490698FAF7DAFB009000281FD1012166
:10EE2000142008F403D60746E06006980188B981EB
:10EE30002988F981F00701D00120C0030799084310
:10EE40003880208A788014206082204600F060F8A4
:10EE5000381DFAF7C1FB208A002108F43DD700983D
:10EE600009B0F0BD545201010A1800000048704773
:10EE7000EC520101FFB5087881B00C46092836D262
:10EE8000142003F06BFC0746217800F0EFF800280F
:10EE90002BD061782078FFF749FF060028D17D68E4
:10EEA000002D0ED020782979814207D12946381DBE
:10EEB000FAF798FB284608F42FD502E02D68002DBC
:10EEC000F1D160780121083008F4B0D505462078EA
:10EED0002871607868716278A11CA81DF9F7C4F9DF
:10EEE0002946381DFAF784FB02E0822600E08126DD
:10EEF00002230648039A049908F41ED6217801706B
:10EF0000467008F455D6002005B0F0BD011400008D
:10EF100010B50446142003F021FC044921600321AC
:10EF20006181123060600120208110BDFC5201011E
:10EF3000F8B517460C46104608F4BCD6012831D166
:10EF4000142003F00BFC0546017C00F08FF8064608
:10EF5000297C22781448914214D1697C6378090293
:10EF60003A46891D9B1D08F4E7D50546068000201A
:10EF70002871607868806278A11C681DF9F774F9BF
:10EF8000284609E0697C062309023A46891D08F4EF
:10EF9000D3D506808021017108F40AD600213846B5
:10EFA00008F49AD60020F8BD140C0000F8B50F46FE
:10EFB000002409781846254609291DD20B007B44F8
:10EFC0001B79DB189F440407101313130A160D0056
:10EFD000052414A510E00A2414A50DE0082416A5A4
:10EFE0000AE0072417A507E00A2418A504E0052471
:10EFF00019A501E006241AA50146A31C1A4808F425
:10F000009BD50646387830707470002C04D02246A8
:10F010002946B01CF9F728F9304608F4C9D5002074
:10F02000F8BD00004E53494E470000004E532D429C
:10F030004C452D312E300000123456FFFE9ABCDEB6
:10F0400000000000025E044000000300312E302E5C
:10F05000302E302D4C450000312E302E3000000077
:10F06000FFEEDDCCBBAA00000314000010B48289BF
:10F07000C489521C93B200222046D040C00706D05B
:10F08000914202D15B1C9BB205E09B1C9BB2521CBF
:10F0900052B2092AF0DB092A02D010BC1846704788
:10F0A00010BC00207047000070B5050005D0134E5D
:10F0B0003068854203D1002070BD72B6FEE704F0CF
:10F0C00043FF6C6904F04CFF7068844202D0B06862
:10F0D000844201D1022070BD0948844204D1A86A4B
:10F0E0000028F7D1032070BD0648844203D0002CCD
:10F0F00001D0012070BD042070BD0000CC4700206D
:10F10000DC6B0020C86B0020002802D00368002BB5
:10F1100001D100207047F8B50D464168044600292A
:10F1200002D0A068884211D21B4EB5420ED8A26808
:10F130006D1C5019814201D39818F8BD216900292E
:10F1400004D11649884203D9B04202D90020F8BD43
:10F150004600226A0027002A05D03146184690470B
:10F16000050012D00CE0A1693046884705000CD09C
:10F17000A2682168521CF9F777F8E169206888478E
:10F1800066602560A0684019F8BDE169206888477D
:10F19000676000202760F8BDFFFFFF7FFFFFFF3F94
:10F1A00070B50D4D04460A2809D10D212846FCF7FB
:10F1B000FBFF80212846FCF787FF0028F9D0E1B249
:10F1C0002846FCF7F1FF80212846FCF77DFF002848
:10F1D000F9D0204670BD000000380140F0B5087835
:10F1E000324F334D334E801E83B00C46062859D221
:10F1F00001007944097949188F4402255434543A5E
:10F2000001203070A0786876A078C00705D02A4920
:10F210002A48FAF7C3F9387AA874B28A002A06D0C5
:10F22000FF20F53070800321254808F447D7F169A5
:10F23000002937D000200090019005206A46107008
:10F24000684688472EE000246C7601F0DBFDF1690A
:10F25000002927D0009406206A4601941070684661
:10F2600088471FE01722A11C1648F8F7FDFF19E098
:10F27000B8780001C0194030807D002812D11C22CE
:10F28000A11C1148F8F7F0FF0F48A18A0182E18A1A
:10F290004182218B8182618BC1820B49608A088304
:10F2A000207F6874002003B0F0BD0000D84D00201E
:10F2B0001C4D0020384D0020E14D00202F4D002036
:10F2C000040F0000164D0020FC4C0020F0B518463D
:10F2D0000D46014685B022230322744808F42CD43D
:10F2E00001210446417028780B286ED20100794430
:10F2F000097949188F4405CDCDCD6F6ABB23CDCD9B
:10F300006C00012020706070694881792171017959
:10F31000A170C17961714179E170017AA171417A7D
:10F32000E171817A2172C16900294ED000200090DC
:10F3300002206A461070684601948847A9E00720B9
:10F3400020700120607068461CF488D1019F009EE7
:10F35000F8F778FF801960820025F8F773FF8119AC
:10F36000601900908170F8F76DFFC11900986D1C4D
:10F37000EDB20175082DF0D30825F8F763FFB91930
:10F38000401861196D1CEDB28870102DF5D3102056
:10F39000207748488178090108184030807D01288D
:10F3A00077D11C22A11C4448F8F75EFF4248A18A8D
:10F3B0000182E18A4182218B8182618BC1823E4937
:10F3C000608A08833D48217F417462E0052000E0A7
:10F3D0000A2020705DE0042222706878012804D0A1
:10F3E000002802D0022833D053E00120304D607055
:10F3F000287C002810D002A81CF430D1F8F722FF96
:10F400002F49F8F7BFFE2F480818029940182E49D7
:10F41000F8F7B8FE009101E0E8680090E96900297A
:10F4200007D00020029003206A46107202A80392BF
:10F4300088471021A01CF8F730FF0098A0700098B2
:10F44000000AE0700098010C2171000E607120E04C
:10F450001748C169002905D0002000900190684636
:10F460000270884720460C3808F498D314E0062030
:10F47000164D2070E878012811D01021A01CF8F753
:10F480000CFFA9886182E988A1822989E182002094
:10F490002076204608F48CD3002005B0F0BD102261
:10F4A0000B49A01CF8F7E0FEEBE70000140E00008B
:10F4B000384D0020D84D0020FC4C00201C4D002071
:10F4C000A0BB0D00A08601003F420F005C4E002053
:10F4D000E74D002000B5084883B0026C002A08D030
:10F4E00000200090029005206B461870684601913C
:10F4F0009047002003B000BDD84D002010B584B067
:10F50000FF2B19D0144C226C002A08D00020009048
:10F51000029006206B4618706846019190470320C0
:10F5200008F4C8D3032814D1A26F002A11D00321F4
:10F530000A4808F4C3D50CE009480123007F0322E0
:10F5400001020848083108F4F7D20721017008F4D5
:10F550002FD3002004B010BDD84D0020090E0000AC
:10F56000384E0020050E0000FFB5180A4C4E83B03F
:10F570000C46B070FF287DD0010234230322494895
:10F58000083108F4D9D20546B0780027010189195D
:10F5900040318872B07821880001801940300181A3
:10F5A000B078617A000180194030C172B078628908
:10F5B0000001811940318A81A289CA81E0890882CB
:10F5C000207C012802D0002807D00BE0B178012070
:10F5D000090189194031887504E0B078000180196B
:10F5E0004030877520883080607A307221460A3139
:10F5F0002D48F9F7D3FF02F0D7F900281BD0607A25
:10F60000012804D103221146284808F4E5D202F06B
:10F61000D3F905280FD201007944097949188F449C
:10F6200006060602060001202821485505E00521AE
:10F630002820415501E0282047550321059808F46A
:10F640004BD317203086B17809018919403148829F
:10F650001748C068002803D00321164808F48ED448
:10F660001548028D002A03D00321144808F426D53A
:10F67000306C00E00EE0002808D0022069460097B8
:10F68000087002950194316C68468847284608F452
:10F690008FD201E001F02EFB002007B0F0BD00008A
:10F6A000D84D0020020E0000E14D0020150D000095
:10F6B000E84E0020030F00005C4E0020020F000007
:10F6C00030B5180A144D00010C46401983B0FF21D3
:10F6D0004030817201F0E2FB002803D102210320B7
:10F6E00008F4FAD22A6C002A08D000200090029078
:10F6F0000320694608706846019490471021074826
:10F70000F8F7CBFD06480068002802D0092008F46D
:10F71000CDD0002003B030BDD84D0020F74D0020E3
:10F72000100C002000B5084883B0C169002907D03B
:10F7300000200090019009206A46107068468847B2
:10F74000002003B000BD0000384D0020FFB591B08F
:10F750000D46122303224348149908F4EDD10021E9
:10F760000446017040480078002862D03E48407C42
:10F77000002833D03C216846F8F78FFD01F006FFE2
:10F78000002841D004A90F913749461EF0B23A2211
:10F790008969504341186846091DF8F765FD6846B8
:10F7A000008B2988884206D10822A91C0F98F8F7F7
:10F7B0009EFD00280BD0207800280BD008A8407CA4
:10F7C000607410226946601CF8F74EFD1CE00120B1
:10F7D0002070F3E73006000ED6D12AE023482988AE
:10F7E000008B884225D10822A91C2148F8F77FFD0B
:10F7F000002809D1012020701E481022407C60742E
:10F800001A49601CF8F730FD2078002811D01648FE
:10F81000C169002907D000200090019007206A46A6
:10F82000107068468847204608F4C2D1002015B001
:10F83000F0BD0D48C169002907D00020009001905B
:10F8400008206A46107068468847022303220A4847
:10F85000149908F471D1012101700621417008F456
:10F86000A7D1E0E7180E0000384D0020FC4C002026
:10F870000C4D00201C4D0020040E000070B50C46FD
:10F8800009781B481B4D1E46002904D0012912D0BF
:10F8900002292BD11AE01C23314608F44DD106462B
:10F8A00020783070287B70802A7B1349301DF8F750
:10F8B000DBFC304607E00A23314608F43DD12178CD
:10F8C00001706989418008F473D10FE00A23314641
:10F8D00008F432D121780170298C4180698C8180B3
:10F8E000A98CC180E98C018108F462D1002070BD2F
:10F8F0000B0E00005C4E0020694E002010B5087809
:10F9000000F03EFF002010BD05480A8842861A0A12
:10F9100012011018098840308182002070470000D1
:10F92000D84D002030B5180AC043000683B00D46FC
:10F93000000E21D0190A0902E1200623032200014A
:10F94000083108F4F9D004460120207002206080BC
:10F95000FF204130A0800B48026C002A08D0002014
:10F96000009004206946087068460195029490470B
:10F97000204608F41DD101E001F0BCF9002003B0DD
:10F9800030BD0000D84D002000B5084883B0026C9F
:10F99000002A08D000200090029008206B461870C2
:10F9A000684601919047002003B000BDD84D00206B
:10F9B00070B518460C46014602230A4808F4BCD02C
:10F9C00005460949A07808736288211D0748F8F7A1
:10F9D0004BFC0020687020782870284608F4E8D096
:10F9E000002070BD0D0E00005C4E0020694E00200E
:10F9F0004A780B48002A05D02030012A08D0022A74
:10FA000009D00AE00279012A07D10978C17004E01F
:10FA10000978017501E00978417500207047000000
:10FA2000D84D002070B54878002806D0FF25124C2C
:10FA300001280BD0022816D01BE0104801790629B6
:10FA400017D10721017101F0C3F812E0207DFF28D2
:10FA50000FD001F0BBF90A4825750169002908D0CB
:10FA60000020884705E0607DFF2802D001F090F972
:10FA70006575002070BD0000F84D0020D84D0020B5
:10FA8000E84E002010B5032B06D010220548891D32
:10FA9000F8F7EAFB002010BD0348017A034801F0A3
:10FAA0002BFEF7E7F74D0020D84D0020E14D002058
:10FAB000F0B50D460878E34EE14934464978002711
:10FAC00020348DB0A1287AD012DCDF490C911B289C
:10FAD00076D006DC012819D003287CD017286DD1F8
:10FAE0004FE128286ED091286DD0A02866D152E130
:10FAF0000246A23A092A61D213007B441B79DB1823
:10FB00009F44FE5CFDFD5CFDFCFDFD006878002867
:10FB100054D1012002F086FE01F02CFE3423032292
:10FB20000721CA4808F408D003210170C8490446D7
:10FB30008A7842700122C276FB224284C54AC2847E
:10FB4000C54A82840A88028487768A888280CA8825
:10FB5000C2800A892281487A8009032805D18878E1
:10FB60000522104201D10120A076A07E042210437C
:10FB7000A076BA486080C878012825D02046102198
:10FB80000A30F8F78AFB316C002907D001206A4659
:10FB9000009710706846019502948847012000F094
:10FBA000EFFD204608F404D0012303220721AC48CE
:10FBB00007F4C2D71A21017007F4FAD733E11EE126
:10FBC000CAE008E069E049E0204610220A300C99BA
:10FBD000F8F74AFBD7E70097019702970397049736
:10FBE000059706970797089709970A970B9701F0CB
:10FBF000DBFE002805D0684601F01CFD0AA801F0D4
:10FC0000E9FC01F0D1FE00280CD06846807900287C
:10FC100008D108A8807B002804D00121684601F0A3
:10FC20004FF900E18A4C6946A0880880E088488046
:10FC3000208988808F71102202A80C99F8F714FB94
:10FC4000E078012804D00697079708970997E4E71A
:10FC5000102206A80C99F8F707FBDEE7E07B0028E6
:10FC600013D11123032207217E4807F465D70546E7
:10FC7000282028707648C078012808D01021681CF8
:10FC8000F8F70BFB284607F493D7E773CBE0102275
:10FC9000681C0C99F8F7E8FAF4E7012002F0C2FDBD
:10FCA0000121032008F418D06F48012444841F2048
:10FCB000049067480178490601D57F210491817835
:10FCC0000522114204D0FF2204998132114304918C
:10FCD0000088C00504D50321049849020843049014
:10FCE000082162480191029003210B2304AA009786
:10FCF0000394C9025E48F9F769FC02E079E04AE042
:10FD000089E0002846D15B4806218786FF200590C0
:10FD1000594801910290082305AA00970394574976
:10FD20005748F9F753FC00287DD100F03BFF00282D
:10FD300079D10221032007F4CFD7B079012808D068
:10FD400001F000F83E484078C0076CD001F042FB5B
:10FD500069E000F0CFFF66E001F026FEE77300F0F7
:10FD600021FF00285FD10221032007F4B5D7B07925
:10FD70000128EED000F0E6FF31484078C007E5D119
:10FD800051E0687800284ED0F179481EF0713D4866
:10FD900001F082FC47E07179491E052906D8A728A1
:10FDA00002D13079002806D100F012FF2878A4286B
:10FDB00001D0A72837D17079042806D0062804D0AE
:10FDC000082808D00C282ED10CE02F480168002903
:10FDD00029D0B07904E01A480169002923D0012014
:10FDE000884720E01648016900291CD00320884775
:10FDF00019E03771FF20F0702075607513E0207DE9
:10FE0000FF2802D06878002802D000F0DFFF0AE067
:10FE1000C8079BD107E0607DFF2802D068780028E2
:10FE200004D000F0B5FF00200DB0F0BDA07D00288B
:10FE3000F9D08807F7D5E17D144801F039FAF2E7E7
:10FE4000E84E0020D84D0020E74D0020040D0000B2
:10FE50005C4E00200502000048080000A08C000055
:10FE6000190D0000230D0000B00B0020D056010139
:10FE7000D20B0020680B0020285701010118000058
:10FE80009C0B0020E14D0020884E0020104E0020E9
:10FE900070B500250C462846401C0628FCDB254E84
:10FEA0002246307E31461A32C96906282AD203001A
:10FEB0007B441B79DB189F4424020910171E06227D
:10FEC000A01CF8F714FA00281BD01BE0237E0920A1
:10FED00001F08EF8002814D114E0237E212001F0D7
:10FEE00087F800280DD10DE0237E162001F080F860
:10FEF000002806D106E0237E192001F079F80028B9
:10FF000000D001250C48807D002811D1716900299D
:10FF100001D020468847002D0AD03169002901D040
:10FF20000220884701F0D8FA217AA01C01F0C0F91C
:10FF3000002070BDE84E0020F84D002010B50A7872
:10FF4000000A000210434A78FF231B021202984362
:10FF50001A4010438A781B02120498431A40104337
:10FF6000C9780002000A09060843F8F774F900206E
:10FF700010BD10B5104607F49DD6002010BD00201E
:10FF8000401C0628FCDB002070470000F8B51C462A
:10FF900017460D46104607F48DD6002811D147208C
:10FFA00002F0DCFB064604233A460321064807F428
:10FFB000C3D5210A01702988B288891A418007F4C3
:10FFC000F7D50020F8BD00000D470000F8B5174632
:10FFD0000C46472002F0C2FB21780646122901D0C8
:10FFE00013291BD1B06805460C351229C288018936
:10FFF00016D006230F4807F49FD5698841806178A1
:020000040101F8
:10000000017107F4D5D5B068002803D007F484D473
:100010000020B0600021384607F45ED60020F8BD0D
:100020000423054807F488D56988018061788170C8
:10003000E7E70000094700000747000000B508484F
:1000400083B0026C002A08D00020009002900920A2
:100050006B461870684601919047002003B000BDC0
:10006000D84D002030B5104D83B0088828861C0A72
:10007000200140190A88403042822A6C0025002A5B
:1000800007D0009507206B460295187068460191CD
:1000900090470648A1004058002801D04030C57460
:1000A000002003B030BD0000D84D0020580B0020C8
:1000B000FFB581B0002000900E46039807F4FAD5F2
:1000C000002802D001284CD04DE0142002F046FB5D
:1000D00007463188FEF760FE05462448092D36D2D2
:1000E0007C68002C1ED02179A94203D02468002C02
:1000F000F9D117E0002C15D06379039A9B1D049960
:1001000007F41AD5054630882880002028716079C8
:1001100068806279A11D681DF8F7A6F8284607F4E3
:1001200047D520E03D740498010A7974384602F0FE
:100130000DFB014601230E48039A07F4FDD4057018
:1001400007F436D50121039807F4C6D50BE0062342
:10015000039A049907F4F0D4318801808021017159
:10016000DDE702200090009805B0F0BD140C0000FF
:1001700002140000FFB585B00E46079807F49AD523
:10018000002802D0022009B0F0BD472002F0E6FAB4
:1001900002900020694608700898070A308803F02A
:1001A000ACF90024694605468C8000281ED10298CF
:1001B0001622016A68460078034650430246103210
:1001C0008A5A5204920F1FD10A5C401C085C1E49D7
:1001D00000021018884217D102AA03A9184603F09A
:1001E0009FF802986946C05D88800224A31D1748C5
:1001F000079A089907F4A0D40746308838803D71E3
:100200007C80002D15D019E03946029802F09EFA44
:10021000014604230E48079A07F48ED407706946F6
:100220000978418007F4C4D40121079807F454D514
:1002300007E0224601A9781DF8F716F8384607F4BA
:10024000B7D4002009B0F0BD02290000140C000052
:1002500004470000FFB58BB00C46472002F07EFA41
:100260000025694605900D740E9804A9070A208898
:1002700003F043F9060061D105981622016A684629
:10028000007C5043024610328A5A5204920F3AD1EF
:100290000A5C401C085C304900021018884232D1C8
:1002A00002950395208800F0DFF802A90023009151
:1002B0001A4608A9F9F7A2F96846008C012109033A
:1002C0000840C043C004C0172146401CFEF79EFAF8
:1002D0000606360E32D168460997007C0190A57952
:1002E00007AA694603F01CF86846028806A8079921
:1002F000F7F7BAFF06A909980A460D54684601881F
:10030000019803F04BF83946059802F01FFAA188CE
:100310000D9A891D8BB20146104807F40DD405468D
:10032000A288A11D801DF7F79FFF2F706846007CF3
:100330006880A088A880284607F43AD40423084897
:100340000D9A0E9907F4F8D321880180867007F47E
:100350002FD400200FB0F0BD022900000A47000092
:10036000160C0000F0B589B00446F9F74DF90546C2
:100370000026154F1BE006A92046F9F715F90023C2
:1003800002AA01A906A80096F9F744F9684600896F
:10039000B84203D169460979022911D00B49884234
:1003A00003D168460079022807D0641CA4B2A8884B
:1003B000A04202D8E888A042DDD2002009B0F0BDFA
:1003C000204609B0F0BD000002290000032800000B
:1003D000F7B5002845D00199002942D08668002A47
:1003E00001D10CE03668002E3BD0316A002938D0AC
:1003F0000198F7F764FF0028F4D12CE03668002E4E
:100400002FD0019C356A002CF8D0002DF6D0AC42DC
:1004100024D02078F7F710FF07462878F7F70CFF6D
:1004200087420DD12078002813D06078641C6D1CA1
:10043000F7F702FF07462878F7F7FEFE8742F1D06C
:100440002078F7F7F9FE04462878F7F7F5FE84429E
:10045000D4D1002E05D0306A002802D0304603B037
:10046000F0BD002003B0F0BDF0B589B00446F9F747
:10047000CBF805460026104F14E006A92046F9F7F0
:1004800093F8002302AA01A906A80096F9F7C2F87A
:1004900068460089B84203D1641CA0B209B0F0BD1F
:1004A000641EA4B2A888A04202D8E888A042E4D280
:1004B000002009B0F0BD00000328000070B5164C04
:1004C0002078002827D101210803FBF733FC002006
:1004D000FBF726FC0120FBF75DFC104D2846F9F7E1
:1004E0004DF903212846F9F7B9F901212846F9F712
:1004F00079F9012121702846F9F79CF9142003F0BD
:100500006BFD702000F00CF8702000F009F800215D
:100510002846F9F78FF970BDA44700200008024073
:1005200070B50546164CFFF7C9FF2946154D2846FC
:10053000F9F7AFF801212846F9F74AF901212846D1
:10054000F9F784F9002807D1641E13D00121284649
:10055000F9F77CF90028F7D001212846F9F796F839
:100560002846F9F770F9044600212846F9F730F9D2
:10057000204670BD00212846F9F72AF9024870BDCF
:10058000A086010000080240FFFF0000F7B5042725
:100590000225494E86B01446082A74D210007844C9
:1005A00000790018874484030D3A3D536370434833
:1005B000019001AB00970799069800F08BF809B0FD
:1005C000F0BD3F4F01213846F9F734F9142003F00C
:1005D00003FD7020FFF7A4FF7020FFF7A1FF044682
:1005E00000213846F9F726F93648B442448001D153
:1005F000354808E02046F9F753F83449F8F708F988
:10060000F8F72EFB00B2694688812A4603AB0095B5
:100610000799069800F05EF809B0F0BDFCF77CFF82
:100620000AE06020FFF77CFFB04201D1002003E028
:100630006021F9F75FF880B26946088102AB224673
:1006400000950799069800F045F809B0F0BD04F050
:10065000F7F97D21C900F7F795FD019001AB22461E
:1006600000970799069800F035F809B0F0BD03F03F
:10067000EFFD019001AB224600970799069800F024
:1006800029F809B0F0BD13E0FDF706F910498842DA
:1006900001D1022000E00120694608740120009089
:1006A00004AB22460799069800F014F809B0F0BD93
:1006B000079809B0F0BD0000FFFF00002200010014
:1006C00000080240A4470020FF7F000000002041F6
:1006D0000040020130B4029C42540546491C88B2D5
:1006E0002C54401C002180B2002C07D95A5C2A549B
:1006F000401C491CC9B280B2A142F7D330BC70473C
:1007000010B5084C82B02078002808D10648009027
:10071000064801906846FDF769FF0120207002B08D
:1007200010BD0000C8470020F13101017D3F0101EB
:10073000F8B50B30C608F600104D19E02068B0423D
:1007400015D3B0420BD96368871B201D0093F7F7C0
:100750008BFDA019009B07604360286004E060687F
:100760002860201DF7F780FD201D2660F8BD251D9F
:100770002C68002CE2D10020F8BD000028480020A1
:1007800010B5A0230949022809D0002203280AD065
:10079000042808D00B704A7000F0A2F810BD0B704E
:1007A00080204870F8E7E0200870F4E7114000204E
:1007B000F8B52A492020486029480121C163294908
:1007C00005228A610021C16327490B20086100F0DE
:1007D00087F82748254A026326494163264B8363ED
:1007E000264CC4632748264D0560274E466027499E
:1007F00081602749C1602749016127494161274933
:10080000816127490163284826494160274FC76015
:10081000274F07610262274A42628362C46205630E
:100820004663254A8263254AC2632648244A0260F9
:10083000184A4260244A8260016324498163244843
:10084000244A41688918244A914206D22349826881
:100850000A63C2684A6300698863F8BD00100140FA
:10086000C027024040250240402702400259F800BC
:1008700040280240025B8500025A8000025D85002C
:10088000025F80508028024002000878020A0800B7
:10089000026EAC500259FC000200C8001270131422
:1008A00002700314026E2800C0280240025D050099
:1008B000125B0500025B8400020A0600026E2C50E7
:1008C00002C3BF00002902401200AC00125D050007
:1008D000104000206F2895FFAF590F00C02602403E
:1008E00030B415481549037D154AFF2B06D1407DCC
:1008F000FF2803D113484078C0070CD01248134B8F
:1009000004789C604078D86111480861114B8B6273
:10091000106030BC7047104B0B6110484861104CA0
:100920008C61104D8D62C8620F48086313600F48D8
:100930005060946030BC7047F84D002000280240A1
:1009400040280240E84E00201140002000270240CD
:10095000127E0200127E0300027E020002C2A0008C
:1009600012C70000027E030012C7800002C2E0002E
:1009700082B01F491D480863FDF7BAFB1DA0FBF7B5
:1009800017FC27A0FBF714FC2EA131A0FBF710FCED
:100990003548016835A0FBF70BFC3BA13FA0FBF7F6
:1009A00007FC47A0FBF704FCFDF7A8F9FCF730FAB9
:1009B000FCF714FBFDF744F801F038F8022000249E
:1009C00002020090234649A10194494803F06CFFBC
:1009D000012002020090002346A10194474803F041
:1009E00063FFF9F755FA03F0D1FBFEE700800081C1
:1009F000007000400A3D3D3D3D3D3D3D3D3D3D3D9E
:100A00003D3D3D3D3D3D3D3D3D3D3D3D3D3D3D3D16
:100A10003D3D3D3D3D3D3D3D3D3D3D3D3D0A0000B3
:100A2000206D636D2D6464632D626C653A20424CC9
:100A300045202B204672656552544F53202B20438E
:100A40004C490A0056312E30302E3334000000005D
:100A5000204669726D776172652076657273696F81
:100A60006E2025730A000000004000202053797397
:100A700074656D436F7265436C6F636B203D202519
:100A80006C7520487A0A000043414949432D4D4383
:100A90004D2D3230323630393032000020424C4554
:100AA00020656E61626C65642C2061647665727489
:100AB0006973696E6720617320222573220A000022
:100AC0003D3D3D3D3D3D3D3D3D3D3D3D3D3D3D3D56
:100AD0003D3D3D3D3D3D3D3D3D3D3D3D3D3D3D3D46
:100AE0003D3D3D3D3D3D3D3D0A000000424C450041
:100AF00031DE0001444953500000000029EB0001A1
:100B000010B50124E4022046FAF7D6FE002805D0ED
:100B10002046FAF7CBFE0D49022008700124240379
:100B20002046FAF7C9FE00280AD02046FAF7BEFE92
:100B3000BFF34F8F07490648C860BFF34F8FFEE7EA
:100B400005484068002800D0804710BD8000002084
:100B50000400FA0500ED00E040400020064800686F
:100B6000002800D08047BFF34F8F05490348C86075
:100B7000BFF34F8FFEE70000404000200400FA055D
:100B800000ED00E0064A11780A2907D28900891889
:100B900048601078401C107001207047002070479A
:100BA000584D002010B5084C084AE1791378002010
:100BB000994207D28800801840688047E079401C3D
:100BC000E071012010BD0000D84D0020584D0020DC
:100BD000F8B5324D0526297928468079304C082908
:100BE0000CD20A007A4412799218974403080D1324
:100BF00013191C2A052801D0FCF778FBF8BD022840
:100C000008D0FCF797FFF8BD607B002802D1E0799F
:100C1000002802D0FDF72CF8F8BDFCF7C7FFF8BD9F
:100C200006202871F8BD0223032207211D4806F47F
:100C300083D7A5210170E9784170072129716E7170
:100C400028E0022303220721174806F475D7074638
:100C5000A7203870E9787970062068710020287123
:100C6000032007F427D0032812D0A879012804D044
:100C7000022802D003280BD104E0207D002801D0F7
:100C8000032003E0A07E002802D00420A87100E029
:100C9000AE71384606F48CD7F8BD0000D84D002060
:100CA000C84E0020A20D0000A30D000010B50028C2
:100CB00004D0014660220C48F7F7D6FA0B490C48DD
:100CC000CA781C2A04D9427B002A01D11C22CA708E
:100CD000C1781F2901D91F21C170017BE22901D9E7
:100CE000E221017310BD0000884E0020A84E0020B4
:100CF000C84E002011490122087907280CD08879B4
:100D0000002809D0012801D0052806D10C48827B93
:100D1000002A03D002200CE08A717047027D002A6D
:100D200001D0032005E0807E002801D0042000E0EF
:100D30000520887110B5FCF7D9FA10BDD84D0020F8
:100D4000C84E002070B5104C0525A079062809D2A0
:100D500001007944097949188F440202040404030C
:100D6000A57170BDA571022303220721074806F46F
:100D7000E3D6A5210170E1784170072121716571E9
:100D800006F416D770BD0000D84D0020A20D00005B
:100D900010B50B4C607DFF2810D0022303220721E1
:100DA000084806F4C9D6A7210170617D4170064A42
:100DB00000215171FF21617506F4FAD610BD0000C3
:100DC000F84D0020A30D0000D84D002010B50A4CAE
:100DD000207DFF280ED0022303220721074806F4B6
:100DE000ABD6A7210170217D4170054A00215171C8
:100DF00006F4DED610BD0000F84D0020A30D000063
:100E0000D84D002010B50848022380780322010243
:100E10000648083106F490D6012101701321417073
:100E200006F4C6D610BD0000D84D0020040E000008
:100E300010B584B0002804D001462A220E48F7F7E6
:100E400013FA0EA00FC86C460FC40B4B0020694666
:100E50001C180A5C247922430A54401CC0B206289C
:100E6000F6D310220A48F7F7FFF90A490A48F8F7BB
:100E700095FB04B010BD00005C4E0020501921907D
:100E80001F04D5624FA489AB90D0CF23000000008F
:100E9000E74D0020604E0020FC0000200020074BA2
:100EA00001460A01D2184032927AFF2A01D0401C32
:100EB000C0B2491CC9B20329F3D37047D84D0020F2
:100EC000F8B507460B46282043430D460322072169
:100ED0000E489B1C06F430D6912101700024064672
:100EE0004570002D0ED9204628214843C119002203
:100EF000CA7180192822801CF7F7B6F9641CE4B285
:100F0000AC42F0D3304606F453D6F8BD910D000044
:100F1000F8B57D262025F600184B194C19490328F1
:100F200012D00A6A01273A430A620A6A9207FCD57C
:100F30000A6AAA430A6201281AD002281AD01E603F
:100F4000F8F76EFB2060F8BD0F480F2782683F025C
:100F50003A438260086A042210430862086A000764
:100F6000FCD5086A284308623D2000011E60E9E7BD
:100F7000064800E006481860E2E700008C00002008
:100F8000900000200010024000100140D10300003A
:100F90005704000010B50446084804238078032253
:100FA00001020748891D06F4C7D506494C80012176
:100FB00001700021418006F4FBD510BDD84D002002
:100FC000010C0000F00B0020084A11780A290AD20F
:100FD000C9004368891800688B6048601078401C1D
:100FE000107001207047002070470000844D0020E1
:100FF000FFB581B01C00064618D01078411CA142F4
:1010000014D8032C12D3401EC5B25078971CB0429E
:1010100006D12A4638460299F7F769F9002808D020
:101020007A19601B801E0406240EE6D1002005B04C
:10103000F0BD012005B0F0BDF0B504466F4E70481C
:1010400083B06D4FB168C1626E490163F16A81621C
:10105000F16B4163B16B816331467C22403138468C
:10106000F7F702F900257D60FD607D626648B86291
:101070007D64BD64FD643D666448B866644838625A
:10108000644865490570032008706448F9140160DC
:101090000904016089140160F06861490746401E37
:1010A0000088604B884200D01F60366E701E00883A
:1010B000884200D05E6001200003009069460195DF
:1010C0000D710820487101278F716846FAF702FCFC
:1010D00084215548F7F7E1F82A215448F7F7DDF85D
:1010E00060215348F7F7D9F852484F4905614561E7
:1010F0008561C561056245628562C562FF264E480D
:10110000CE70067546750020020152184032401C10
:10111000C0B296720328F7D32068086460684864F8
:1011200046486189C187217A4548032901D841771A
:1011300000E0457701212020FAF7FCFD414A4249B1
:10114000042001F09DFA4249404808600A4641499E
:10115000052001F095FA404A4049072001F090FA35
:1011600040493F4808600A463F49082001F088FA94
:101170003E4A3F49092001F083FA3E4805633E4854
:10118000414907703D4805703D4805703D4808607D
:1011900001203E49C00208803D494F2008703D496A
:1011A000082008703C480721067046708670C170A0
:1011B000057145718571C57111483849C16138495A
:1011C000016238494162002002F0B2FC3649032036
:1011D00006F4C6D50021032006F47ED5002001F0D8
:1011E00021FB012303220721304806F4A5D4077010
:1011F00006F4DED403B0F0BDC00900200080000179
:10120000C00000205D0B01010D470020493C010199
:10121000010B0101C6000020D800002000E100E021
:10122000FEE7000040400020D84D00205C4E00202A
:10123000884E0020D84E0020F84D0020184E002087
:10124000384E002080400020808001009D53010125
:10125000C0400020C08001000041002000DB0100F0
:10126000814100204041002040DB0100C0460020B9
:10127000C06102000070004060000020C900002032
:10128000610000200090D0036C0000206800002066
:10129000630000206400002008010020C526010131
:1012A000ED2701018D27010130580101020D0000D9
:1012B000F8B5404D0646687D3F4C0F46FF281CD0D0
:1012C0002046C268002A03D003213C4806F4F6D623
:1012D0003A23032207213A4806F42ED4A4210170B0
:1012E000697D0446417037480022017800291ED0EC
:1012F0000121A170A28002701BE06D200223032255
:101300000721400106F418D4A22101702E49C978A2
:10131000417006F44DD4EF7531462C48F8F73EF98C
:101320000120A8756078022108436070F8BDA270A2
:10133000A2800120E07019214901E1802248218129
:10134000038CE381438C2382838C6382C38CA382CE
:10135000FF23E2824133184D23836D786D070DD54D
:101360000525E5706181A181018CE184418C218595
:10137000818C6185C08CA085E28523863820075545
:10138000204631463230F8F709F9E078810703D575
:101390000220FFF7F5F906E0400701D5032000E041
:1013A0000120FFF7EDF90A490C204871204606F4A8
:1013B000FFD3F8BDF84D0020E84E0020030F0000D9
:1013C000A10D0000584E00205C4E0020104E002061
:1013D000D84D0020F8B52C4E2C4D317D0127687872
:1013E000FF2941D0C1073ED0B8436870284900208A
:1013F00008703A2303220721264806F49DD30446A9
:10140000A4202070307D60702878A07068788006F5
:10141000800F20716888E080A8882081E888E081BA
:1014200028892082E7700120FFF7AAF96878400731
:101430000AD5E07802210843E07068886081A888B6
:10144000A0810320FFF79CF96878000703D5E078B6
:101450000C210843E0701049082048710020B07545
:10146000204606F4A5D3F8BD384368706D200223EA
:1014700003220721400106F45FD3A121017007492F
:10148000C9784170EDE70000F84D0020E84E0020DB
:10149000584E0020A10D0000D84D00205C4E0020C9
:1014A00010B50A4C607DFF280ED0022303220721CD
:1014B000074806F441D3A5210170617D4170054ABA
:1014C0000D21517106F474D310BD0000F84D0020B9
:1014D000A20D0000D84D002070B50B4C207DFF28D8
:1014E00011D00A4D687909280DD002230322072163
:1014F000074806F421D3A5210170217D41700921FF
:10150000697106F455D370BDF84D0020D84D002008
:10151000A20D000010B504464088A1880246491C6F
:1015200019234A43DB019A420FDC06280DD3228897
:1015300090420AD3E2887D23DB009A4205D84B0013
:10154000C9184843D100884201DD002010BD0D4874
:101550000E238078032201020B48083106F4ECD2F6
:10156000092101702188418061888180A188C18022
:10157000E188018100214181491E818106F418D34F
:10158000012010BDD84D00200E0E000010B5084AF5
:10159000084B906901888478994206D1917CA142D8
:1015A00004D20024FAF770FB00E00024204610BDAE
:1015B000384D0020341200000B4610B504493A2281
:1015C0008969504341181846091DF6F74DFE10BDB4
:1015D000384D002010B590B004463C216846F6F71F
:1015E0005CFEFFF7D3FF401EC0B26946FFF7E4FF81
:1015F00008A8807CA0710CA920460331F7F7CEFF24
:1016000010B010BD10B590B004463C216846F6F706
:1016100044FEFFF7BBFF401EC0B26946FFF7CCFF98
:1016200008A8007CA0710AA920460231F7F7B6FF8E
:1016300010B010BD10B590B004463C216846F6F7D6
:101640002CFEFFF7A3FF401EC0B26946FFF7B4FFB0
:101650000AA920460231F7F7A1FF08A8007CA07173
:10166000204606A9102208300231F6F7FDFD084891
:10167000C17820461830012904D01021F6F70DFE5C
:1016800010B010BD10220349F6F7EEFD10B010BDEA
:101690005C4E0020E74D002070B590B00D46064628
:1016A000FFF774FF002D23D0854221D81823032291
:1016B0000721104806F440D204461720207001206C
:1016C00060703146A01CF7F769FF3C216846F6F7C9
:1016D000E4FD6D1EE8B26946FFF76EFF204606A9DD
:1016E000102208300231F6F7BFFD204606F460D222
:1016F00010B070BD140D0000F3B58FB00C463C2146
:101700006846F6F7CAFDFFF741FF012C1AD0002802
:1017100016D0154D0AAE0236441EE0B23A22A9692F
:10172000504341186846091DF6F79EFD06223146D2
:101730000F98F6F7DCFD00280DD02006000EEBD147
:1017400011B0F0BD0949421ECA7101460F98FFF75A
:10175000A3FF11B0F0BD06A9102205480231F6F72B
:1017600083FD11B0F0BD0000384D0020D84D0020A1
:10177000F74D002070B5284C82B020688003FCD55E
:10178000264D687FFFF7C4FB606A606A012630431C
:101790006062606AB04360622148C08F0A2811D934
:1017A000E16932071143E1611E494A6832434A60E8
:1017B0001E491D4A0A6003224A6088601C4808606E
:1017C0001C480860684619F449D71B49009808600E
:1017D000687FFF252D02032811D000F027F9206B28
:1017E000A8432063206B3F21490208432063206BFC
:1017F0003043206301220321104806F45FD41048CF
:101800000168A94301600F490868FF221204904350
:10181000086002B070BD000000100240384E002089
:10182000184E002040100240555500000030004086
:10183000AAAA0000CCCC000048400020010F000004
:1018400000E400E008E400E0F0B5D7B054A819F4D3
:1018500005D74A490024886AC96A54990122411A65
:1018600009010909D206914204D95499081A0001C4
:1018700000094142424E40290CDC7088002809D002
:10188000401E7080142203213E4806F417D4002025
:1018900057B0F0BD3C48FF21569029316846F6F715
:1018A000FCFC707CB569002832D0FFF76FFE6946FA
:1018B0008870B17C6F4688420BD23A214843024679
:1018C000291D381DF6F7D0FC69468878401C8870C1
:1018D00008E03A21401E4843024629463E31381D61
:1018E000F6F7C2FC694688783A214843C0190A468F
:1018F00036385699F6F7B8FC244869460880B0692E
:10190000FAF7C2F9FF2227326946B069FAF7EAF915
:10191000FF20F53070804A944B944C944D944E9433
:101920004F9450945194529417485394418D40AA27
:101930001185818D5185C08D9085154C48AA257CD7
:101940009573102213494CA8F6F78EFC1248C07804
:10195000012804D11022114950A8F6F785FC012670
:101960000F48002DC67306D1A07C002803D00121AA
:101970004AA8FFF7A5FA0B48067088E7C080024026
:10198000384D0020040F0000FC4C002034120000F1
:101990001C4D0020164D00205C4E0020E74D00201D
:1019A000F84D0020584E002002480078002800D052
:1019B00001207047384D0020014800797047000031
:1019C000384D002070B517493CC80E4684B04036EB
:1019D0003CC64368026880684B65134C0A6588659D
:1019E000607C002818D0002569460D72FAF75EF970
:1019F000FFF7CCFD69460872E1690126002906D08F
:101A000068460095067002A80190684688476846B7
:101A1000007A002802D0267004B070BD257004B092
:101A200070BD0000FC4C0020384D002004490868BF
:101A3000401C0860012801D0012070470020704739
:101A40002440002003490868002802D0401E086096
:101A50000120704724400020F8B50C462849294B46
:101A60004118294F294A0026069D002908D001293E
:101A700022D0274940180A282FD301202870F8BD0A
:101A800020780A2838D2214980000958214A9142F9
:101A900003D11E490E501E502EE0B9422CD1032214
:101AA000082311461C4806F447D02178017061686C
:101AB000416006F47DD01FE020780A281CD2800007
:101AC0001158B94218D11958115020781349626839
:101AD0004018032106F4F2D20EE0C0B20A280BD25D
:101AE00084001159002907D0B94205D0094FB942E5
:101AF00002D016511E5188472E700020F8BD0000FC
:101B0000FBF0FFFFD44C0020F33D0101AC4C002062
:101B1000F9F0FFFFF13D0101060F0000070F000083
:101B2000102909D810B50C460A4601460348F6F7B5
:101B30009BFB0348848110BD704700008A6A002027
:101B400068470020F7B55C4F82B0387814460D46E0
:101B5000002809D0042C0FD2012211213B6A0298DF
:101B600000F098F905B0F0BD00230222112102987F
:101B700000F090F905B0F0BD084600F079F9241F97
:101B800000943B6A2D1D98420ED03879002802D06F
:101B900078790028EED102221121029800F07AF91A
:101BA0000120787105B0F0BD78691E19864206D90A
:101BB00003221121029800F06DF905B0F0BD3E62DC
:101BC000B86AB0420FD2B96A38694018FAF75CF8BF
:101BD000002801D0052207E00120B96A0003081897
:101BE000B862B042EFD30022002A3CD1386B002803
:101BF00022D03249042808D2002C1BD02B780B5459
:101C0000401C641E6D1C3863F4E73E46042811D165
:101C1000716A3069294B401804221946FAF762F8B4
:101C2000002801D0052203E0706A001D00227062C6
:101C300000203063002A16D1042C1DD37A6A38693B
:101C4000A608B600801829463246FAF74BF8002855
:101C500001D0052203E0786A801900227862AD196C
:101C6000A41B002A08D011213B6A029800F012F947
:101C7000FBF746FD05B0F0BD002C05D022462946F5
:101C80000E48F6F7F1FA3C630020787138793B6A28
:101C900000280AD00098190B181A000B000309033A
:101CA000884202D178698342E4D10022112102984E
:101CB00000F0F0F805B0F0BD684700209447002020
:101CC000F7B5664C8CB02378002B11D0042A07D0CE
:101CD00001221221236A0C9800F0DCF80FB0F0BD4D
:101CE000084600F0C5F80646236A6069834206D0BC
:101CF000022212210C9800F0CDF80FB0F0BD206B3D
:101D00000025002815D0042806D25549FF220A5480
:101D1000401C20630428FAD3636A206950490422D6
:101D2000C018F9F7DFFF00287ED1606A2563001D27
:101D3000606261692069FCF74FFDB04202D1A16980
:101D4000884209D004221221236A0C9800F0A2F8DC
:101D5000FBF7D6FC0FB0F0BD2069001D00F088F83D
:101D600021690A460832904203D362698918814288
:101D700009D806221221236A0C9800F08BF8FBF791
:101D8000BFFC0FB0F0BD374E6F460FCE0FC70FCE62
:101D90000FC7B268716830680A920890324F009895
:101DA000203E0991B84206D128213046FCF714FDA7
:101DB0000A9988420AD000950195029503950495E9
:101DC000059506950795089509950A950097274A60
:101DD0002169914201D1012000E00220019091424D
:101DE000684601D1083000E0183001606169416047
:101DF000A1698160E169C16028216846FCF7ECFCBB
:101E00000A903046F9F740FF00280FD12C2269468E
:101E10003046F9F767FF002808D12C223146684682
:101E2000F6F765FA002800E000E009D0052212214B
:101E3000236A0C9800F02EF8FBF762FC0FB0F0BD9F
:101E4000A5700022122163690C9800F023F802F0BB
:101E5000F7FD60630120E0700FB0F0BD684700201F
:101E6000944700200040000111C011CA0080000109
:101E70000378C2781946437812061B021943837807
:101E8000C0781B04194311430902090A00060843DC
:101E90007047000070B586B06C4621746274A374FC
:101EA000190AE174190C2175190E61751E498C6BA4
:101EB000002C30D0CA216A4611701F2151709070D9
:101EC0000620D0700020107104A9501DF7F766FBA2
:101ED00016480923164D00AA01321178090248401C
:101EE0000021521C060402D54000684000E040007A
:101EF000491CC9B280B20829F4D319465B1E9BB2B3
:101F00000029EAD16946C872000A08730D216846A3
:101F1000A04706B070BD0146062304AA1F20FBF7A8
:101F200053F906B070BD000068470020FFFF0000B5
:101F30002110000070B50C460546FCF743FA214617
:101F40002846FCF761FAFCF74DFA02490120887037
:101F500070BD00006847002070B5FEF7D1FBFCF7AC
:101F600009FB04002FD01A4D2889F6F75DFE0246C2
:101F70000B4618A12046FCF7B1FAE868F6F754FEC4
:101F800002460B4614A12046FCF7A8FA1348007835
:101F9000F6F74AFE02460B4611A12046FCF79EFAD0
:101FA0002046FCF7F7FB05462046FCF7EFFA002D2C
:101FB00009D02846FCF74EFD0BA0FCF74BFD284648
:101FC000FCF7F0FB70BD09A0FCF744FD70BD0000FC
:101FD000CC6A00206C65640070776D00B04700200B
:101FE00076616C69640000000D0A00006A736F6E10
:101FF0003A20616C6C6F63206661696C0D0A0000A9
:1020000070B5134C01256078002802D1F9F74EFE17
:10201000657010483021FCF7DFFB0E490E4E086357
:102020003046F9F731FE00280DD1342209493046F7
:10203000F9F758FE002806D1342231460548F6F754
:1020400056F9002801D0012070BD2570002070BD18
:10205000B0470020CC6A002000600001F3B583B0D7
:102060000498002106688068009137187D1C305C58
:102070002C4622287ED10498406807E05C2A04D1CF
:102080005B1C834277D2491C641C641CA31B8342E3
:1020900002D22278222AF1D1A21B82426BD220786E
:1020A000222868D1E01B401A0499401C096988471E
:1020B000009000285ED0A54270D229785C2903D018
:1020C0000170401C6D1CD8E00223611B012952DB0A
:1020D0006A78662A15D008DC222A22D02F2A20D03E
:1020E0005C2A1ED0622A46D108E06E2A0DD0722AE0
:1020F0000FD0742A11D0752A3DD115E00821017046
:1021000010E00C210170401CB6E00A210170401C57
:10211000B2E00D210170401CAEE009210170401CAD
:10212000AAE00270401CA7E00022944606296FDB5B
:10213000AF1C1346F95C0E46303E092E02D8303AE9
:102140008A180BE00E46413E052E01D8373A04E0CE
:102150000E46613E052E1FD8573A8A18032B00D22F
:1021600012015B1C042BE5D337218902531A554910
:102170008B4201E09CE094E07BD91B23DB02D31A65
:102180008B423FD80C23A91D9E46631A062B70DB99
:102190000B785C2B6DD102E00022E5E770E04B7814
:1021A000752B66D1891C019100210E46019B9B5D18
:1021B0001F46303F092F02D8303959180BE01F460F
:1021C000413F052F01D8373904E01F46613F052FF5
:1021D00016D857395918032E00D20901761C042E3F
:1021E000E4D337239B02CE1A01239B029E4240D2A6
:1021F00092058905120B890D0A439901521803E0D3
:102200000021EEE706218E46802A02D2012315E046
:102210002FE00121C9028A4203D20223C0218C4649
:102220000CE0012109048A4202D20323E02104E0E8
:1022300025498A421DD80423F0218C46591E0906DF
:10224000090E0AD0164680273E43BF273E4046541B
:10225000491E92090906090EF4D1012B03D96146E2
:102260000A43027002E05106490E0170C01873461D
:1022700000E00023002B14D0ED18A54200D21CE78B
:102280000021017003981021C16003990098086132
:10229000049804990068201A401C8860012005B049
:1022A000F0BD0098002803D0049841690098884741
:1022B000002D04D004980068291A04988160002039
:1022C00005B0F0BDFF030000FFFF1000F0B591B0B6
:1022D0000C0006467ED0216800297BD0A068636888
:1022E000021D9A4206D808180422DBA1F6F715F859
:1022F000002833D0A0686268411D914207D8216848
:1023000005220818D6A1F6F708F800282ED0A068F4
:102310006268011D914207D8216804220818D2A1E1
:10232000F5F7FBFF002829D06268A168914203D22B
:102330002068405C22282BD091427AD22068405CF1
:102340002D2802D03038092873D80020014610907B
:1023500020682E22002807D06B464DE00420F06054
:10236000A068001DA060012011B0F0BD0120F06048
:10237000A068401DA060012011B0F0BD0220F060F7
:1023800001207061A068001DA060012011B0F0BDA7
:1023900021463046FFF762FE11B0F0BD25682818CF
:1023A000085C342820D00DDC05462B3D092D28D2B1
:1023B0002F007F443F79FF19BF44162316182316B8
:1023C0001616160038280FD008DC35280CD0362811
:1023D0000AD000E074E0372813D105E0392803D093
:1023E000452801D065280CD1585400E05A54491CA6
:1023F0003F2906D2002C04D0A06867684518BD426A
:10240000CCD30020585410A9184601F0E3FC0F4625
:10241000054610996846884252D0F761944A954B18
:1024200028463946B561F6F7A1FC03D89248706199
:102430000FE019E00022914B28463946F6F782FC5E
:1024400002D80120C00703E028463946F6F722FCEF
:1024500070610820F060109AA1686846101A081888
:10246000A060012011B0F0BD7D20C000914203D2D8
:1024700023685B5C5B2B06D0914279D22268515C69
:102480007B2967D074E00027E1683D4681426FD226
:10249000491CE1602168A068095C5B2968D1401C87
:1024A000A0602046FBF7FCFF6168A068884203D269
:1024B0002268125C5D2A38D0884202D3401EA06098
:1024C00056E0401EA060204610300090FCF7C8F88F
:1024D000002839D0002F23D0286045600546A06829
:1024E000401CA0602046FBF7DBFF21462846FFF793
:1024F000EDFE00282AD02046FBF7D2FF002C25D085
:102500006168A068884203D22168095C2C290AD03E
:10251000626890421AD22168085C5D2816D104E0F6
:1025200007463D46DBE70098D0E7E068401EE060E4
:10253000002F00D07D602020B760F060A068401CB4
:10254000A060012011B0F0BD002F11D03846FCF77B
:102550001DF80DE00027E1683D46814208D2491C84
:10256000E1606168A068884202D2115C7B2902D0D8
:10257000002011B0F0BD401CA0602046FBF790FF8A
:102580006168A068884203D22268125C7D2A4CD020
:10259000884293D2401EA060204610300090FCF785
:1025A0005FF8002855D0002F4ED0286045600546C2
:1025B000002CCBD0A0686168401C8842C6D2A060C5
:1025C0002046FBF76DFF21462846FFF747FD002810
:1025D000BCD02046FBF764FF2869286200202861F0
:1025E0006168A0688842B1D22168095C3A29ADD1FE
:1025F000401CA0602046FBF753FF21462846FFF70A
:1026000065FE0028A2D02046FBF74AFF6168A0685B
:10261000884203D22168095C2C2918D06268904254
:1026200094D22168085C7D2890D1E068401EE0606B
:10263000002F00D07D604020B760F060A068401C93
:10264000A060012011B0F0BD07463D46B0E70098FC
:10265000A5E7002F8CD079E76E756C6C0000000048
:1026600066616C736500000074727565000000009F
:102670000000C0FFFFFFDF41FFFFFF7F0000E0C160
:10268000102819D230B40D4C83001B199D698903A1
:102690002D0B2D03090D0D439D619969084D92097C
:1026A00092052940920A1143996101226169824091
:1026B0001143616130BC7047704700000020024048
:1026C000FF0FC0FFF3B5054681B00026408800F03B
:1026D00003F901000AD01C4F6A88002014234343E9
:1026E000DB195B8A934203D142262AE0402628E088
:1026F000401CC0B20A28F1D3002E22D1002414209D
:102700006043C019408AFF2806D0641CE4B20A2C3A
:10271000F5D30A2C14D014E0284608300090142079
:102720006043C0190E686B78AA880746A91DB04798
:102730000600EED1688878820298398A0180E8E73D
:102740004B26304603B0F0BD904B00200288500469
:10275000400CD20B01D009020843704710B400248A
:10276000094A214614234B439B185B8A834204D1B8
:10277000142041438818C46803E0491CC9B20A29DF
:10278000F0D3204610BC7047904B002030B4FF239C
:10279000040AC5B20A490020142242435218128A80
:1027A000AA4204D1142250434018438A03E0401C3B
:1027B000C0B20A28F0D3200230BC18437047000092
:1027C000904B0020084A11780A290AD2C9004368B0
:1027D000891800688B6048601078401C10700120D8
:1027E0007047002070470000584C002030B4FF2391
:1027F000040AC5B20A490020142242435218528AE0
:10280000AA4204D1142250434018038A03E0401C1A
:10281000C0B20A28F0D3200230BC18437047000031
:10282000904B0020F1B582B00299294E002000297A
:1028300000D1307000250298002804D0012834D03F
:1028400002283ED10FE0294614225143214A28464E
:1028500009308C182082C0B205F49CD2207C21461D
:1028600005F47ED22DE0284614214843194900235F
:102870004718B87C009030781C4600280DD9E0003D
:102880008019828800998A4202D180688047034675
:10289000641C3078E4B2A042F1D8002B02D0596811
:1028A00038468847387C05F499D21422094B6A438C
:1028B0000021D018FF24C1604482995041600181F9
:1028C00041816D1CEDB20A2DB5D303B0F0BD0000FF
:1028D000584C0020904B002070B50146094DCEB2F7
:1028E00000202978044600290BD9E10049198A887B
:1028F000B24201D188688047641C2978E4B2A142C1
:10290000F3D870BD584C0020F7B500248AB000946D
:102910000194029403940E4604940594069407943B
:102920000894FF27013711681546384688470596F1
:1029300001970090AA686968286806900098089234
:10294000079100283CD069460A9800F0CDF800288D
:1029500030D00098002806D002994018F5F7A8FC5E
:10296000029940180290AA68002A07D0029900989C
:10297000491C904706001DD0009418E00298296871
:10298000401C8847060015D002980199401C8142DE
:1029900001D20A4601E0029A521C30460099F5F72E
:1029A00063FC029834546968009888470094304664
:1029B0000DB0F0BD0098002802D0696888470094E7
:1029C00000200DB0F0BD0000F8B500240A46054611
:1029D000002910D0002D10D001460078002826D004
:1029E00008780C283BD015DC082838D0092836D0C8
:1029F0000A2815D133E00020F8BD03211046FCF76A
:102A000083FB0028F8D022210170417000218170E1
:102A10000120F8BD0D2822D0222820D05C281ED00D
:102A2000202800D2641D4878491C0028D8D1481BB2
:102A30000719F91C1046FCF767FB061EE9D0002CAD
:102A40000FD0222030702878741C002834D0C0B2F7
:102A50001F2813D9222811D05C2837D10EE0641C1E
:102A6000E1E7222434703A462946701CF5F7FCFB56
:102A7000F0194470002181700120F8BD5C202070A5
:102A80002A78641C0C2A23D006DC082A1DD0092AC7
:102A900024D00A2A06D11DE00D2A1DD0222A12D0E8
:102AA0005C2A13D00EA12046F9F792FB241D68780A
:102AB000641C6D1C0028CAD12221F019417000212C
:102AC00081700120F8BD222000E062202070EEE736
:102AD0006620FBE76E20F9E77220F7E77420F5E740
:102AE0007525303478000000002801D0002901D17C
:102AF00000207047F0B50546007B8BB00C461028CF
:102B00007ED008DC012819D0022821D0042809D061
:102B1000082876D128E0202874D0402873D0802857
:102B20007DD19BE005212046FCF7EEFA002803D07A
:102B3000DCA1F6F77BFD01200BB0F0BD062120469D
:102B4000FCF7E2FA0028F7D0D8A1F6F727FD08E055
:102B500005212046FCF7D8FA0028EDD0D5A1F6F7DC
:102B600065FD01200BB0F0BD07910024AF69EE694F
:102B700000942E20019403940494059402940694E6
:102B80000894314609940A90002F01D0012000E0FA
:102B9000002001434800C9494008081AC00F14D159
:102BA000012170004905C84201D1002F0DD068698C
:102BB000F6F726F83A463346F6F7C4F80BD1C0A12B
:102BC00068466A69F9F704FB26E0BEA16846F9F792
:102BD000FFFA054621E03A463346BCA16846F9F7BC
:102BE000F7FA054608AABBA16846F5F7A5FB012838
:102BF0000CD13A46334609990898FBF73DFF03E0AC
:102C00003EE00CE041E094E0002806D13A4633462D
:102C1000B1A16846F9F7DCFA05461A2D02D3002067
:102C20000BB0F0BD691C0798FCF76EFA0028F7D0CE
:102C3000002D0BD92E236A46115D0A9EB14201D1A7
:102C4000035500E00155641CAC42F5D30021015549
:102C50000798806841190798816082E728690028F1
:102C6000DED0F5F725FB401C064601462046FCF762
:102C70004BFA0028D4D032462969F5F7F5FA70E707
:102C80002869FFF7A1FE0BB0F0BDAD680121204619
:102C9000FCF73AFA0028F6D05B210170A068401CCE
:102CA000A060E068401CE060002D34D00026214682
:102CB0002846FFF719FF002813D0002C09D0206800
:102CC000002806D0A1684018F5F7F2FAA16841186B
:102CD000A160286800281BD06069002804D0022762
:102CE00003E030460BB0F0BD0127791C2046FCF70D
:102CF0000BFA0028F5D02C2101706169401C0029D5
:102D000002D020210170401C0670A068C019A0608C
:102D10002D68002DCBD102212046FCF7F5F90028C3
:102D2000E0D05D21017000214170E068401EE0604C
:102D300017E76069AD68002801D0022700E001278D
:102D4000791C2046FCF7E0F90028CBD07B210170EC
:102D5000E168401C491CE16062690A21002A00D038
:102D60000170A068C019A060002D78D000276069AC
:102D7000002814D02046E168FCF7C6F9002825D0C9
:102D8000E2680021002A06D909220270E368401C8B
:102D9000491C8B42F9D8E168A0684018A060214620
:102DA000286AFFF711FE002810D0002C09D02068F7
:102DB000002806D0A1684018F5F77AFAA1684118F2
:102DC000A1606069002804D0022603E038460BB0F9
:102DD000F0BD012631462046FCF796F90028F5D0D3
:102DE0003A2101706169401C002901D0092101705C
:102DF000A06821468019A0602846FFF775FE0028CC
:102E0000E4D0002C09D02068002806D0A168401822
:102E1000F5F74EFAA1684118A1606069002800D05A
:102E200001202968002900D001214618711C204684
:102E3000FCF76AF90028C9D02968002902D02C21A2
:102E40000170401C6169002902D00A210170401CF8
:102E50000770A0688019A0602D68002D87D1606977
:102E6000002802D0E168491C00E002212046FCF75E
:102E70004BF90028ABD0616900290BD0E268002132
:102E8000012A07D009220270E368401C491C5B1E1E
:102E90008B42F8D87D21017000214170E068401E0E
:102EA000E0605EE66E756C6C0000000066616C733D
:102EB0006500000074727565000000000000F07F7E
:102EC000256400006E756C6C0000000025312E3109
:102ED00035670000256C670025312E31376700000B
:102EE00070B505460078002813D00A4E2846F5F73D
:102EF000DFF984B20D2C00D90D2471782346481CCB
:102F000070702A460220FAF75FF92D1928780028F8
:102F1000ECD170BD5A470020F8B5069E1F46182E0A
:102F200001D9182500E0354613460A4601460CA093
:102F30000096F9F73DF90024002D07D9395D11A05D
:102F4000F9F736F9641CA4B2AC42F7D3AE4202D909
:102F50000EA0F9F72DF90FA0F9F72AF9F8BD000036
:102F60005B424C452025735D20747970653D307857
:102F700025303258207365713D2575206C656E3D96
:102F8000257500002025303258000000202E2E2EFE
:102F9000000000000D0A0000F8B5134E0F467569D9
:102FA00004463068001D00F025FF601C07D1002F8B
:102FB00005D031680D48091D00F0B9FFF8BD306833
:102FC0002C1944603168AC4204D2B068091D00F08D
:102FD00095FFF8BD7068091D00F090FF306B8442CA
:102FE000F7D23463F8BD0000CC470020DC6B002032
:102FF000124D134E134FE868002817D000F0A4FFBD
:10300000F068C468201D00F0F5FE2869401E2861A4
:10301000E868401EE86000F0A3FF206B00F0AEFF00
:10302000204600F0ABFFE8680028E7D138680128A7
:1030300001D900F0C5FF00F043FFDCE7CC470020DA
:10304000C86B0020006B002030B4124900E011462C
:103050000A688242FBD34B685C18844203D1406803
:1030600018184860084643681C1894420CD10A4C52
:103070002468A24206D052689A1842600A68126810
:10308000026002E0046000E00260814200D008605B
:1030900030BC70471848002008480020F7B582B0BF
:1030A000039800260068002859D00398416802461A
:1030B0004968083241600092914201D149684160FB
:1030C0004068C06801900398416849684160009A6F
:1030D000914201D149684160CF6824200299704330
:1030E000441804983D46002F01D11E490D68256003
:1030F000294634316160E96A2161296BE161696CBB
:10310000A1600023E96CA3616161052813D0154912
:103110000A68954201D1237311E0207303280ED170
:10312000886B401C8863A86A002801D002202073A5
:1031300001F098FD03E02846FBF7B6FF2073286BEB
:1031400000210278A52A04D14278401C491CA52AF6
:10315000FAD0880820840198761C8742B3D1304683
:1031600005B0F0BDCC47002003480068401C72B693
:1031700000D0FEE7FEE7000020480020F8B5054635
:1031800000F0E2FE2E46403605243457002C0FDDB9
:103190002F462437686A00280AD0384601F030FDEF
:1031A000002801D000F0A0FF641E64B2002CF1DC06
:1031B0000027FF43777100F0D3FE00F0C5FE042422
:1031C0003457002C10DD2846103000902869002864
:1031D0000AD0009801F014FD002801D000F084FF0F
:1031E000641E64B2002CF1DC377100F0B9FEF8BD4A
:1031F000F8B50446002500F0F1FF374E002730688F
:10320000364A002801D0F0681BE009213448C90281
:10321000430705D0C01DC008314BC000C31AC91AEE
:1032200041180839C908C9005760106031604F6003
:103230000B1A0F6043600160B3600120C007736028
:10324000F06004423FD1002C3DD0204608304107B9
:1032500008D04107490F0823591A0818410701D01F
:1032600072B6FEE700282ED0716888422BD81B4921
:10327000146801E0214614466268824202D2226844
:10328000002AF7D1326894421DD00D6822680A6086
:10329000616808350A1A102A09D921184B0701D08C
:1032A00072B6FEE74A6060600846FFF7CDFE6168CF
:1032B0007068401A7060B268904200D2B060F068E6
:1032C00027600143616001F0CDFC680701D072B650
:1032D000FEE72846F8BD00000848002018480020F6
:1032E000F06B002004490868002803D00868026DCC
:1032F000521C026508687047CC47002010B40124B6
:10330000031F24061C601B1F1960191F034B0B6051
:1033100014390A6010BC403870470000693101015F
:1033200070B5064614460D464720FFF717FA0369A5
:10333000002B0DD01879B04207D158792880981DFC
:103340002060002B04D0002070BD1B68002BF1D141
:103350000020288020600A2070BD000070B516464D
:103360000C46104604F4A6D4002813D14720FFF7DA
:10337000F5F90546062332461946074804F4DCD31E
:10338000A988628889180180A1884180A17901718A
:1033900004F40ED4002070BD180C0000F7B50646EA
:1033A0000D464720FFF7DAF904690746002C14D0D0
:1033B0002079B0420BD16079A8420CD03846214622
:1033C0001030F6F70FF9204604F4A6D205E0246881
:1033D000002CEDD101E0002C0AD128460121083053
:1033E00004F424D30446014638461030F6F700F9B9
:1033F000267165712A46A01D0299F4F735FF002059
:1034000003B0F0BDF8B5C5680124287F0F46012838
:103410001ADD0E4E2046162250430246296A10320B
:103420008A5A5204920F0BD10A5C401C085C0002BD
:103430001018B04204D1E1B20022384600F03EF943
:10344000287F641CA042E5DCF8BD000002290000D2
:10345000F8B5C5680124287F0F4601281ADD0E4EF5
:103460002046162250430246296A10328A5A5204D4
:10347000920F0BD10A5C401C085C00021018B0428D
:1034800004D1E1B20022384600F018F9287F641C0C
:10349000A042E5DCF8BD00000229000070B5C46858
:1034A00005462069002803D00020002802D00EE045
:1034B0000120FAE7264610363046F6F781F804F484
:1034C0002BD22069002808D000210029F4D0002048
:1034D000E860204604F420D270BD0121F5E710B564
:1034E00004464720FFF73AF982790021A24202D927
:1034F0008088001981B2084610BD70B504460D469B
:103500004720FFF72BF9014680888022A04206D889
:1035100089794118A14202D9201A28700022104648
:1035200070BDFFB585B00E9D064629780120884004
:10353000401E049018460E210840328A69681F46D2
:103540004030019200230390009302912B7804AA4B
:10355000A9680698F6F770F8009000282AD1012192
:10356000282004F463D20446AA6869682868626265
:103570002162E061F46006980188A180217FA17139
:10358000F80701D00120C003079908432080308A42
:10359000608047207082304600F0AAF82046103044
:1035A000F6F71AF8217F206A00F008F8308A002127
:1035B00004F492D3009809B0F0BD0000F3B583B0D5
:1035C0000020019004980125012845DD1621039A69
:1035D00069438818028A5204920F39D1039A4078BD
:1035E000515C000209181D48814231D101A80290A6
:1035F000EFB204264720FFF7B1F800900469002CD1
:1036000014D02079B8420BD16079B0420CD0009828
:1036100021461030F5F7E6FF204604F47DD105E0A1
:103620002468002CEDD101E0002C0AD130460121A4
:10363000083004F4FBD10446014600981030F5F739
:10364000D7FF277166713246A01D0299F4F70CFE70
:1036500004986D1C8542B9DB05B0F0BD022900005D
:10366000004870471453010170B5064610480D46D6
:10367000007800281AD04720FFF7B8F8A91D8BB2B0
:10368000014603220B4804F457D204460A482A464E
:10369000807820700120607005206080A580314610
:1036A000A01DF4F7E1FD204604F482D270BD0000B5
:1036B0003747002006470000D84D002070B584B081
:1036C0000E461446054601AA69463046FFF728FE15
:1036D0006846028802A80199F4F7C6FD02A844557D
:1036E0000246684601883046FFF758FE04B070BDB8
:1036F00010B504464720FFF731F80449216009213D
:103700006181183060600120208110BD24530101C7
:10371000FFB583B00C464720FFF720F805468088A8
:1037200061882678401887B2059804F4C3D201282E
:1037300007D03846FCF716FE6946FFF7DEFE002884
:1037400002D0022007B0F0BD0121059804F4C4D2D4
:103750000C3C0020AC60287368460078687301AAAE
:1037600002A9FFF7DDFDA86801990446895D0C34C4
:10377000890720D5A188C28808318BB23102C120C7
:103780000001891D04F4D8D1064613203070A888A2
:1037900061884018B080A088F0803046A288A11DC2
:1037A0000830F4F761FD304604F402D20121059897
:1037B00004F492D201E004F4AFD0012007B0F0BDD0
:1037C00010B5FAF749FB002010BDFFB583B00C46D9
:1037D0004720FEF7C3FF0546808861882678401899
:1037E00087B2059804F466D2012807D03846FCF762
:1037F000B9FD6946FFF781FE002802D0022007B01C
:10380000F0BD0C3CAC602E7368460078687301AA6A
:1038100002A9FFF785FDA86801990446895D0C346B
:10382000890720D0A188C28808318BB23102C1201B
:103830000001891D04F480D1064612203070A8884A
:1038400061884018B080A088F0803046A288A11D11
:103850000830F4F709FD304604F4AAD10121059897
:1038600004F43AD201E004F457D0012007B0F0BDCF
:1038700010B50C464720FEF771FF80886188A31DB4
:10388000401880B2A1880022FAF772FA002010BD19
:10389000F8B5488800900C468E88F9F7A9FB0028F7
:1038A0001DD0182E01D9182700E03746324626A031
:1038B0000099F8F77DFC0025002F08D9601981795F
:1038C0002AA0F8F775FC6D1CADB2BD42F6D3BE421E
:1038D00002D928A0F8F76CFC28A0F8F769FC00983A
:1038E000022821D0062804D0082822D00C2829D16B
:1038F00024E0022E26D1E0882149012802D00028A8
:1039000008D01FE001200870F9F772FB002819D0D9
:103910001CA006E000200870F9F76AFB002811D00F
:103920001EA0F8F745FC0DE0A188A01DF9F77CFB6F
:1039300008E0A188A01DF9F7BBFA03E0A188A01D4B
:10394000F9F792FF0020F8BD5B424C455D2077728D
:1039500069746520696E643A206174745F69647883
:103960003D2575206C656E3D2575000020253032A3
:1039700058000000202E2E2E000000000D0A00002E
:10398000374700205B424C455D206E6F7469667955
:1039900020656E61626C65640D0A00005B424C45F7
:1039A0005D206E6F746966792064697361626C650D
:1039B000640D0A00FFB581B000276846078048887B
:1039C0001C460D46082825D00C2828D00A282AD0C5
:1039D00005206946088016A66846008821460830FA
:1039E00083B21548039A04F4A7D087712978044656
:1039F000017068460288A28069886180002A03D02D
:103A00003146E01DF4F730FC204604F4D1D000200C
:103A100005B0F0BD6846F9F7C1FA0646DCE768462E
:103A2000F9F782FE02E06846F9F7E0FD0646D3E7C3
:103A30004E53494E470000000547000070B516463A
:103A40000C46104604F436D1012818D1A1791A4841
:103A5000002916D02178062309023246891D04F474
:103A60006BD00546A078FFF73AFD288080202871AA
:103A7000284604F49DD00021304604F42DD10020C6
:103A800070BDA1883246891D8BB221780902891D3B
:103A900004F452D00546A078FFF721FD28800020CD
:103AA0002871A0886880A288E11D681DF4F7DCFBFE
:103AB000284604F47DD0DEE7140C0000F3B583B093
:103AC00005001AD028680190284680380290C76FF8
:103AD00004983E1F864200D906462846F8F7BEFBEA
:103AE00004460091324629460498FCF721FE0199CC
:103AF000002806D0016005B0F0BD0498F8F7E0FB9F
:103B0000F9E729600299002CCF670AD02168621872
:103B1000291F8A4202D9291B091F2160009961606F
:103B2000E9E7024A00991160E5E700002848002013
:103B300010B5012400206407206003F453D72E48F9
:103B400002882E480168002003F4D8D72C48028848
:103B50002C480168012003F4D1D72B48008882B299
:103B60002A480168022003F4C9D72948008882B294
:103B700028480168032003F4C1D72748416AF0228E
:103B800011434162254816F4ABD726482449016009
:103B900025494161254981602549C16025498161E7
:103BA0002549C161264925488863FCF701FE206844
:103BB000C0B2F5F747FD23480078002806D0002062
:103BC00017F4D4D201460020F5F742FD2068C0B2B8
:103BD000F5F744FDF5F748FD2068C0B217F452D060
:103BE0002068C0B217F45CD02068C0B217F41AD2B3
:103BF0000120206010BD00001C01002018010020E1
:103C00002401002020010020340100203001002088
:103C10002C010020280100204025024074020020D1
:103C2000500250008080024000080F0058086A00CF
:103C3000420500000F0505060F000F034000D000ED
:103C40004080024062000020F0B5314C83B0E06952
:103C500080075AD502202062A56B082017F42AD3CA
:103C6000012017F435D32B4900270869401946086D
:103C7000B219801A086128480068F4F7D5FF0022BD
:103C8000264BF4F71DFF019100903E212846F5F7E1
:103C9000F1FC80197941F4F7D5FF019B009AF4F704
:103CA000A7FEF5F71BF805461D4A0023F4F794FA22
:103CB00006461B49F5F7DEFC1A49281A081A81B294
:103CC00022041948324342600160206B0821884376
:103CD00008432063A069072109078843A061A169FF
:103CE000012081430143A1612062FCF761FD0F487F
:103CF000104A0078410041180D4808184178D161F8
:103D00000D498078C8600D48077003B0F0BD000011
:103D100000800240A80200209000002000408F4058
:103D2000710200007002000040800240104000203C
:103D300034520101402502408025024080000020CD
:103D4000F0B587B004460D466846F7F757FEE60023
:103D50001F4C694630190746069080880090012064
:103D60000190A059F7F7EEFDB988A059F7F75DFE6D
:103D70006846F7F743FEED002F19B8880090012040
:103D8000019060596946F7F7DDFDB9886059F7F78A
:103D90004AFE1920F5F774FC6846F7F72FFE0698DF
:103DA0003146808800260196029600906058694648
:103DB000F7F7C8FD6846F7F721FEB8880196029626
:103DC000009060596946F7F7BDFD07B0F0BD0000EF
:103DD000A85A010100B50A4683B000210091019163
:103DE00001466846F5F719F90199009803B000BD3E
:103DF000704770474368826801699A6083684268C7
:103E00005A604A68824201D182684A600022026197
:103E10000868401E08600868704700000148006993
:103E200070470000CC470020F8B51746204A0646E8
:103E30000024906B0725401C90631069814232D3A7
:103E400014206D1E1B4968434118242060438019CB
:103E50000122FFF723F90419002DF1D12420144D7C
:103E60006043801902226968FFF718F904192420B9
:103E7000604380190222A968FFF710F90419242071
:103E80006043801904220C49FFF708F90419242023
:103E90006043801903220949FFF700F90419002F34
:103EA00001D00020386000F0DDFE2046F8BD0000A3
:103EB000CC470020006B0020C86B0020DC6B00208A
:103EC00010B500F0BDFD04490968401A0349884255
:103ED00001D2F7F717FE10BD38470020B80B0000DD
:103EE0000146083100224160D243C1608260016115
:103EF00000210160704700210161704730B40C68F7
:103F0000621C02D00246083202E0026904E01A464E
:103F100053681D68A542FAD953684B6099608A605E
:103F2000516008610168491C016030BC70474268FB
:103F30004A6093688B60936859609160086101687A
:103F4000491C01607047000072B604480168491CB2
:103F50000160BFF34F8FBFF36F8F70472048002081
:103F600005490868002804D0401E086000D162B6E8
:103F7000704772B6FEE700002048002000281CD0E1
:103F800070B504460D4D083C6068E968084201D1EF
:103F900072B6FEE72268002A01D072B6FEE78843B7
:103FA000606000F01BF9606869684018686020462E
:103FB000FFF74AF800F056FE70BD70470848002031
:103FC0000120044900074860BFF34F8FBFF36F8F94
:103FD0007047000000ED00E010B500280FD009493F
:103FE0008A6B002A01D072B6FEE78A6B521C8A6384
:103FF0000021FEF7D1FF00F035FE002801D1FFF7C8
:10400000DFFF10BDCC47002002498A6A026049697F
:1040100041607047CC470020F0B585B000270546C9
:1040200007702C4801690291006924214843FFF779
:10403000DFF806004CD000220299FFF7F5FE039747
:104040000290002841D90398242148438019017B1C
:10405000052911D20A007A44127992189744020471
:1040600006080A00582408E0522406E0422404E02E
:10407000532402E0442400E0002441682846F4F779
:1040800043F92846F4F714F90F2804D220212954C3
:10409000401C0F28FBD32F542D180398242148438C
:1040A0008019018C826801920091036922460AA15D
:1040B0002846F8F78DF82846F4F7FAF845190398DA
:1040C0000299401C03908842BDD33046FFF756FF4B
:1040D00005B0F0BDCC4700200925630925750925E9
:1040E000750925750D0A00000149012048627047D5
:1040F000CC47002010B50C46002809D005490968B6
:104100001831FFF7FBFE01212046FEF745FF10BDE9
:1041100072B6FEE7CC47002070B50B4604002FD0E6
:10412000226D002A0ED0E16C994200D21946E06A55
:10413000884225D0012A23D1124D2A68944203D106
:1041400072B6FEE772B6FEE7E162A269002A02DB00
:104150000722511AA16114220B4E50436169801944
:1041600081420DD1201DFFF745FEE06AA969884212
:1041700000D9A861142148438019211DFFF7D7FEFB
:1041800070BD0000CC470020006B002010B582B04D
:104190000D4800240190234680220CA100940D4874
:1041A00000F082FB012803D0401C0BD172B6FEE761
:1041B00072B600210848C94301630121C16144610D
:1041C00000F052F802B010BD0048002049444C45B0
:1041D00000000000F12F0101CC4700200248816B54
:1041E000491C816370470000CC470020164B986B38
:1041F000002802D001205862704700205862986958
:10420000142102464A4311498A58002A0AD100283B
:1042100006D01422401E42438A58002AF7D001E0FB
:1042200072B6FEE7142210B4424351184A680C4695
:10423000526808344A60A24201D152684A60D1688B
:104240001960986110BC7047CC470020006B0020BB
:104250000148406870470000084800200148806815
:10426000704700000848002070B50F48016AFF221F
:10427000120411430162016A1202114301620B4CE4
:1042800000252561A5610A487D21C9000068F3F772
:1042900079FF401E60610720206106480560F3F742
:1042A00027FF002070BD000000ED00E000E000E00E
:1042B000004000202048002010B5024600210120C7
:1042C00000F00CF8041E07D00021416001600B468D
:1042D0000A46C16000F05BF8204610BDF8B51746ED
:1042E0000E46050016D0002E16D070435030FEF753
:1042F0007FFF04000CD020465030002E0ED02060EE
:10430000266420460121E56300F00AF84C20075599
:104310002046F8BD72B6FEE70020E7E72460EFE72D
:1043200070B50D46040026D0FFF70EFE216CE06B41
:1043300048432168411861600021A1632168A160A0
:10434000E06B216C401E4843216822464118002042
:10435000C0434032E1601071507120461030002D92
:104360000BD0FFF7BDFD20462430FFF7B9FDFFF766
:10437000F7FD012070BD72B6FEE721690029F6D075
:1043800000F03EFC0028F2D0FFF71AFEEFE7FFB581
:10439000002783B00446002803D00498002802D0E8
:1043A00006E072B6FEE7206C002801D072B6FEE788
:1043B0000698022804D1E06B012801D072B6FEE70E
:1043C00000F02EFB002804D10598002801D072B619
:1043D000FEE720462546103040350290FFF7B4FD39
:1043E000A06BE16B884208D30698022805D0059897
:1043F00000284AD0002F4BD04EE0069E0499A56BB2
:104400000027226C002A11D0002E19D0E068F3F7A3
:104410002BFFE168206C091AE1602268914202D208
:104420006168081AE060022E17D019E020680028A1
:1044300016D1606800F074FB0746002060600FE052
:10444000A068F3F711FF216CA0684018A0606168B4
:10445000884205D32068A06002E0002D00D06D1EC8
:104460006D1CA563606A002806D02046243000F049
:10447000C7FB002802D103E0002F01D0FFF7A0FD09
:10448000FFF76EFD012007B0F0BDFFF769FD20E0EA
:104490006846FFF7B9FD0127FFF762FDFFF79EFEB3
:1044A000FFF752FD04202856401C00D1287105203A
:1044B0002856401C00D16871FFF752FD05A96846D7
:1044C00000F0C0F9002807D02046FEF757FE00F0A4
:1044D000C9FB002007B0F0BDFFF736FDA06BE16B14
:1044E000884201D1012600E00026FFF739FD002EA9
:1044F0000ED005990298FFF7FDFD2046FEF73EFE1F
:1045000000F0B0FB002800D068E7FFF759FD65E731
:104510002046FEF733FE00F0A5FB5FE770B50D46C1
:10452000040004D0206C002803D072B6FEE772B6F7
:10453000FEE72068002804D16068002801D072B628
:10454000FEE7F3F7E9FDA16B0646E06B884219D957
:104550002246403205201056491CA163411C03D05D
:10456000401C507101240EE0606A0028FAD02046F9
:10457000243000F045FB0028F4D0002DF2D00120BB
:104580002860EFE700243046F3F7CAFD204670BDEF
:10459000F7B5002784B00446002803D0059800280A
:1045A00002D006E072B6FEE7206C002801D072B699
:1045B000FEE700F035FA002804D10698002801D063
:1045C00072B6FEE720462546243040350290FFF7BC
:1045D000BBFCA66B002E21D0226C059B002A0BD0C1
:1045E000E0688018E0606168884201D32068E0607C
:1045F00001461846F3F738FE761EA66320690028A8
:1046000007D02046103000F0FBFA002801D0FFF759
:10461000D7FCFFF7A5FC012007B0F0BD06980028E5
:1046200002D0002F05D008E0FFF79AFC002007B069
:10463000F0BD6846FFF7E8FC0127FFF791FCFFF7A4
:10464000CDFDFFF781FC04202856401C00D12871C5
:1046500005202856401C00D16871FFF781FC06A98F
:10466000684600F0EFF8002811D02046FEF786FDDE
:1046700000F0F8FAFFF768FCA06B002827D00026AE
:10468000FFF76EFC002EA2D0002007B0F0BDFFF7B0
:104690005BFCA06B002812D00026FFF761FC002E07
:1046A0000FD006990298FFF725FD2046FEF766FD1C
:1046B00000F0D8FA00288AD1FFF782FC87E70126AC
:1046C000EBE72046FEF75AFD00F0CCFA7FE7012623
:1046D000D6E7F3B5002785B004460097002804D03C
:1046E000206C002803D072B6FEE772B6FEE700F039
:1046F00097F9002804D10698002801D072B6FEE789
:1047000020462546243040350190FFF71DFCA06B64
:10471000002817D0401EA0632068002802D1FEF7B1
:10472000E1FD60602069002807D02046103000F0CD
:1047300067FA002801D0FFF743FCFFF711FC0120C6
:1047400007B0F0BD0698002802D0002F0AD00DE077
:104750000098002801D072B6FEE7FFF701FC0020A8
:1047600007B0F0BD02A8FFF74FFC0127FFF7F8FBE9
:10477000FFF734FDFFF7E8FB04202856401C00D16A
:10478000287105202856401C00D16871FFF7E8FB0E
:1047900006A902A800F056F800281BD02046FEF714
:1047A000EDFC00F05FFAFFF7CFFBA06B00283ED0D6
:1047B0000026FFF7D5FB002EA7D0009800283ED09A
:1047C000FFF7C2FB606A002833D0206B0721006826
:1047D000091A2FE0FFF7B8FBA06B002808D00026CD
:1047E000FFF7BEFB002E1CD02068002802D009E095
:1047F0000126F5E7FFF7A8FB606800F0C5F9009017
:10480000FFF7AEFB06990198FFF774FC2046FEF710
:10481000B5FC00F027FA002800D076E7FFF7D0FBC0
:1048200073E72046FEF7AAFC00F01CFA6DE70126AC
:10483000BFE700216068FFF76FFCFFF791FB0020E6
:1048400007B0F0BDF8B50D46040012D0002D12D00F
:10485000FFF77AFB134E726963682868D11A471C08
:104860000BD02768B66AB74209D0934207D8012413
:1048700013E072B6FEE772B6FEE700240DE0884250
:1048800008D9401A28600748816A21604069606041
:10489000002402E0002001242860FFF761FB20468D
:1048A000F8BD0000CC470020FFB585B090000F9FF9
:1048B0000E9D0290FEF79CFC06001ED05C20FEF7C9
:1048C00097FC040016D02663059901910899009180
:1048D00030460299069EA5220391F3F7D7FC03996F
:1048E000206B091F4018C008C0000290400708D084
:1048F00072B6FEE73046FFF741FB0020C04309B027
:10490000F0BD2118325C20310A75315C002902D0DB
:10491000401C1028F5D3264600204036F070072DA5
:1049200000D30625E5620020E5642065201DFFF721
:10493000E2FA20461830FFF7DEFA24610720411B17
:104940006462A161002161653176009A0199029843
:10495000FEF7D4FC2060002F00D03C602546FFF716
:10496000F3FA284E3069401C30613068264F002829
:1049700003D0F069002821D026E035603069012895
:1049800022D1002414206043C019FFF7A9FA641C47
:10499000072CF7D31D48FFF7A3FA1D48FFF7A0FA2D
:1049A0001C48FFF79DFA1C48FFF79AFA1B48FFF7CF
:1049B00097FA164870601430B06005E03068E96A14
:1049C000C06A884200D83560F06A401CF0626864B2
:1049D000E86AB169884200D9B06114214843C0191E
:1049E000291DFFF7A4FAFFF7BBFAF069002806D0EB
:1049F0003068E96AC06A884201D2FFF7E1FA012013
:104A000009B0F0BDCC470020006B00208C6B00206B
:104A1000A06B0020B46B0020C86B0020DC6B002072
:104A20000648C169002904D0806B002803D000200B
:104A3000704701207047022070470000CC470020DB
:104A40000148406970470000CC470020F8B5324F5C
:104A50000026B86B002808D0386A401C3862786A93
:104A6000002800D001263046F8BD7D696D1C7D61AF
:104A700015D178680068002801D072B6FEE7786822
:104A8000B9687960B860B86A401CB8627868006834
:104A9000002813D07868C068C06840683863386BF5
:104AA000854211D37868006800280AD07868C06809
:104AB000C4686068854211D2386305E00020C043B5
:104AC000ECE70020C043386338681421C06A4843CB
:104AD000124908580128C2D90126C0E7201DFFF756
:104AE00089F9A06A002803D020461830FFF782F920
:104AF000E06AB969884200D9B8611421484307497E
:104B00004018211DFFF713FAE06A3968C96A884224
:104B1000C8D30126C6E70000CC470020006B002068
:104B200070B500210446002828D0154D286884421D
:104B300001D072B6FEE7206D002808D0401E206527
:104B4000E36CE26A9A4219D0002802D016E072B6ED
:104B5000FEE7201DFFF74EF9E06C0721E062081A1E
:104B6000A061E06AA969884200D9A861142148437C
:104B700004494018211DFFF7DAF90121084670BDEC
:104B8000CC470020006B002070B504460020002CAC
:104B90002AD0194DE16A2A68D26A914225D2A069C9
:104BA000002804DB28680721C06A081AA061E06AAF
:104BB0001422124E504361698019814210D1201D88
:104BC000FFF718F92868C06AE062A969884200D92D
:104BD000A861142148438019211DFFF7A8F902E0BC
:104BE0002868C06AE062012070BDE16C2A68D26A60
:104BF0009142F8D370BD0000CC470020006B00202C
:104C000070B5C068C468002C0BD02046183006462A
:104C1000FFF7F0F8104DA86B002804D031460F487C
:104C20000EE072B6FEE7201DFFF7E4F8E06AA9691E
:104C3000884200D9A8611421484309494018211D20
:104C4000FFF775F9E06A2968C96A884202D901202C
:104C5000686270BD002070BDCC470020B46B00209E
:104C6000006B0020F8B52E4D0027A86B002808D057
:104C7000FFF76AF9A86B401EA863A86B002802D052
:104C800046E072B6FEE72869002841D0254E30681C
:104C900000282AD0F068C46820461830FFF7AAF828
:104CA000201DFFF7A7F8E06AA969884200D9A8612A
:104CB000142148431C494018211DFFF738F9E06AC8
:104CC0002968C96A884201D30120686230680028D7
:104CD000E0D1002C09D068682946006800281BD064
:104CE0004868C068C068406808632C6A002C09D016
:104CF0000126FFF7ABFE002800D06E62641EF8D1DB
:104D000000202862686A002802D00127FFF758F9BE
:104D1000FFF726F93846F8BD0020C043E4E700005D
:104D2000CC470020B46B0020006B002040BA7047D5
:104D3000C0BA70470138FDD170470000F7B50325B0
:104D4000AD06286A82B016460C464008400028622C
:104D5000286A022108432862286A8007FCD466205A
:104D6000686001272F61A86AC005FCD5992068609A
:104D70002F61A86AC005FCD5FF209130FFF7DAFF4C
:104D8000FF230133AB626846EF60352169602F6114
:104D9000A96AC905FCD5AB62A969EF60C9B2052251
:104DA0006A602F61AA6AD205FCD5AB62AA690902C2
:104DB000D2B211430180C80702D0032005B0F0BD74
:104DC000AB626869FF210831884368616869C91E60
:104DD0000843686102980002483068600820A860B3
:104DE000EE602F61A86AC005FCD5FF200130A862E3
:104DF0000023F61CB0080ED0B208114800689900D4
:104E00006054060A09194E70060C000E8E705B1C69
:104E1000C8709A42F1D8FF200130A8626869FF216A
:104E2000083188436861686938436861286A800886
:104E300080002862286A38432862002005B0F0BD4F
:104E40008000000C032080064169FF220832914354
:104E50004161426901210A434261026A920892005B
:104E60000262026A0A4302627047000000200321C6
:104E70008906096A4908490003229206116211460F
:104E8000096A0222114303229206116200BF032124
:104E90008906096A022211400229F8D0D1010322B1
:104EA000920691620321D1609F215160012111611D
:104EB00000BF03218906896AFF2201321140914215
:104EC000F7D1032292069162114688694969FF224F
:104ED0000832914303229206516111464969012229
:104EE00011430322920651611146096A890889001B
:104EF00011621146096A01221143032292061162CE
:104F000070470000000001020000000001020304DD
:104F10000138FDD170470000F0B40324A406236AD1
:104F20005B085B002362236A02252B432362236A0A
:104F30009B07FCD4FF230133A3626569DE1DB543E3
:104F4000656165691E1D3543656100026B306060F7
:104F50000820A060E26001262661A06AC005FCD599
:104F6000A3620023D21C90080ED095080F48006859
:104F70009A008854070A52185770070C000E977051
:104F80005B1CD0709D42F1D86069FF2108318843D5
:104F90006061606930436061206A8008800020623F
:104FA000206A30432062F0BC002070478000000C73
:104FB000F8B5064601200025C004864201D9052027
:104FC000F8BD0324A406206A400840002062206A3D
:104FD000022108432062206A8007FCD4FF270137A2
:104FE000A76200F0BBF8002801D0032515E00620D9
:104FF000606001212161A06AC005FCD5A762300272
:10500000203060602161A06AC005FCD5A7620C4811
:1050100000F0C8F8002800D102256069FF2108319E
:10502000884360616069012108436061206A8008EB
:1050300080002062206A084320622846F8BD0000F4
:10504000E6960100F7B506460120C00482B0154679
:10505000864202D9052005B0F0BD03208006016A12
:10506000490849000162016A022211430162016A92
:105070008907FCD4FF2101318162F2B28C1AA5426A
:1050800000D8ACB20398009000F068F8002840D136
:1050900006214806416001210161816AC905FCD5EC
:1050A000FF2101310320800681624169FF2208321D
:1050B000914341614169042211434161310232311E
:1050C0004160C4600022002C16D9009887183B78F4
:1050D000F87819467B7800061B021943BB781B043D
:1050E000194301430802F978000A090608431949DF
:1050F0000860121DA242E8D301210320800601614D
:10510000816AC905FCD5FF2101318162124800F096
:1051100049F8A54209D00398361900192D1BFF2420
:1051200001340390A542ADD8ABE703208006416966
:10513000FF220832914341614169012211434161DB
:10514000016A890889000162016A11430162002035
:1051500005B0F0BD8000000C1A06000038B401252F
:10516000032080066A46C560352141600561816A79
:10517000C905FCD5FF24013484628169C560CBB2C6
:10518000052141600561816AC905FCD58462806999
:105190001902C0B2014388B21180C00700D00120BB
:1051A00038BC7047F8B400210125032292066B46F3
:1051B000D560352454601561946AE405FCD5FF2759
:1051C000013797629469D560E4B20526566015618F
:1051D000966AF605FCD5976296692402F6B23443C6
:1051E0001C80E30722D0814202D9F8BC002070471E
:1051F000032292066B46D560352454601561491C24
:10520000946AE405FCD597629469D560E4B20526FA
:1052100056601561966AF605FCD59762926924027C
:10522000D2B21443A2B21C80D207DCD1F8BC012058
:105230007047000000171300171000170E00170921
:1052400000170400170000171801171401171501A3
:1052500017190000002800020000000003280002C7
:1052600000000000292A00020080800003280002BC
:1052700000000000242A00020080800003280002B1
:1052800000000000252A00020080800003280002A0
:1052900000000000272A000200808000032800028E
:1052A00000000000262A000200808000032800027F
:1052B00000000000282A000200808000032800026D
:1052C00000000000232A00020080080003280002DA
:1052D000000000002A2A00020080080003280002C3
:1052E00000000000502A000200800700CDED000100
:1052F0005BED000159ED000157ED000100140000C5
:1053000075EE0001130C0000B10001010314000050
:1053100031EF0001233501019D34010151340101B8
:1053200005340101130C000075010101150C00008A
:1053300055020101170C00008DFF0001000C000058
:10534000CDFF000106470000CB37010103470000F5
:105350007138010108470000113701010E470000B4
:105360005D330101054700003D3A0101FFFF0000E8
:1053700031DB0001130E0000CDF20001150E00001C
:10538000DDF10001170E00004DF70001190E0000BD
:1053900025F700016C53010105000000F7B586B048
:1053A000002002905C48154604695C480E46824223
:1053B00001D9054602E0002D00D10125002C08D0BE
:1053C000A1880698814204D1E088B04201D1012031
:1053D000029053480390844606980104314300200C
:1053E000002C1CD00A0CA7888BB2974207D1E78803
:1053F0009F4204D1002807D02168016007E02046C1
:105400002468002CEFD10AE0614622680A60216816
:10541000002902D00020206001E061464860002C95
:1054200007D10221102000F095F8069981800446EA
:10543000C6802801052100F077F807467D200E463A
:105440004643EFF31085012080F31088684600F092
:1054500087F885F3108800980490C0190501019918
:1054600027202D098E1900010591864203D96D1C54
:105470002D012D09361AE660A5600398294F86464E
:105480000020844670460068002813D0A268E168B6
:105490000091C36881680193531A1B011B09BB4229
:1054A0000AD2914203D1019A0099914204D98446CB
:1054B0000068E9E77246546020606046002801D029
:1054C000046001E071460C601348029900690029EC
:1054D00001D1A04203D1C168806800F047F8EFF322
:1054E0001084012080F3108802A800F039F884F3BA
:1054F0001088039902980191291A0901090900905D
:10550000B94204D2A84205D10198864202D80320AC
:1055100000F032F809B0F0BDC8010020FFFF7F02A3
:10552000D8010020FFFFFF0730B50B4601460020E1
:105530002022012409E00D46D5409D4205D31D4699
:105540009540491B2546954040191546521E002D91
:10555000F1DC30BD03B40148019001BD2D7A01009A
:1055600003B40148019001BD5DB6020003B40148D7
:10557000019001BD9DB6020003B40148019001BD38
:10558000AD78010030B4C36882688868084D141A89
:105590002401C9682409AC4203D2904204D18B4251
:1055A00002D830BC0120704730BC0020704700009A
:1055B000FFFFFF070A0C838889B2934204D1C08899
:1055C000884201D1012070470020704770B4054621
:1055D00000680022002810D00B0C86888CB29E42F6
:1055E00007D1C688A64204D10168002A07D01160FD
:1055F00006E0024600680028EFD170BC70472960C1
:105600000168002903D00021016070BC70476A6006
:1056100070BC7047F0B5104F026886460025002A1E
:1056200010D0C8688C6893688446E01A00010009AD
:10563000D668B84208D2A34201D1B44504D9154670
:105640001268ECE7704641600A60002D01D02960C5
:10565000F0BD70460160F0BDFFFFFF0770B584B07C
:1056600004460E46EFF31085012080F3108802A84F
:10567000FFF776FF85F310880298039902460090A1
:105680000191A01A000107490009884204D2A242F0
:1056900005D10198864202D8012004B070BD0020D7
:1056A00004B070BDFFFFFF0730B583B00446EFF3D1
:1056B0001085012080F310886846FFF751FF85F3BD
:1056C0001088019900986160206003B030BD00002F
:1056D0000028000200000000032800020000000073
:1056E000002A000A008020000328000200000000B9
:1056F000012A0002008002000328000200000000CE
:10570000042A0002008008000328000200000000B4
:10571000A62A000200800100032800020000000009
:10572000C92A0002008001000028000200000000D9
:105730000328000200000000052A00200080040069
:105740000229000A000002000328000200000000F5
:10575000292B000A0080100003280002000000002E
:105760002A2B000200801000FFFF000015D400016A
:10577000A40D0000F1F90001A50D000025FA0001BB
:105780001A0D00003DFF0001150D000085FA000113
:10579000000D0000B1FA00011C0D000073FF0001B4
:1057A000A70D000091FE0001A80D00007FFF000181
:1057B000020C000065000101000C00003D00010129
:1057C000010E000069F500010F0E000025F900012F
:1057D000110E000089F900012C0E000009F90001EA
:1057E000030E0000C1F600010A0E00007DF8000162
:1057F000300E0000FDF800010C0E0000B1F90001B0
:10580000000E0000D5F40001090E0000FDF40001B7
:10581000010F000055D60001020F0000DDD200018B
:10582000030F000039D60001040F000049180101E0
:1058300068570101364700200100190002140000DA
:10584000ADEF00013C580101010000008459010145
:105850000300000001102EC78A0E7390E111C208E8
:105860006027000000280000000000000000000089
:1058700000000000000200000000032800000000FB
:1058800000000000000000000000000A000000000E
:1058900001002EC78A0E7390E111C2086027000034
:1058A000000400C000020129000000000000000008
:1058B000000000000000000A00801400032800001F
:1058C000000000000000000000000000000A0000CE
:1058D000000002002EC78A0E7390E111C2086027F3
:1058E0000000001000C000020229000000000000BB
:1058F0000000000000000000000A008014000328DF
:105900000000000000000000000000000000000A8D
:105910000000000003002EC78A0E7390E111C20838
:1059200060270000000A00C00002032800000000F9
:1059300000000000000000000000000A000000005D
:1059400004002EC78A0E7390E111C2086027000080
:10595000000200C000020328000000000000000058
:10596000000000000000000A0000000005002EC733
:105970008A0E7390E111C20860270000000A00C07F
:105980000002000004470000B53901010A47000089
:105990009138010107470000C1370101CC5F0101C7
:1059A000985F010111B10001685F0101505F0101C1
:1059B000F5B60001705F0101045E010159B50001F7
:1059C000845F0101D85C010155A80001E85E010176
:1059D000405D0101DDA70001745E0101405E01012F
:1059E000F5B100010C600101145D0101B99E0001D7
:1059F00024600101BC600101819F0001D45F0101AD
:105A0000F05E0101619B000134600101305C010125
:105A1000959B0001AC6001013C600101759800019B
:105A2000705E0101A05C0101C5B2000114600101BA
:105A3000B05D010125B500011C600101685C010138
:105A4000D9B20001DC5F0101B05E0101EDA90001E6
:105A50008C5F01011C5F0101A1AC00012C60010100
:105A60007C5D01011DAD0001B460010174600101A4
:105A70003DB00001A4600101785E0101B1B60001F2
:105A8000785F0101E45F010141B60001E05E0101C0
:105A9000D05D0101CDB0000101020304050607003D
:105AA000777C395E79710000000C01400100000034
:105AB000000C01400200000000080140010000004D
:105AC0000008014002000000000C01400008000036
:105AD000000C0140002000000008014040000000D0
:105AE0003F065B4F666D7D077F6F00404040404042
:105AF00040404040414141414140404040404040A1
:105B000040404040404040404040400502020202C8
:105B100002020202020202020202022020202020CF
:105B20002020202020020202020202029090909087
:105B30009090101010101010101010101010101065
:105B400010101010101002020202020288888888C9
:105B500088880808080808080808080808080808C5
:105B6000080808080808020202024000EB5A010176
:105B7000666C6F7720636F6E74726F6C3A206E6F15
:105B80006E653B2074783A20444D412043483120D3
:105B900028706F6C6C6564293B2072783A20444D04
:105BA00041204348322072696E672028334B422CD3
:105BB0002069646C6520697271290D0A000000007B
:105BC0005B6F74615D2062696E617279206D6F64D4
:105BD00065204F4E202D2073656E64203078434140
:105BE000204F5441206672616D6573206E6F770D92
:105BF0000A28626C655F70726F746F636F6C2E6DD4
:105C0000642073656374696F6E20362E363B204FB7
:105C100054415F41424F5254206F722033732069C8
:105C2000646C65206578697473290D0A00000000B2
:105C30006273736574203C6669656C643E203C76D3
:105C4000616C3E3A20777269746520626F6F74737D
:105C5000657474696E67206669656C642028636189
:105C6000726566756C21290070696E736574203CDD
:105C700070784E3E205B307C315D3A207365742F26
:105C800072656164204750494F206C6576656C20D1
:105C9000287061302D362F7062302D31332900008D
:105CA0006F74613A205541525420656E7465727369
:105CB000204F54412062696E617279206672616D75
:105CC00065206D6F646520287365652068656C705C
:105CD000206F74612900000073686F772064657617
:105CE00069636520696E666F202874656D702F7614
:105CF00064642F66616E2C2073616D652061732072
:105D0000424C4520494E464F5F51554552592061FE
:105D10006C6C2900617070676574205B6A736F6ECC
:105D20005D3A2073686F77206170702070617261D6
:105D30006D7320286C65642F70776D29000000005A
:105D4000626C656C6F67205B6F6E7C6F66665D3A38
:105D500020424C452074726166666963206C6F67EF
:105D600020286576656E7473202B206672616D65E0
:105D7000206865782064756D70290000646973700F
:105D8000736574203C70696E312D377C616C6C3E9C
:105D9000205B307C317C7A5D3A20647269766520C4
:105DA000646973706C61792070696E2873290000D2
:105DB00072657365743A2073797374656D207265CA
:105DC00073657420287265626F6F7429000000008B
:105DD00068616E673A20776564676520746865203E
:105DE000434C49207461736B2028495744472077FE
:105DF00061746368646F6720666972652074657397
:105E00007429000073686F77204672656552544F9D
:105E1000532072756E74696D6520696E666F2028F7
:105E2000757074696D652F7461736B732F6865612C
:105E3000702F7461736B206C69737429000000000B
:105E40006C6564203C317C323E203C6F6E7C6F661A
:105E5000667C746F67676C653E3A20636F6E747220
:105E60006F6C20626F617264204C4544000000003A
:105E70006F7461006C656400756172747273743A5A
:105E80002072652D696E697420555341525431203A
:105E90002834363038303020384E31292C20666C8A
:105EA0007573682072782071756575650000000053
:105EB00064697370203C76616C75653E205B665D3D
:105EC000205B6865785D3A2073657420372D7365B3
:105ED0006720646973706C61792076616C75650008
:105EE00068616E6700000000626C656C6F6700009F
:105EF000627364756D703A2073686F7720626F6F9C
:105F00007473657474696E67207265636F72642060
:105F10002B2063726320636865636B006469737030
:105F20006175746F205B6F6E7C6F66665D3A20658D
:105F30006E61626C652F64697361626C6520617566
:105F4000746F20646973706C6179207363616E0093
:105F500073686F77206669726D7761726520766508
:105F60007273696F6E00000076657273696F6E0000
:105F7000737973696E666F0075617274696E666FAE
:105F800000000000646576696E666F006469737076
:105F90006175746F0000000068656C70205B636D54
:105FA000645D3A206C69737420636F6D6D616E641B
:105FB00073202F2073686F77206F6E6520636F6D7D
:105FC0006D616E6427732068656C700068656C7025
:105FD00000000000627364756D7000006469737086
:105FE0000000000075617274696E666F3A20736814
:105FF0006F77205553415254312070696E732F6270
:106000006175642F666F726D6174000061707067F6
:1060100065740000726573657400000070696E73CA
:10602000657400006170707365740000646973705A
:10603000736574006273736574000000617070733F
:1060400077205B317C325D3A207377697463682016
:10605000626F6F742062616E6B20286372632076BA
:106060006572696669656429202B207265626F6FAD
:1060700074000000666163746F72793A2072657310
:10608000746F726520706172616D7320746F20642B
:10609000656661756C747320616E64207265626FF1
:1060A0006F74000075617274727374006170707344
:1060B00077000000666163746F72790061707073BD
:1060C0006574203C6C65647C70776D3E203C766125
:1060D0006C3E207C20617070736574206A736F6EF3
:1060E000207B226C6564223A3530307D0000000050
:1060F00075736167653A20617070736574203C6CDC
:1061000065647C70776D3E203C76616C3E207C201F
:10611000617070736574206A736F6E207B226C658A
:1061200064223A3530302C2270776D223A35307D3A
:106130000D0A000061707073773A2062616E6B2502
:106140006C7520696D61676520637263206D69738A
:106150006D6174636820287265636F7264203078A3
:106160002530386C582C2061637475616C20307850
:106170002530386C58290D0A00000000202020200E
:1061800020202020206231616464727C623261646C
:1061900064727C623173697A657C623273697A6594
:1061A0007C62316372637C62326372637C623176DB
:1061B00065727C6232766572203C6865787C6465C5
:1061C000633E0D0A00000000E8610101004000206C
:1061D00034080000449500010068010134480020A3
:1061E000BC750000F02A000011D490D00322A01A40
:1061F000FF01011013C202025420382B11D80D499F
:106200000868496813F008FB0498EFF78EFF04460E
:10621000C1888088FF22FFF79DFD2046FFF73AFCEA
:10622000B3E705B0F0BD981407D8011B20C80424BB
:1062300030D702100E4B1847FBFD06460520307084
:106240007580281699B181301D3946E5F773FD3008
:1062500046F9F70EFF0E222946422C45FD0740382D
:10626000112E0CD0534B052203212846FDF733FE97
:10627000121E134B75162D05D0398F142902D01418
:1062800099897912E01010211176FAF74BF8044D34
